LX51 LINKER/LOCATER V4.66.41.0                                                          06/16/2023  10:23:34  PAGE 1


LX51 LINKER/LOCATER V4.66.41.0, INVOKED BY:
C:\KEIL_V5\C51\BIN\LX51.EXE .\release\STARTUP.obj, .\release\main.obj, .\release\user.obj, .\release\key.obj, .\release\
>> port_mcu.obj, .\release\HS6220_RF.obj, .\release\register.obj, .\release\gpio.obj, .\release\timer.obj, .\release\uar
>> t.obj, .\release\pwm.obj, .\release\adc.obj, .\release\flash.obj, .\release\spi.obj, .\release\iic.obj TO .\release\B
>> L003C4 REGFILE (.\release\BL003C4.ORC) PRINT (.\release\listings\BL003C4.map) DISABLEWARNING (16) REMOVEUNUSED


CPU MODE:     8051 MODE
MEMORY MODEL: LARGE


INPUT MODULES INCLUDED:
  .\release\STARTUP.obj (?C_STARTUP)
         COMMENT TYPE 1: A51 / ASM51 Assembler
  .\release\main.obj (MAIN)
         COMMENT TYPE 0: C51 V9.54
  .\release\user.obj (USER)
         COMMENT TYPE 0: C51 V9.54
  .\release\key.obj (KEY)
         COMMENT TYPE 0: C51 V9.54
  .\release\port_mcu.obj (PORT_MCU)
         COMMENT TYPE 0: C51 V9.54
  .\release\HS6220_RF.obj (HS6220_RF)
         COMMENT TYPE 0: C51 V9.54
  .\release\register.obj (REGISTER)
         COMMENT TYPE 0: C51 V9.54
  .\release\gpio.obj (GPIO)
         COMMENT TYPE 0: C51 V9.54
  .\release\timer.obj (TIMER)
         COMMENT TYPE 0: C51 V9.54
  .\release\uart.obj (UART)
         COMMENT TYPE 0: C51 V9.54
  .\release\pwm.obj (PWM)
         COMMENT TYPE 0: C51 V9.54
  .\release\adc.obj (ADC)
         COMMENT TYPE 0: C51 V9.54
  .\release\flash.obj (FLASH)
         COMMENT TYPE 0: C51 V9.54
  .\release\spi.obj (SPI)
         COMMENT TYPE 0: C51 V9.54
  .\release\iic.obj (IIC)
         COMMENT TYPE 0: C51 V9.54
  C:\KEIL_V5\C51\LIB\C51L.LIB (?C_INIT)
         COMMENT TYPE 1: A51 / ASM51 Assembler
  C:\KEIL_V5\C51\LIB\C51L.LIB (?C?COPY)
         COMMENT TYPE 1: A51 / ASM51 Assembler
  C:\KEIL_V5\C51\LIB\C51L.LIB (?C?CLDPTR)
         COMMENT TYPE 1: A51 / ASM51 Assembler
  C:\KEIL_V5\C51\LIB\C51L.LIB (?C?CLDOPTR)
         COMMENT TYPE 1: A51 / ASM51 Assembler
  C:\KEIL_V5\C51\LIB\C51L.LIB (?C?CILDPTR)
         COMMENT TYPE 1: A51 / ASM51 Assembler
  C:\KEIL_V5\C51\LIB\C51L.LIB (?C?CSTPTR)
         COMMENT TYPE 1: A51 / ASM51 Assembler
  C:\KEIL_V5\C51\LIB\C51L.LIB (?C?CSTOPTR)
         COMMENT TYPE 1: A51 / ASM51 Assembler
  C:\KEIL_V5\C51\LIB\C51L.LIB (?C?IMUL)
         COMMENT TYPE 1: A51 / ASM51 Assembler
  C:\KEIL_V5\C51\LIB\C51L.LIB (?C?UIDIV)
         COMMENT TYPE 1: A51 / ASM51 Assembler
  C:\KEIL_V5\C51\LIB\C51L.LIB (?C?ILDIX)
         COMMENT TYPE 1: A51 / ASM51 Assembler
  C:\KEIL_V5\C51\LIB\C51L.LIB (?C?ULDIV)
         COMMENT TYPE 1: A51 / ASM51 Assembler
  C:\KEIL_V5\C51\LIB\C51L.LIB (?C?ULCMP)
         COMMENT TYPE 1: A51 / ASM51 Assembler
LX51 LINKER/LOCATER V4.66.41.0                                                        06/16/2023  10:23:34  PAGE 2


  C:\KEIL_V5\C51\LIB\C51L.LIB (?C?LSTXDATA)
         COMMENT TYPE 1: A51 / ASM51 Assembler
  C:\KEIL_V5\C51\LIB\C51L.LIB (?C?LSTKXDATA)
         COMMENT TYPE 1: A51 / ASM51 Assembler
  C:\KEIL_V5\C51\LIB\C51L.LIB (?C?LIMUL)
         COMMENT TYPE 1: A51 / ASM51 Assembler
  C:\KEIL_V5\C51\LIB\C51L.LIB (PRINTF)
         COMMENT TYPE 1: A51 / ASM51 Assembler
  C:\KEIL_V5\C51\LIB\C51L.LIB (?C?PLDIXDATA)
         COMMENT TYPE 1: A51 / ASM51 Assembler
  C:\KEIL_V5\C51\LIB\C51L.LIB (?C?PSTXDATA)
         COMMENT TYPE 1: A51 / ASM51 Assembler
  C:\KEIL_V5\C51\LIB\C51L.LIB (?C?CCASE)
         COMMENT TYPE 1: A51 / ASM51 Assembler


ACTIVE MEMORY CLASSES OF MODULE:  .\release\BL003C4 (?C_STARTUP)

BASE        START       END         USED      MEMORY CLASS
==========================================================
C:000000H   C:000000H   C:00FFFFH   001246H   CODE
I:000000H   I:000000H   I:0000FFH   000001H   IDATA
X:000000H   X:000000H   X:00FFFFH   000138H   XDATA
I:000020H.0 I:000020H.0 I:00002FH.7 000002H.1 BIT
C:000000H   C:000000H   C:00FFFFH             CONST
I:000000H   I:000000H   I:00007FH   00000DH   DATA


MEMORY MAP OF MODULE:  .\release\BL003C4 (?C_STARTUP)


START     STOP      LENGTH    ALIGN  RELOC    MEMORY CLASS   SEGMENT NAME
=========================================================================

* * * * * * * * * * *   D A T A   M E M O R Y   * * * * * * * * * * * * *
000000H   000007H   000008H   ---    AT..     DATA           "REG BANK 0"
000008H   00000CH   000005H   BYTE   UNIT     DATA           _DATA_GROUP_
00000DH.0 00001FH.7 000013H.0 ---    ---      **GAP**
000020H.0 000021H.0 000001H.1 BIT    UNIT     BIT            _BIT_GROUP_
000021H.1 000021H.4 000000H.4 BIT    UNIT     BIT            ?BI?KEY
000021H.5 000021H.7 000000H.3 BIT    UNIT     BIT            ?BI?USER
000022H.0 000022H.0 000000H.1 BIT    UNIT     BIT            ?BI?PORT_MCU
000022H.1 000022H   000000H.7 ---    ---      **GAP**
000023H   000023H   000001H   BYTE   UNIT     IDATA          ?STACK

* * * * * * * * * * *   C O D E   M E M O R Y   * * * * * * * * * * * * *
000000H   000002H   000003H   ---    OFFS..   CODE           ?CO??C_STARTUP?0
000003H   000005H   000003H   BYTE   OFFS..   CODE           ?GPIO?00003
000006H   000009H   000004H   BYTE   UNIT     CODE           ?PR?FEED_WATCHDOG?REGISTER
00000AH   00000AH   000001H   BYTE   UNIT     CODE           ?PR?INT0_RPT?GPIO
00000BH   00000DH   000003H   BYTE   OFFS..   CODE           ?TIMER?0000B
00000EH   000011H   000004H   BYTE   UNIT     CODE           ?PR?WDT_RPT?REGISTER
000012H   000012H   000001H   BYTE   UNIT     CODE           ?PR?INT1_RPT?GPIO
000013H   000015H   000003H   BYTE   OFFS..   CODE           ?GPIO?00013
000016H   000019H   000004H   BYTE   UNIT     CODE           ?PR?INT2_7_RPT?GPIO
00001AH   00001AH   000001H   BYTE   UNIT     CODE           ?PR?TIMER1_SERVICE?TIMER
00001BH   00001DH   000003H   BYTE   OFFS..   CODE           ?TIMER?0001B
00001EH   000021H   000004H   BYTE   UNIT     CODE           ?PR?INT8_15_RPT?GPIO
000022H   000022H   000001H   BYTE   UNIT     CODE           ?PR?TIMER4_SERVICE?TIMER
000023H   000025H   000003H   BYTE   OFFS..   CODE           ?UART?00023
000026H   000029H   000004H   BYTE   UNIT     CODE           ?PR?ADC_RPT?ADC
00002AH   00002AH   000001H   ---    ---      **GAP**
00002BH   00002DH   000003H   BYTE   OFFS..   CODE           ?REGISTER?0002B
00002EH   00003AH   00000DH   BYTE   UNIT     CODE           ?PR?_DELAY_US?PORT_MCU
00003BH   00003DH   000003H   BYTE   OFFS..   CODE           ?PORT_MCU?0003B
LX51 LINKER/LOCATER V4.66.41.0                                                        06/16/2023  10:23:34  PAGE 3


00003EH   000040H   000003H   BYTE   UNIT     CODE           ?PR?SYSTEM_FLOW_CONTROL?USER
000041H   000042H   000002H   ---    ---      **GAP**
000043H   000045H   000003H   BYTE   OFFS..   CODE           ?SPI?00043
000046H   00004AH   000005H   ---    ---      **GAP**
00004BH   00004DH   000003H   BYTE   OFFS..   CODE           ?TIMER?0004B
00004EH   000052H   000005H   ---    ---      **GAP**
000053H   000055H   000003H   BYTE   OFFS..   CODE           ?TIMER?00053
000056H   00005AH   000005H   ---    ---      **GAP**
00005BH   00005DH   000003H   BYTE   OFFS..   CODE           ?PWM?0005B
00005EH   000062H   000005H   ---    ---      **GAP**
000063H   000065H   000003H   BYTE   OFFS..   CODE           ?TIMER?00063
000066H   00006AH   000005H   ---    ---      **GAP**
00006BH   00006DH   000003H   BYTE   OFFS..   CODE           ?ADC?0006B
00006EH   000072H   000005H   ---    ---      **GAP**
000073H   000075H   000003H   BYTE   OFFS..   CODE           ?GPIO?00073
000076H   00007AH   000005H   ---    ---      **GAP**
00007BH   00007DH   000003H   BYTE   OFFS..   CODE           ?GPIO?0007B
00007EH   000082H   000005H   ---    ---      **GAP**
000083H   000085H   000003H   BYTE   OFFS..   CODE           ?IIC?00083
000086H   000423H   00039EH   BYTE   UNIT     CODE           ?C?LIB_CODE
000424H   000788H   000365H   BYTE   UNIT     CODE           ?PR?PRINTF?PRINTF
000789H   000856H   0000CEH   BYTE   UNIT     CODE           ?PR?TASK_KEY_SCAN?KEY
000857H   000924H   0000CEH   BYTE   UNIT     CODE           ?PR?IIC_RPT?IIC
000925H   0009D6H   0000B2H   BYTE   UNIT     CODE           ?PR?_UART1_RX_DATA_INT?UART
0009D7H   000A88H   0000B2H   BYTE   UNIT     CODE           ?PR?_ADC_SAMPLING_CONTINUOUS?ADC
000A89H   000B2FH   0000A7H   BYTE   UNIT     CODE           ?PR?_SPI_SLAVE_READ_INT?SPI
000B30H   000BC6H   000097H   BYTE   UNIT     CODE           ?PR?SYSTEM_TIMER_PRO?USER
000BC7H   000C52H   00008CH   BYTE   UNIT     CODE           ?C_C51STARTUP
000C53H   000CBEH   00006CH   BYTE   UNIT     CODE           ?PR?DEBUG_RPT?PORT_MCU
000CBFH   000D28H   00006AH   BYTE   UNIT     CODE           ?PR?_TURN_ON_PWM0_IDP?PWM
000D29H   000D81H   000059H   BYTE   UNIT     CODE           ?PR?SYSTEM_POWER_DOWN?PORT_MCU
000D82H   000DDAH   000059H   BYTE   UNIT     CODE           ?PR?TIMER5_SERVICE?TIMER
000DDBH   000E2FH   000055H   BYTE   UNIT     CODE           ?C_INITSEG
000E30H   000E81H   000052H   BYTE   UNIT     CODE           ?PR?SPI_RPT?SPI
000E82H   000ED0H   00004FH   BYTE   UNIT     CODE           ?PR?MAIN?MAIN
000ED1H   000F1FH   00004FH   BYTE   UNIT     CODE           ?PR?UART1_RPT?UART
000F20H   000F69H   00004AH   BYTE   UNIT     CODE           ?PR?USER_GPIO_INITIAL?USER
000F6AH   000FB2H   000049H   BYTE   UNIT     CODE           ?PR?_CONFIG_PWM0_MODULE?PWM
000FB3H   000FF2H   000040H   BYTE   UNIT     CODE           ?PR?RESET_CHECK?REGISTER
000FF3H   001030H   00003EH   BYTE   UNIT     CODE           ?PR?DEBUG_INIT?PORT_MCU
001031H   001069H   000039H   BYTE   UNIT     CODE           ?PR?TIMER3_SERVICE?TIMER
00106AH   0010A0H   000037H   BYTE   UNIT     CODE           ?CO?MAIN
0010A1H   0010D5H   000035H   BYTE   UNIT     CODE           ?PR?USER_KEY_PRO?USER
0010D6H   001109H   000034H   BYTE   UNIT     CODE           ?PR?_TURN_OFF_PWM0?PWM
00110AH   00113CH   000033H   BYTE   UNIT     CODE           ?PR?_USER_PRINTF?PORT_MCU
00113DH   00116BH   00002FH   BYTE   UNIT     CODE           ?PR?TIMER0_SERVICE?TIMER
00116CH   001195H   00002AH   BYTE   UNIT     CODE           ?PR?CONFIG_SYSCLK_IHRC_MODULE?REGISTER
001196H   0011BAH   000025H   BYTE   UNIT     CODE           ?PR?PWM_RPT?PWM
0011BBH   0011D9H   00001FH   BYTE   UNIT     CODE           ?PR?CONFIG_ADC_MODULE?ADC
0011DAH   0011F1H   000018H   BYTE   UNIT     CODE           ?PR?_PUTCHAR?PORT_MCU
0011F2H   001205H   000014H   BYTE   UNIT     CODE           ?PR?_DEBUG_PUTCHAR?PORT_MCU
001206H   001219H   000014H   BYTE   UNIT     CODE           ?PR?HARDWARE_INIT?PORT_MCU
00121AH   00122DH   000014H   BYTE   UNIT     CODE           ?PR?CONFIG_TIMER0_MODULE?TIMER
00122EH   00123FH   000012H   BYTE   UNIT     CODE           ?PR?USER_REGISTER_INITIAL?USER
001240H   00124FH   000010H   BYTE   UNIT     CODE           ?PR?ADC_SAMPLING_SINGLE?ADC
001250H   00125EH   00000FH   BYTE   UNIT     CODE           ?CO?USER
00125FH   001268H   00000AH   BYTE   UNIT     CODE           ?PR?ENABLE_WATCHDOG?REGISTER
001269H   001270H   000008H   BYTE   UNIT     CODE           ?PR?DISABLE_WATCHDOG?REGISTER

* * * * * * * * * * *  X D A T A   M E M O R Y  * * * * * * * * * * * * *
000000H   000039H   00003AH   BYTE   UNIT     XDATA          _XDATA_GROUP_
00003AH   00006FH   000036H   BYTE   UNIT     XDATA          ?XD?USER
000070H   000080H   000011H   BYTE   UNIT     XDATA          ?XD?ADC
000081H   00008DH   00000DH   BYTE   UNIT     XDATA          ?XD?PWM
00008EH   000097H   00000AH   BYTE   UNIT     XDATA          ?XD?IIC
LX51 LINKER/LOCATER V4.66.41.0                                                        06/16/2023  10:23:34  PAGE 4


000098H   00009FH   000008H   BYTE   UNIT     XDATA          ?XD?SPI
0000A0H   0000A6H   000007H   BYTE   UNIT     XDATA          ?XD?KEY
0000A7H   0000ADH   000007H   BYTE   UNIT     XDATA          ?XD?UART
0000AEH   0000B1H   000004H   BYTE   UNIT     XDATA          ?XD?REGISTER
0000B2H   0000B4H   000003H   BYTE   UNIT     XDATA          ?XD?PORT_MCU
0000B5H   0000B7H   000003H   BYTE   UNIT     XDATA          ?XD?HS6220_RF
0000B8H   0000BAH   000003H   BYTE   UNIT     XDATA          ?XD?TIMER
0000BBH   00FE7FH   00FDC5H   ---    ---      **GAP**
00FE80H   00FE80H   000001H   BYTE   OFFS..   XDATA          ?XD?MAIN?86
00FE81H   00FE83H   000003H   ---    ---      **GAP**
00FE84H   00FE84H   000001H   BYTE   OFFS..   XDATA          ?XD?MAIN?23
00FE85H   00FE85H   000001H   BYTE   OFFS..   XDATA          ?XD?MAIN?25
00FE86H   00FE86H   000001H   BYTE   OFFS..   XDATA          ?XD?MAIN?26
00FE87H   00FE87H   000001H   ---    ---      **GAP**
00FE88H   00FE88H   000001H   BYTE   OFFS..   XDATA          ?XD?MAIN?85
00FE89H   00FE89H   000001H   BYTE   OFFS..   XDATA          ?XD?MAIN?22
00FE8AH   00FE8AH   000001H   BYTE   OFFS..   XDATA          ?XD?MAIN?72
00FE8BH   00FE8BH   000001H   BYTE   OFFS..   XDATA          ?XD?MAIN?55
00FE8CH   00FE90H   000005H   ---    ---      **GAP**
00FE91H   00FE91H   000001H   BYTE   OFFS..   XDATA          ?XD?MAIN?41
00FE92H   00FE92H   000001H   BYTE   OFFS..   XDATA          ?XD?MAIN?99
00FE93H   00FE93H   000001H   BYTE   OFFS..   XDATA          ?XD?MAIN?60
00FE94H   00FE94H   000001H   BYTE   OFFS..   XDATA          ?XD?MAIN?17
00FE95H   00FE95H   000001H   BYTE   OFFS..   XDATA          ?XD?MAIN?37
00FE96H   00FE96H   000001H   BYTE   OFFS..   XDATA          ?XD?MAIN?102
00FE97H   00FE97H   000001H   BYTE   OFFS..   XDATA          ?XD?MAIN?97
00FE98H   00FE98H   000001H   BYTE   OFFS..   XDATA          ?XD?MAIN?71
00FE99H   00FE99H   000001H   ---    ---      **GAP**
00FE9AH   00FE9AH   000001H   BYTE   OFFS..   XDATA          ?XD?MAIN?40
00FE9BH   00FE9BH   000001H   BYTE   OFFS..   XDATA          ?XD?MAIN?39
00FE9CH   00FE9CH   000001H   BYTE   OFFS..   XDATA          ?XD?MAIN?122
00FE9DH   00FE9DH   000001H   BYTE   OFFS..   XDATA          ?XD?MAIN?4
00FE9EH   00FE9EH   000001H   BYTE   OFFS..   XDATA          ?XD?MAIN?61
00FE9FH   00FE9FH   000001H   BYTE   OFFS..   XDATA          ?XD?MAIN?116
00FEA0H   00FEA0H   000001H   BYTE   OFFS..   XDATA          ?XD?MAIN?50
00FEA1H   00FEA1H   000001H   ---    ---      **GAP**
00FEA2H   00FEA2H   000001H   BYTE   OFFS..   XDATA          ?XD?MAIN?24
00FEA3H   00FEA3H   000001H   ---    ---      **GAP**
00FEA4H   00FEA4H   000001H   BYTE   OFFS..   XDATA          ?XD?MAIN?29
00FEA5H   00FEA5H   000001H   BYTE   OFFS..   XDATA          ?XD?MAIN?31
00FEA6H   00FEA6H   000001H   ---    ---      **GAP**
00FEA7H   00FEA7H   000001H   BYTE   OFFS..   XDATA          ?XD?MAIN?34
00FEA8H   00FEA9H   000002H   ---    ---      **GAP**
00FEAAH   00FEAAH   000001H   BYTE   OFFS..   XDATA          ?XD?MAIN?45
00FEABH   00FEABH   000001H   BYTE   OFFS..   XDATA          ?XD?MAIN?38
00FEACH   00FEACH   000001H   BYTE   OFFS..   XDATA          ?XD?MAIN?7
00FEADH   00FEADH   000001H   BYTE   OFFS..   XDATA          ?XD?MAIN?11
00FEAEH   00FEAEH   000001H   BYTE   OFFS..   XDATA          ?XD?MAIN?10
00FEAFH   00FEAFH   000001H   BYTE   OFFS..   XDATA          ?XD?MAIN?16
00FEB0H   00FEB0H   000001H   BYTE   OFFS..   XDATA          ?XD?MAIN?103
00FEB1H   00FEB1H   000001H   BYTE   OFFS..   XDATA          ?XD?MAIN?105
00FEB2H   00FEB2H   000001H   BYTE   OFFS..   XDATA          ?XD?MAIN?106
00FEB3H   00FEB3H   000001H   BYTE   OFFS..   XDATA          ?XD?MAIN?108
00FEB4H   00FEB7H   000004H   ---    ---      **GAP**
00FEB8H   00FEB8H   000001H   BYTE   OFFS..   XDATA          ?XD?MAIN?35
00FEB9H   00FEB9H   000001H   BYTE   OFFS..   XDATA          ?XD?MAIN?36
00FEBAH   00FEBBH   000002H   ---    ---      **GAP**
00FEBCH   00FEBCH   000001H   BYTE   OFFS..   XDATA          ?XD?MAIN?96
00FEBDH   00FEBDH   000001H   BYTE   OFFS..   XDATA          ?XD?MAIN?14
00FEBEH   00FEBEH   000001H   BYTE   OFFS..   XDATA          ?XD?MAIN?52
00FEBFH   00FEBFH   000001H   ---    ---      **GAP**
00FEC0H   00FEC0H   000001H   BYTE   OFFS..   XDATA          ?XD?MAIN?65
00FEC1H   00FEC1H   000001H   BYTE   OFFS..   XDATA          ?XD?MAIN?79
00FEC2H   00FEC2H   000001H   BYTE   OFFS..   XDATA          ?XD?MAIN?68
00FEC3H   00FEC3H   000001H   BYTE   OFFS..   XDATA          ?XD?MAIN?84
LX51 LINKER/LOCATER V4.66.41.0                                                        06/16/2023  10:23:34  PAGE 5


00FEC4H   00FEC4H   000001H   BYTE   OFFS..   XDATA          ?XD?MAIN?70
00FEC5H   00FEC5H   000001H   BYTE   OFFS..   XDATA          ?XD?MAIN?91
00FEC6H   00FEC6H   000001H   BYTE   OFFS..   XDATA          ?XD?MAIN?74
00FEC7H   00FEC7H   000001H   BYTE   OFFS..   XDATA          ?XD?MAIN?93
00FEC8H   00FEC8H   000001H   BYTE   OFFS..   XDATA          ?XD?MAIN?78
00FEC9H   00FEC9H   000001H   BYTE   OFFS..   XDATA          ?XD?MAIN?95
00FECAH   00FECAH   000001H   BYTE   OFFS..   XDATA          ?XD?MAIN?83
00FECBH   00FECBH   000001H   BYTE   OFFS..   XDATA          ?XD?MAIN?98
00FECCH   00FECCH   000001H   BYTE   OFFS..   XDATA          ?XD?MAIN?90
00FECDH   00FECDH   000001H   BYTE   OFFS..   XDATA          ?XD?MAIN?100
00FECEH   00FECEH   000001H   BYTE   OFFS..   XDATA          ?XD?MAIN?92
00FECFH   00FECFH   000001H   BYTE   OFFS..   XDATA          ?XD?MAIN?101
00FED0H   00FED0H   000001H   BYTE   OFFS..   XDATA          ?XD?MAIN?53
00FED1H   00FED1H   000001H   BYTE   OFFS..   XDATA          ?XD?MAIN?57
00FED2H   00FED2H   000001H   BYTE   OFFS..   XDATA          ?XD?MAIN?54
00FED3H   00FED3H   000001H   BYTE   OFFS..   XDATA          ?XD?MAIN?58
00FED4H   00FED7H   000004H   ---    ---      **GAP**
00FED8H   00FED8H   000001H   BYTE   OFFS..   XDATA          ?XD?MAIN?82
00FED9H   00FED9H   000001H   BYTE   OFFS..   XDATA          ?XD?MAIN?89
00FEDAH   00FEDFH   000006H   ---    ---      **GAP**
00FEE0H   00FEE0H   000001H   BYTE   OFFS..   XDATA          ?XD?MAIN?64
00FEE1H   00FEE1H   000001H   BYTE   OFFS..   XDATA          ?XD?MAIN?77
00FEE2H   00FEE2H   000001H   BYTE   OFFS..   XDATA          ?XD?MAIN?67
00FEE3H   00FEE3H   000001H   BYTE   OFFS..   XDATA          ?XD?MAIN?81
00FEE4H   00FEE4H   000001H   BYTE   OFFS..   XDATA          ?XD?MAIN?69
00FEE5H   00FEE5H   000001H   BYTE   OFFS..   XDATA          ?XD?MAIN?88
00FEE6H   00FEE7H   000002H   ---    ---      **GAP**
00FEE8H   00FEE8H   000001H   BYTE   OFFS..   XDATA          ?XD?MAIN?111
00FEE9H   00FEE9H   000001H   BYTE   OFFS..   XDATA          ?XD?MAIN?112
00FEEAH   00FEEAH   000001H   BYTE   OFFS..   XDATA          ?XD?MAIN?115
00FEEBH   00FEEDH   000003H   ---    ---      **GAP**
00FEEEH   00FEEEH   000001H   BYTE   OFFS..   XDATA          ?XD?MAIN?62
00FEEFH   00FEEFH   000001H   ---    ---      **GAP**
00FEF0H   00FEF0H   000001H   BYTE   OFFS..   XDATA          ?XD?MAIN?56
00FEF1H   00FEF1H   000001H   BYTE   OFFS..   XDATA          ?XD?MAIN?59
00FEF2H   00FEF7H   000006H   ---    ---      **GAP**
00FEF8H   00FEF8H   000001H   BYTE   OFFS..   XDATA          ?XD?MAIN?51
00FEF9H   00FEF9H   000001H   BYTE   OFFS..   XDATA          ?XD?MAIN?12
00FEFAH   00FEFAH   000001H   BYTE   OFFS..   XDATA          ?XD?MAIN?13
00FEFBH   00FEFBH   000001H   BYTE   OFFS..   XDATA          ?XD?MAIN?15
00FEFCH   00FEFFH   000004H   ---    ---      **GAP**
00FF00H   00FF00H   000001H   BYTE   OFFS..   XDATA          ?XD?MAIN?124
00FF01H   00FF01H   000001H   BYTE   OFFS..   XDATA          ?XD?MAIN?1
00FF02H   00FF02H   000001H   BYTE   OFFS..   XDATA          ?XD?MAIN?3
00FF03H   00FF03H   000001H   BYTE   OFFS..   XDATA          ?XD?MAIN?6
00FF04H   00FF04H   000001H   ---    ---      **GAP**
00FF05H   00FF05H   000001H   BYTE   OFFS..   XDATA          ?XD?MAIN?104
00FF06H   00FF07H   000002H   ---    ---      **GAP**
00FF08H   00FF08H   000001H   BYTE   OFFS..   XDATA          ?XD?MAIN?0
00FF09H   00FF0FH   000007H   ---    ---      **GAP**
00FF10H   00FF10H   000001H   BYTE   OFFS..   XDATA          ?XD?MAIN?2
00FF11H   00FF11H   000001H   BYTE   OFFS..   XDATA          ?XD?MAIN?5
00FF12H   00FF12H   000001H   BYTE   OFFS..   XDATA          ?XD?MAIN?8
00FF13H   00FF13H   000001H   BYTE   OFFS..   XDATA          ?XD?MAIN?9
00FF14H   00FF3FH   00002CH   ---    ---      **GAP**
00FF40H   00FF40H   000001H   BYTE   OFFS..   XDATA          ?XD?MAIN?119
00FF41H   00FF41H   000001H   BYTE   OFFS..   XDATA          ?XD?MAIN?121
00FF42H   00FF42H   000001H   BYTE   OFFS..   XDATA          ?XD?MAIN?123
00FF43H   00FF4FH   00000DH   ---    ---      **GAP**
00FF50H   00FF50H   000001H   BYTE   OFFS..   XDATA          ?XD?MAIN?117
00FF51H   00FF51H   000001H   BYTE   OFFS..   XDATA          ?XD?MAIN?118
00FF52H   00FF52H   000001H   BYTE   OFFS..   XDATA          ?XD?MAIN?120
00FF53H   00FF5FH   00000DH   ---    ---      **GAP**
00FF60H   00FF60H   000001H   BYTE   OFFS..   XDATA          ?XD?MAIN?107
00FF61H   00FF61H   000001H   BYTE   OFFS..   XDATA          ?XD?MAIN?109
LX51 LINKER/LOCATER V4.66.41.0                                                        06/16/2023  10:23:34  PAGE 6


00FF62H   00FF62H   000001H   BYTE   OFFS..   XDATA          ?XD?MAIN?110
00FF63H   00FF7FH   00001DH   ---    ---      **GAP**
00FF80H   00FF80H   000001H   BYTE   OFFS..   XDATA          ?XD?MAIN?42
00FF81H   00FF81H   000001H   BYTE   OFFS..   XDATA          ?XD?MAIN?44
00FF82H   00FF82H   000001H   ---    ---      **GAP**
00FF83H   00FF83H   000001H   BYTE   OFFS..   XDATA          ?XD?MAIN?47
00FF84H   00FF84H   000001H   BYTE   OFFS..   XDATA          ?XD?MAIN?48
00FF85H   00FF85H   000001H   BYTE   OFFS..   XDATA          ?XD?MAIN?49
00FF86H   00FF87H   000002H   ---    ---      **GAP**
00FF88H   00FF88H   000001H   BYTE   OFFS..   XDATA          ?XD?MAIN?43
00FF89H   00FF89H   000001H   BYTE   OFFS..   XDATA          ?XD?MAIN?46
00FF8AH   00FF8CH   000003H   ---    ---      **GAP**
00FF8DH   00FF8DH   000001H   BYTE   OFFS..   XDATA          ?XD?MAIN?33
00FF8EH   00FF8EH   000001H   ---    ---      **GAP**
00FF8FH   00FF8FH   000001H   BYTE   OFFS..   XDATA          ?XD?MAIN?94
00FF90H   00FF90H   000001H   BYTE   OFFS..   XDATA          ?XD?MAIN?73
00FF91H   00FF91H   000001H   BYTE   OFFS..   XDATA          ?XD?MAIN?18
00FF92H   00FF93H   000002H   ---    ---      **GAP**
00FF94H   00FF94H   000001H   BYTE   OFFS..   XDATA          ?XD?MAIN?76
00FF95H   00FF95H   000001H   BYTE   OFFS..   XDATA          ?XD?MAIN?19
00FF96H   00FF97H   000002H   ---    ---      **GAP**
00FF98H   00FF98H   000001H   BYTE   OFFS..   XDATA          ?XD?MAIN?80
00FF99H   00FF99H   000001H   BYTE   OFFS..   XDATA          ?XD?MAIN?21
00FF9AH   00FF9BH   000002H   ---    ---      **GAP**
00FF9CH   00FF9CH   000001H   BYTE   OFFS..   XDATA          ?XD?MAIN?87
00FF9DH   00FF9FH   000003H   ---    ---      **GAP**
00FFA0H   00FFA0H   000001H   BYTE   OFFS..   XDATA          ?XD?MAIN?32
00FFA1H   00FFA1H   000001H   BYTE   OFFS..   XDATA          ?XD?MAIN?30
00FFA2H   00FFA2H   000001H   BYTE   OFFS..   XDATA          ?XD?MAIN?28
00FFA3H   00FFA3H   000001H   BYTE   OFFS..   XDATA          ?XD?MAIN?20
00FFA4H   00FFA4H   000001H   BYTE   OFFS..   XDATA          ?XD?MAIN?75
00FFA5H   00FFA5H   000001H   BYTE   OFFS..   XDATA          ?XD?MAIN?27
00FFA6H   00FFA6H   000001H   BYTE   OFFS..   XDATA          ?XD?MAIN?114
00FFA7H   00FFA7H   000001H   BYTE   OFFS..   XDATA          ?XD?MAIN?113
00FFA8H   00FFA8H   000001H   BYTE   OFFS..   XDATA          ?XD?MAIN?66
00FFA9H   00FFA9H   000001H   BYTE   OFFS..   XDATA          ?XD?MAIN?63

* * * * * * * * *   R E M O V E D     S E G M E N T S   * * * * * * * *
   *DEL*:           000051H   BYTE   UNIT     CODE           ?PR?USER_RFTX_PRO?USER
   *DEL*:           000052H   BYTE   UNIT     CODE           ?PR?USER_RFRX_PRO?USER
   *DEL*:           00001EH   BYTE   UNIT     CODE           ?PR?_DELAY_MS?PORT_MCU
   *DEL*:           000013H   BYTE   UNIT     CODE           ?PR?_DELAY_MS_INT?PORT_MCU
   *DEL*:           00002BH   BYTE   UNIT     CODE           ?PR?HS6220_SPI_INIT?HS6220_RF
   *DEL*:           000038H   BYTE   UNIT     CODE           ?PR?_SPI_3WIRE_SENDBYTE?HS6220_RF
   *DEL*:           000026H   BYTE   UNIT     CODE           ?PR?SPI_3WIRE_READBYTE?HS6220_RF
   *DEL*:           000006H   BYTE   UNIT     CODE           ?PR?_SPI_SENDBYTE?HS6220_RF
   *DEL*:           000004H   BYTE   UNIT     CODE           ?PR?SPI_READBYTE?HS6220_RF
   *DEL*:           000015H   BYTE   UNIT     CODE           ?PR?_HS6220_WRITE_BYTE?HS6220_RF
   *DEL*:           000040H   BYTE   UNIT     CODE           ?PR?_HS6220_WR_BUFFER?HS6220_RF
   *DEL*:           000005H   BYTE   UNIT     XDATA          ?XD?_HS6220_WR_BUFFER?HS6220_RF
   *DEL*:           00000AH   BYTE   UNIT     CODE           ?PR?_HS6220_READ_BYTE?HS6220_RF
   *DEL*:           000035H   BYTE   UNIT     CODE           ?PR?_HS6220_READ_BUFFER?HS6220_RF
   *DEL*:           000005H   BYTE   UNIT     XDATA          ?XD?_HS6220_READ_BUFFER?HS6220_RF
   *DEL*:           00000AH   BYTE   UNIT     CODE           ?PR?_HS6220_OPERATION?HS6220_RF
   *DEL*:           00014DH   BYTE   UNIT     CODE           ?PR?HS6220_INIT?HS6220_RF
   *DEL*:           000005H   BYTE   UNIT     XDATA          ?XD?HS6220_INIT?HS6220_RF
   *DEL*:           000011H   BYTE   UNIT     CODE           ?PR?_HS6220_WR_CMD?HS6220_RF
   *DEL*:           00001CH   BYTE   UNIT     CODE           ?PR?_HS6220_BANK_SWITCH?HS6220_RF
   *DEL*:           00001DH   BYTE   UNIT     CODE           ?PR?_HS6220_CHANGE_RATE?HS6220_RF
   *DEL*:           00000EH   BYTE   UNIT     CODE           ?PR?_HS6220_CHANGE_CH?HS6220_RF
   *DEL*:           00003AH   BYTE   UNIT     CODE           ?PR?_HS6220_CHANGE_PWR?HS6220_RF
   *DEL*:           00000BH   BYTE   UNIT     CODE           ?PR?_HS6220_CHANGE_ADDR?HS6220_RF
   *DEL*:           0000A8H   BYTE   UNIT     CODE           ?PR?_HS6220_RECEIVEPACK?HS6220_RF
   *DEL*:           000001H   BYTE   UNIT     XDATA          ?XD?_HS6220_RECEIVEPACK?HS6220_RF
   *DEL*:           000028H   BYTE   UNIT     CODE           ?PR?_HS6220_SENDPACK?HS6220_RF
LX51 LINKER/LOCATER V4.66.41.0                                                        06/16/2023  10:23:34  PAGE 7


   *DEL*:           000005H   BYTE   UNIT     XDATA          ?XD?_HS6220_SENDPACK?HS6220_RF
   *DEL*:           00002BH   BYTE   UNIT     CODE           ?PR?_HS6220_MODESWITCH?HS6220_RF
   *DEL*:           000007H   BYTE   UNIT     CODE           ?PR?HS6220_CLEAR_ALL_IRQ?HS6220_RF
   *DEL*:           000005H   BYTE   UNIT     CODE           ?PR?HS6220_FLUSH_TX?HS6220_RF
   *DEL*:           000005H   BYTE   UNIT     CODE           ?PR?HS6220_FLUSH_RX?HS6220_RF
   *DEL*:           000005H   BYTE   UNIT     CODE           ?PR?HS6220_CE_HIGH?HS6220_RF
   *DEL*:           000005H   BYTE   UNIT     CODE           ?PR?HS6220_CE_LOW?HS6220_RF
   *DEL*:           000006H   BYTE   UNIT     CODE           ?PR?HS6220_READ_PAYLOAD_LENGTH?HS6220_RF
   *DEL*:           00002AH   BYTE   UNIT     CODE           ?PR?CONFIG_SYSCLK_CRYSTAL_MODULE?REGISTER
   *DEL*:           000015H   BYTE   UNIT     CODE           ?PR?CONFIG_SYSCLK_OUTPUT?REGISTER
   *DEL*:           00000CH   BYTE   UNIT     CODE           ?PR?ENABLE_WATCHDOG_FOR_STOP?REGISTER
   *DEL*:           00001FH   BYTE   UNIT     CODE           ?PR?_HD_CRC_CALCULATE?REGISTER
   *DEL*:           000030H   BYTE   UNIT     CODE           ?PR?CONFIG_GPIO_POWER_ON?GPIO
   *DEL*:           00007FH   BYTE   UNIT     CODE           ?PR?CONFIG_GPIO_EXT_INT?GPIO
   *DEL*:           000017H   BYTE   UNIT     CODE           ?PR?CONFIG_TIMER1_MODULE?TIMER
   *DEL*:           00001BH   BYTE   UNIT     CODE           ?PR?CONFIG_TIMER3_MODULE?TIMER
   *DEL*:           000025H   BYTE   UNIT     CODE           ?PR?CONFIG_TIMER4_MODULE?TIMER
   *DEL*:           00001FH   BYTE   UNIT     CODE           ?PR?CONFIG_TIMER5_MODULE?TIMER
   *DEL*:           000058H   BYTE   UNIT     CODE           ?PR?_CONFIG_UART1_MODULE?UART
   *DEL*:           00000BH   BYTE   UNIT     CODE           ?PR?_UART1_TX_BYTE?UART
   *DEL*:           000033H   BYTE   UNIT     CODE           ?PR?_UART1_TX_DATA?UART
   *DEL*:           000003H   BYTE   UNIT     XDATA          ?XD?_UART1_TX_DATA?UART
   *DEL*:           000015H   BYTE   UNIT     CODE           ?PR?_UART1_TX_DATA_START?UART
   *DEL*:           000006H   BYTE   UNIT     XDATA          ?XD?_UART1_TX_DATA_START?UART
   *DEL*:           00002CH   BYTE   UNIT     CODE           ?PR?_UART1_TX_DATA_INT?UART
   *DEL*:           000006H   BYTE   UNIT     XDATA          ?XD?_UART1_TX_DATA_INT?UART
   *DEL*:           0000F6H   BYTE   UNIT     CODE           ?PR?_NUMBER_TO_STRING?UART
   *DEL*:           00001DH   BYTE   UNIT     XDATA          ?XD?_NUMBER_TO_STRING?UART
   *DEL*:           00003CH   BYTE   UNIT     CODE           ?PR?_TURN_ON_PWM0_CPM?PWM
   *DEL*:           000023H   BYTE   UNIT     CODE           ?PR?_CHANGE_DUTY_PWM0_CPM?PWM
   *DEL*:           00004AH   BYTE   UNIT     CODE           ?PR?_CHANGE_DUTY_PWM0_IDP?PWM
   *DEL*:           000049H   BYTE   UNIT     CODE           ?PR?_CONFIG_PWM1_MODULE?PWM
   *DEL*:           00003CH   BYTE   UNIT     CODE           ?PR?_TURN_ON_PWM1_CPM?PWM
   *DEL*:           000023H   BYTE   UNIT     CODE           ?PR?_CHANGE_DUTY_PWM1_CPM?PWM
   *DEL*:           00006AH   BYTE   UNIT     CODE           ?PR?_TURN_ON_PWM1_IDP?PWM
   *DEL*:           00004AH   BYTE   UNIT     CODE           ?PR?_CHANGE_DUTY_PWM1_IDP?PWM
   *DEL*:           000034H   BYTE   UNIT     CODE           ?PR?_TURN_OFF_PWM1?PWM
   *DEL*:           000049H   BYTE   UNIT     CODE           ?PR?_CONFIG_PWM2_MODULE?PWM
   *DEL*:           00003CH   BYTE   UNIT     CODE           ?PR?_TURN_ON_PWM2_CPM?PWM
   *DEL*:           000023H   BYTE   UNIT     CODE           ?PR?_CHANGE_DUTY_PWM2_CPM?PWM
   *DEL*:           00006AH   BYTE   UNIT     CODE           ?PR?_TURN_ON_PWM2_IDP?PWM
   *DEL*:           00004AH   BYTE   UNIT     CODE           ?PR?_CHANGE_DUTY_PWM2_IDP?PWM
   *DEL*:           000034H   BYTE   UNIT     CODE           ?PR?_TURN_OFF_PWM2?PWM
   *DEL*:           000018H   BYTE   UNIT     CODE           ?PR?CONFIG_PWM3_MODULE?PWM
   *DEL*:           00000BH   BYTE   UNIT     CODE           ?PR?_TURN_ON_PWM3?PWM
   *DEL*:           00000CH   BYTE   UNIT     CODE           ?PR?TURN_OFF_PWM3?PWM
   *DEL*:           00015BH   BYTE   UNIT     CODE           ?PR?ADC_SAMPLING_PERIOD?ADC
   *DEL*:           000009H   BYTE   UNIT     XDATA          ?XD?ADC_SAMPLING_PERIOD?ADC
   *DEL*:           000026H   BYTE   UNIT     CODE           ?PR?_FLASH_ERASE_SECTOR?FLASH
   *DEL*:           000028H   BYTE   UNIT     CODE           ?PR?_FLASH_WRITE_ONE_BYTE?FLASH
   *DEL*:           000043H   BYTE   UNIT     CODE           ?PR?_FLASH_WRITE_MULTI_BYTE?FLASH
   *DEL*:           000003H   BYTE   UNIT     XDATA          ?XD?_FLASH_WRITE_MULTI_BYTE?FLASH
   *DEL*:           00003AH   BYTE   UNIT     CODE           ?PR?_FLASH_READ_MULTI_BYTE?FLASH
   *DEL*:           000002H   BYTE   UNIT     XDATA          ?XD?_FLASH_READ_MULTI_BYTE?FLASH
   *DEL*:           0000AFH   BYTE   UNIT     CODE           ?PR?FLASH_TEST_CODE?FLASH
   *DEL*:           000010H   BYTE   UNIT     XDATA          ?XD?FLASH_TEST_CODE?FLASH
   *DEL*:           000010H   BYTE   UNIT     CONST          ?CO?FLASH
   *DEL*:           000031H   BYTE   UNIT     CODE           ?PR?CONFIG_SPI_MASTER_MODULE?SPI
   *DEL*:           000036H   BYTE   UNIT     CODE           ?PR?_SPI_MASTER_WRITE?SPI
   *DEL*:           000003H   BYTE   UNIT     XDATA          ?XD?_SPI_MASTER_WRITE?SPI
   *DEL*:           000039H   BYTE   UNIT     CODE           ?PR?_SPI_MASTER_READ?SPI
   *DEL*:           000003H   BYTE   UNIT     XDATA          ?XD?_SPI_MASTER_READ?SPI
   *DEL*:           000034H   BYTE   UNIT     CODE           ?PR?CONFIG_SPI_SLAVE_MODULE?SPI
   *DEL*:           00003DH   BYTE   UNIT     CODE           ?PR?SPI_MASTER_TEST_CODE?SPI
   *DEL*:           000010H   BYTE   UNIT     XDATA          ?XD?SPI_MASTER_TEST_CODE?SPI
LX51 LINKER/LOCATER V4.66.41.0                                                        06/16/2023  10:23:34  PAGE 8


   *DEL*:           000010H   BYTE   UNIT     CONST          ?CO?SPI
   *DEL*:           000021H   BYTE   UNIT     CODE           ?PR?CONFIG_IIC_MASTER_MODULE?IIC
   *DEL*:           000064H   BYTE   UNIT     CODE           ?PR?_IIC_MASTER_SENDDATA?IIC
   *DEL*:           000003H   BYTE   UNIT     XDATA          ?XD?_IIC_MASTER_SENDDATA?IIC
   *DEL*:           00009AH   BYTE   UNIT     CODE           ?PR?_IIC_MASTER_READDATA?IIC
   *DEL*:           000003H   BYTE   UNIT     XDATA          ?XD?_IIC_MASTER_READDATA?IIC
   *DEL*:           000027H   BYTE   UNIT     CODE           ?PR?CONFIG_IIC_SLAVE_MODULE?IIC



OVERLAY MAP OF MODULE:   .\release\BL003C4 (?C_STARTUP)


FUNCTION/MODULE                             BIT_GROUP   DATA_GROUP   XDATA_GROUP
--> CALLED FUNCTION/MODULE                 START  STOP  START  STOP  START  STOP
================================================================================
?C_C51STARTUP                              ----- -----  ----- -----  ----- -----
  +--> MAIN/MAIN
  +--> ?C_INITSEG

MAIN/MAIN                                  ----- -----  ----- -----  ----- -----
  +--> HARDWARE_INIT/PORT_MCU
  +--> USER_GPIO_INITIAL/USER
  +--> USER_REGISTER_INITIAL/USER
  +--> DEBUG_INIT/PORT_MCU
  +--> ?CO?MAIN
  +--> _USER_PRINTF/PORT_MCU
  +--> FEED_WATCHDOG/REGISTER
  +--> SYSTEM_TIMER_PRO/USER
  +--> SYSTEM_FLOW_CONTROL/USER
  +--> SYSTEM_POWER_DOWN/PORT_MCU

HARDWARE_INIT/PORT_MCU                     ----- -----  ----- -----  ----- -----
  +--> RESET_CHECK/REGISTER
  +--> CONFIG_SYSCLK_IHRC_MODULE/REGISTER
  +--> CONFIG_TIMER0_MODULE/TIMER
  +--> CONFIG_ADC_MODULE/ADC
  +--> _CONFIG_PWM0_MODULE/PWM
  +--> ENABLE_WATCHDOG/REGISTER

RESET_CHECK/REGISTER                       ----- -----  ----- -----  ----- -----

CONFIG_SYSCLK_IHRC_MODULE/REGISTER         ----- -----  ----- -----  ----- -----

CONFIG_TIMER0_MODULE/TIMER                 ----- -----  ----- -----  ----- -----

CONFIG_ADC_MODULE/ADC                      ----- -----  ----- -----  ----- -----

_CONFIG_PWM0_MODULE/PWM                    ----- -----  ----- -----  ----- -----

ENABLE_WATCHDOG/REGISTER                   ----- -----  ----- -----  ----- -----

USER_GPIO_INITIAL/USER                     ----- -----  ----- -----  ----- -----

USER_REGISTER_INITIAL/USER                 ----- -----  ----- -----  ----- -----

DEBUG_INIT/PORT_MCU                        ----- -----  ----- -----  ----- -----

?CO?MAIN                                   ----- -----  ----- -----  ----- -----

_USER_PRINTF/PORT_MCU                      ----- -----  ----- -----  0000H 0002H
  +--> _DEBUG_PUTCHAR/PORT_MCU

_DEBUG_PUTCHAR/PORT_MCU                    ----- -----  ----- -----  ----- -----

LX51 LINKER/LOCATER V4.66.41.0                                                        06/16/2023  10:23:34  PAGE 9


FEED_WATCHDOG/REGISTER                     ----- -----  ----- -----  ----- -----

SYSTEM_TIMER_PRO/USER                      ----- -----  ----- -----  ----- -----
  +--> TASK_KEY_SCAN/KEY
  +--> _ADC_SAMPLING_CONTINUOUS/ADC
  +--> ?CO?USER
  +--> PRINTF/PRINTF

TASK_KEY_SCAN/KEY                          ----- -----  ----- -----  ----- -----

_ADC_SAMPLING_CONTINUOUS/ADC               ----- -----  ----- -----  0000H 0007H
  +--> ADC_SAMPLING_SINGLE/ADC
  +--> _DELAY_US/PORT_MCU

ADC_SAMPLING_SINGLE/ADC                    ----- -----  ----- -----  ----- -----

_DELAY_US/PORT_MCU                         ----- -----  ----- -----  ----- -----

?CO?USER                                   ----- -----  ----- -----  ----- -----

PRINTF/PRINTF                              20H.0 21H.0  0008H 000CH  0000H 0027H
  +--> _PUTCHAR/PORT_MCU

_PUTCHAR/PORT_MCU                          ----- -----  ----- -----  ----- -----

SYSTEM_FLOW_CONTROL/USER                   ----- -----  ----- -----  ----- -----
  +--> USER_KEY_PRO/USER

USER_KEY_PRO/USER                          ----- -----  ----- -----  ----- -----
  +--> _TURN_ON_PWM0_IDP/PWM
  +--> _TURN_OFF_PWM0/PWM

_TURN_ON_PWM0_IDP/PWM                      ----- -----  ----- -----  ----- -----

_TURN_OFF_PWM0/PWM                         ----- -----  ----- -----  ----- -----

SYSTEM_POWER_DOWN/PORT_MCU                 ----- -----  ----- -----  ----- -----
  +--> DISABLE_WATCHDOG/REGISTER
  +--> CONFIG_SYSCLK_IHRC_MODULE/REGISTER
  +--> CONFIG_ADC_MODULE/ADC
  +--> FEED_WATCHDOG/REGISTER
  +--> ENABLE_WATCHDOG/REGISTER

DISABLE_WATCHDOG/REGISTER                  ----- -----  ----- -----  ----- -----

?C_INITSEG                                 ----- -----  ----- -----  ----- -----

*** NEW ROOT *****************************

DEBUG_RPT/PORT_MCU                         ----- -----  ----- -----  ----- -----

*** NEW ROOT *****************************

WDT_RPT/REGISTER                           ----- -----  ----- -----  ----- -----

*** NEW ROOT *****************************

INT0_RPT/GPIO                              ----- -----  ----- -----  ----- -----

*** NEW ROOT *****************************

INT1_RPT/GPIO                              ----- -----  ----- -----  ----- -----

*** NEW ROOT *****************************

LX51 LINKER/LOCATER V4.66.41.0                                                        06/16/2023  10:23:34  PAGE 10


INT2_7_RPT/GPIO                            ----- -----  ----- -----  ----- -----

*** NEW ROOT *****************************

INT8_15_RPT/GPIO                           ----- -----  ----- -----  ----- -----

*** NEW ROOT *****************************

TIMER0_SERVICE/TIMER                       ----- -----  ----- -----  ----- -----

*** NEW ROOT *****************************

TIMER1_SERVICE/TIMER                       ----- -----  ----- -----  ----- -----

*** NEW ROOT *****************************

TIMER3_SERVICE/TIMER                       ----- -----  ----- -----  ----- -----

*** NEW ROOT *****************************

TIMER4_SERVICE/TIMER                       ----- -----  ----- -----  ----- -----

*** NEW ROOT *****************************

TIMER5_SERVICE/TIMER                       ----- -----  ----- -----  ----- -----

*** NEW ROOT *****************************

UART1_RPT/UART                             ----- -----  ----- -----  ----- -----
  +--> _UART1_RX_DATA_INT/UART

_UART1_RX_DATA_INT/UART                    ----- -----  ----- -----  0028H 0030H

*** NEW ROOT *****************************

PWM_RPT/PWM                                ----- -----  ----- -----  ----- -----

*** NEW ROOT *****************************

ADC_RPT/ADC                                ----- -----  ----- -----  ----- -----

*** NEW ROOT *****************************

SPI_RPT/SPI                                ----- -----  ----- -----  ----- -----
  +--> _SPI_SLAVE_READ_INT/SPI

_SPI_SLAVE_READ_INT/SPI                    ----- -----  ----- -----  0031H 0039H

*** NEW ROOT *****************************

IIC_RPT/IIC                                ----- -----  ----- -----  ----- -----



PUBLIC SYMBOLS OF MODULE:  .\release\BL003C4 (?C_STARTUP)


      VALUE       CLASS    TYPE      PUBLIC SYMBOL NAME
      =================================================
*DEL*:00000000H   XDATA    BYTE      ?_HS6220_read_buffer?BYTE
*DEL*:00000000H   XDATA    BYTE      ?_HS6220_SendPack?BYTE
*DEL*:00000000H   XDATA    BYTE      ?_HS6220_wr_buffer?BYTE
      02000000H   XDATA    ---       ?_PRINTF517?BYTE
      02000000H   XDATA    ---       ?_PRINTF?BYTE
      02000000H   XDATA    ---       ?_SPRINTF517?BYTE
LX51 LINKER/LOCATER V4.66.41.0                                                        06/16/2023  10:23:34  PAGE 11


      02000000H   XDATA    ---       ?_SPRINTF?BYTE
*DEL*:00000000H   XDATA    BYTE      ?_uart1_tx_data_start?BYTE
      010003FEH   CODE     ---       ?C?CCASE
      010001C2H   CODE     ---       ?C?CILDPTR
      01000195H   CODE     ---       ?C?CLDOPTR
      0100017CH   CODE     ---       ?C?CLDPTR
      00000000H   NUMBER   ---       ?C?CODESEG
      01000156H   CODE     ---       ?C?COPY
      010001F6H   CODE     ---       ?C?CSTOPTR
      010001E4H   CODE     ---       ?C?CSTPTR
      0100027FH   CODE     ---       ?C?ILDIX
      01000218H   CODE     ---       ?C?IMUL
      010003B1H   CODE     ---       ?C?LIMUL
      01000380H   CODE     ---       ?C?LSTKXDATA
      01000374H   CODE     ---       ?C?LSTXDATA
      010003DEH   CODE     ---       ?C?PLDIXDATA
      010003F5H   CODE     ---       ?C?PSTXDATA
      0100022AH   CODE     ---       ?C?UIDIV
      01000363H   CODE     ---       ?C?ULCMP
      010002D1H   CODE     ---       ?C?ULDIV
      00000000H   NUMBER   ---       ?C?XDATASEG
      01000C0EH   CODE     ---       ?C_START
      01000000H   CODE     ---       ?C_STARTUP
      010009D7H   CODE     ---       _adc_sampling_continuous
*DEL*:00000000H   CODE     ---       _change_duty_pwm0_cpm
*DEL*:00000000H   CODE     ---       _change_duty_pwm0_idp
*DEL*:00000000H   CODE     ---       _change_duty_pwm1_cpm
*DEL*:00000000H   CODE     ---       _change_duty_pwm1_idp
*DEL*:00000000H   CODE     ---       _change_duty_pwm2_cpm
*DEL*:00000000H   CODE     ---       _change_duty_pwm2_idp
      01000F6AH   CODE     ---       _config_pwm0_module
*DEL*:00000000H   CODE     ---       _config_pwm1_module
*DEL*:00000000H   CODE     ---       _config_pwm2_module
*DEL*:00000000H   CODE     ---       _config_uart1_module
      010011F2H   CODE     ---       _debug_putchar
*DEL*:00000000H   CODE     ---       _delay_ms
*DEL*:00000000H   CODE     ---       _delay_ms_int
      0100002EH   CODE     ---       _delay_us
*DEL*:00000000H   CODE     ---       _flash_erase_sector
*DEL*:00000006H   CODE     ---       _flash_read_multi_byte
*DEL*:00000000H   CODE     ---       _flash_write_multi_byte
*DEL*:00000000H   CODE     ---       _flash_write_one_byte
*DEL*:00000000H   CODE     ---       _hd_crc_calculate
*DEL*:00000000H   CODE     ---       _HS6220_Bank_Switch
*DEL*:00000000H   CODE     ---       _HS6220_Change_Addr
*DEL*:00000000H   CODE     ---       _HS6220_Change_CH
*DEL*:00000000H   CODE     ---       _HS6220_Change_Pwr
*DEL*:00000000H   CODE     ---       _HS6220_Change_Rate
*DEL*:00000000H   CODE     ---       _HS6220_ModeSwitch
*DEL*:00000000H   CODE     ---       _HS6220_Operation
*DEL*:00000000H   CODE     ---       _HS6220_read_buffer
*DEL*:00000000H   CODE     ---       _HS6220_read_byte
*DEL*:00000000H   CODE     ---       _HS6220_ReceivePack
*DEL*:00000000H   CODE     ---       _HS6220_SendPack
*DEL*:00000006H   CODE     ---       _HS6220_wr_buffer
*DEL*:00000000H   CODE     ---       _HS6220_wr_cmd
*DEL*:00000000H   CODE     ---       _HS6220_write_byte
*DEL*:00000000H   CODE     ---       _Iic_Master_ReadData
*DEL*:00000000H   CODE     ---       _Iic_Master_SendData
*DEL*:00000000H   CODE     ---       _number_to_string
      0100048FH   CODE     ---       _PRINTF
      0100048FH   CODE     ---       _PRINTF517
      010011DAH   CODE     ---       _putchar
*DEL*:00000000H   CODE     ---       _SPI_3wire_sendByte
*DEL*:00000000H   CODE     ---       _spi_master_read
LX51 LINKER/LOCATER V4.66.41.0                                                        06/16/2023  10:23:34  PAGE 12


*DEL*:00000000H   CODE     ---       _spi_master_write
*DEL*:00000003H   CODE     ---       _SPI_SendByte
      01000489H   CODE     ---       _SPRINTF
      01000489H   CODE     ---       _SPRINTF517
      010010D6H   CODE     ---       _turn_off_pwm0
*DEL*:00000000H   CODE     ---       _turn_off_pwm1
*DEL*:00000000H   CODE     ---       _turn_off_pwm2
*DEL*:00000000H   CODE     ---       _turn_on_pwm0_cpm
      01000CBFH   CODE     ---       _turn_on_pwm0_idp
*DEL*:00000000H   CODE     ---       _turn_on_pwm1_cpm
*DEL*:00000000H   CODE     ---       _turn_on_pwm1_idp
*DEL*:00000000H   CODE     ---       _turn_on_pwm2_cpm
*DEL*:00000000H   CODE     ---       _turn_on_pwm2_idp
*DEL*:00000000H   CODE     ---       _turn_on_pwm3
*DEL*:00000000H   CODE     ---       _uart1_tx_byte
*DEL*:00000000H   CODE     ---       _uart1_tx_data
*DEL*:00000000H   CODE     ---       _uart1_tx_data_start
      0100110AH   CODE     ---       _user_printf
*SFR* 000000D0H.6 DATA     BIT       AC
*SFR* 000000E0H   DATA     BYTE      ACC
      01000026H   CODE     ---       adc_rpt
*DEL*:00000000H   CODE     ---       adc_sampling_period
      01001240H   CODE     ---       adc_sampling_single
*SFR* 000000B4H   DATA     BYTE      ADCC0
*SFR* 000000B5H   DATA     BYTE      ADCC1
      0200FE9BH   XDATA    BYTE      ADCC2
      0200FE9AH   XDATA    BYTE      ADCC3
      0200FE9EH   XDATA    BYTE      ADCCONTV
      0200FE9CH   XDATA    BYTE      ADCDLYH
      0200FE9DH   XDATA    BYTE      ADCDLYL
      0200FE9FH   XDATA    BYTE      ADCGAPV
      0200FEACH   XDATA    BYTE      ADCHTRH
      0200FEADH   XDATA    BYTE      ADCHTRL
      0200FEAEH   XDATA    BYTE      ADCLTRH
      0200FEAFH   XDATA    BYTE      ADCLTRL
*SFR* 000000B6H   DATA     WORD      ADCR
*SFR* 000000B7H   DATA     BYTE      ADCRH
*SFR* 000000B6H   DATA     BYTE      ADCRL
      0200FF8DH   XDATA    BYTE      ADCST_MAP
      0200FE98H   XDATA    BYTE      ADCWC
      0200FEABH   XDATA    BYTE      AWDCON
*SFR* 000000F0H   DATA     BYTE      B
      00000021H.6 BIT      BIT       b_aden_flag
      00000021H.5 BIT      BIT       b_base_1ms_int
      00000022H.0 BIT      BIT       b_debug_rx_end
      00000021H.1 BIT      BIT       b_key1_long_trig
      00000021H.3 BIT      BIT       b_key1_short_trig
      00000021H.2 BIT      BIT       b_key2_long_trig
      00000021H.4 BIT      BIT       b_key2_short_trig
      00000021H.7 BIT      BIT       b_pwmen_flag
      020000BAH   XDATA    BYTE      b_t5_input_level
      0200FEA4H   XDATA    BYTE      BORC
      0200FEA5H   XDATA    BYTE      BORDBC
*SFR* 000000F8H.5 DATA     BIT       BORF
      0200FE8BH   XDATA    BYTE      BRTSEL
      0200FF88H   XDATA    BYTE      CAP0_MAP
      0200FF89H   XDATA    BYTE      CAP1_MAP
      0200FED8H   XDATA    BYTE      CAPCON0
      0200FED9H   XDATA    BYTE      CAPCON1
      0200FED0H   XDATA    BYTE      CAPH0
      0200FED2H   XDATA    BYTE      CAPH1
      0200FED1H   XDATA    BYTE      CAPL0
      0200FED3H   XDATA    BYTE      CAPL1
*SFR* 0000008FH   DATA     BYTE      CLKCON
      0200FE91H   XDATA    BYTE      CLKDIV
LX51 LINKER/LOCATER V4.66.41.0                                                        06/16/2023  10:23:34  PAGE 13


      0200FF8FH   XDATA    BYTE      CLKO_MAP
      0200FE93H   XDATA    BYTE      CLKOUT
*SFR* 0000008EH   DATA     BYTE      CLKSWR
      0200FF60H   XDATA    BYTE      COMP0EN
      0200FF61H   XDATA    BYTE      COMP1EN
      0200FF62H   XDATA    BYTE      COMP2EN
      010011BBH   CODE     ---       config_adc_module
*DEL*:00000000H   CODE     ---       config_gpio_ext_int
*DEL*:00000000H   CODE     ---       config_gpio_power_on
*DEL*:00000000H   CODE     ---       config_iic_master_module
*DEL*:00000000H   CODE     ---       config_iic_slave_module
*DEL*:00000000H   CODE     ---       config_pwm3_module
*DEL*:00000000H   CODE     ---       config_spi_master_module
*DEL*:00000000H   CODE     ---       config_spi_slave_module
*DEL*:00000000H   CODE     ---       config_sysclk_crystal_module
      0100116CH   CODE     ---       config_sysclk_ihrc_module
*DEL*:00000000H   CODE     ---       config_sysclk_output
      0100121AH   CODE     ---       config_timer0_module
*DEL*:00000000H   CODE     ---       config_timer1_module
*DEL*:00000000H   CODE     ---       config_timer3_module
*DEL*:00000000H   CODE     ---       config_timer4_module
*DEL*:00000000H   CODE     ---       config_timer5_module
      0200FEA2H   XDATA    BYTE      CRCC
*SFR* 000000BFH   DATA     BYTE      CRCH
*SFR* 000000BEH   DATA     BYTE      CRCL
*SFR* 000000BEH   DATA     WORD      CRCR
*SFR* 000000D0H.7 DATA     BIT       CY
      0200FE97H   XDATA    BYTE      DBGFLAG
      01000FF3H   CODE     ---       debug_init
      01000C53H   CODE     ---       debug_rpt
      01001269H   CODE     ---       disable_watchdog
*SFR* 00000083H   DATA     BYTE      DPH
*SFR* 00000082H   DATA     BYTE      DPL
*SFR* 00000082H   DATA     WORD      DPTR
*SFR* 000000A8H.7 DATA     BIT       EA
*SFR* 000000B8H.5 DATA     BIT       EADC
*SFR* 000000B8H.3 DATA     BIT       EIIC
      0100125FH   CODE     ---       enable_watchdog
*DEL*:00000000H   CODE     ---       enable_watchdog_for_stop
*SFR* 000000A8H.4 DATA     BIT       ES1
*SFR* 000000A8H.6 DATA     BIT       ES2
*SFR* 000000B8H   DATA     BIT       ESPI
*SFR* 000000A8H.1 DATA     BIT       ET0
*SFR* 000000A8H.3 DATA     BIT       ET1
*SFR* 000000B8H.1 DATA     BIT       ET3
*SFR* 000000B8H.2 DATA     BIT       ET4
*SFR* 000000B8H.4 DATA     BIT       ET5
*SFR* 000000A8H.5 DATA     BIT       EWDT
*SFR* 000000A8H   DATA     BIT       EX0
*SFR* 000000A8H.2 DATA     BIT       EX1
*SFR* 000000B8H.6 DATA     BIT       EX2_7
*SFR* 000000B8H.7 DATA     BIT       EX8_15
*SFR* 000000F8H.6 DATA     BIT       EXRSTF
*SFR* 000000D0H.5 DATA     BIT       F0
*SFR* 000000D0H.1 DATA     BIT       F1
*SFR* 00000098H.7 DATA     BIT       FE
      01000006H   CODE     ---       feed_watchdog
*DEL*:00000000H   CODE     ---       flash_test_code
      0200FE92H   XDATA    BYTE      FREQ_CLK
      01001206H   CODE     ---       hardware_init
      020000B0H   XDATA    ---       hs24m_trim
      020000AEH   XDATA    ---       hs32m_trim
*DEL*:00000000H   CODE     ---       HS6220_CE_High
*DEL*:00000000H   CODE     ---       HS6220_CE_Low
*DEL*:00000000H   CODE     ---       HS6220_Clear_All_Irq
LX51 LINKER/LOCATER V4.66.41.0                                                        06/16/2023  10:23:34  PAGE 14


*DEL*:00000000H   CODE     ---       HS6220_Flush_Rx
*DEL*:00000000H   CODE     ---       HS6220_Flush_Tx
*DEL*:00000000H   CODE     ---       HS6220_Init
*DEL*:00000000H   CODE     ---       HS6220_read_payload_length
*DEL*:00000000H   CODE     ---       HS6220_SPI_Init
*SFR* 000000F9H   DATA     WORD      IAP_ADDR
*SFR* 000000FAH   DATA     BYTE      IAP_ADDRH
*SFR* 000000F9H   DATA     BYTE      IAP_ADDRL
*SFR* 000000FCH   DATA     WORD      IAP_CMD
*SFR* 000000FDH   DATA     BYTE      IAP_CMDH
*SFR* 000000FCH   DATA     BYTE      IAP_CMDL
*SFR* 000000FBH   DATA     BYTE      IAP_DATA
*SFR* 000000A8H   DATA     BYTE      IE
*SFR* 000000B8H   DATA     BYTE      IE1
      01000857H   CODE     ---       IIC_Rpt
*SFR* 000000AFH   DATA     BYTE      IICADR
*SFR* 000000A6H   DATA     BYTE      IICCON
*SFR* 000000AEH   DATA     BYTE      IICDAT
*SFR* 000000A7H   DATA     BYTE      IICSTA
*SFR* 000000A2H   DATA     BYTE      INSCON
      0200FEBCH   XDATA    BYTE      INT01_PINS
      0100000AH   CODE     ---       int0_rpt
      01000012H   CODE     ---       int1_rpt
      01000016H   CODE     ---       int2_7_rpt
      0100001EH   CODE     ---       int8_15_rpt
*SFR* 000000A9H   DATA     BYTE      IP0
*SFR* 000000AAH   DATA     BYTE      IP1
*SFR* 000000B9H   DATA     BYTE      IP2
*SFR* 000000BAH   DATA     BYTE      IP3
*SFR* 000000B1H   DATA     BYTE      IP4
*SFR* 000000D1H   DATA     BYTE      LCDCON
*SFR* 000000BBH   DATA     BYTE      LVDC
*SFR* 000000BCH   DATA     BYTE      LVDCMP
      0200FEA7H   XDATA    BYTE      LVDDBC
      0200FE96H   XDATA    BYTE      LXTALSPD
      01000E82H   CODE     ---       main
      0200FFA7H   XDATA    BYTE      MISO_MAP
      0200FFA6H   XDATA    BYTE      MOSI_MAP
*SFR* 000000D0H.2 DATA     BIT       OV
*SFR* 000000D0H   DATA     BIT       P
*SFR* 00000080H   DATA     BYTE      P0
      0200FF40H   XDATA    BYTE      P00DBC
      0200FF41H   XDATA    BYTE      P01DBC
      0200FF42H   XDATA    BYTE      P02DBC
*SFR* 00000080H   DATA     BIT       P0_0
*SFR* 00000080H.1 DATA     BIT       P0_1
*SFR* 00000080H.2 DATA     BIT       P0_2
*SFR* 00000080H.3 DATA     BIT       P0_3
*SFR* 00000080H.4 DATA     BIT       P0_4
*SFR* 00000080H.5 DATA     BIT       P0_5
*SFR* 00000080H.6 DATA     BIT       P0_6
*SFR* 00000080H.7 DATA     BIT       P0_7
      0200FF05H   XDATA    BYTE      P0LPU
      0200FF00H   XDATA    BYTE      P0M0
      0200FF01H   XDATA    BYTE      P0M1
      0200FF02H   XDATA    BYTE      P0M2
      0200FF03H   XDATA    BYTE      P0M3
      0200FF50H   XDATA    BYTE      P0OUT
*SFR* 00000090H   DATA     BYTE      P1
*SFR* 00000090H   DATA     BIT       P1_0
*SFR* 00000090H.1 DATA     BIT       P1_1
      0200FF08H   XDATA    BYTE      P1M0
      0200FF51H   XDATA    BYTE      P1OUT
*SFR* 000000A0H   DATA     BYTE      P2
*SFR* 000000A0H   DATA     BIT       P2_0
LX51 LINKER/LOCATER V4.66.41.0                                                        06/16/2023  10:23:34  PAGE 15


*SFR* 000000A0H.1 DATA     BIT       P2_1
*SFR* 000000A0H.2 DATA     BIT       P2_2
*SFR* 000000A0H.3 DATA     BIT       P2_3
*SFR* 000000A0H.4 DATA     BIT       P2_4
*SFR* 000000A0H.5 DATA     BIT       P2_5
*SFR* 000000A0H.6 DATA     BIT       P2_6
*SFR* 000000A0H.7 DATA     BIT       P2_7
      0200FF10H   XDATA    BYTE      P2M0
      0200FF11H   XDATA    BYTE      P2M1
      0200FF12H   XDATA    BYTE      P2M2
      0200FF13H   XDATA    BYTE      P2M3
      0200FF52H   XDATA    BYTE      P2OUT
*SFR* 00000087H   DATA     BYTE      PCON
      0200FEB8H   XDATA    BYTE      PINTE0
      0200FEB9H   XDATA    BYTE      PINTE1
*SFR* 00000096H   DATA     BYTE      PINTF0
*SFR* 00000097H   DATA     BYTE      PINTF1
      0200FEB0H   XDATA    BYTE      PITS0
      0200FEB1H   XDATA    BYTE      PITS1
      0200FEB2H   XDATA    BYTE      PITS2
      0200FEB3H   XDATA    BYTE      PITS3
*SFR* 000000F8H   DATA     BIT       PLVRSTF
*SFR* 000000F8H.7 DATA     BIT       PORF
*SFR* 000000D0H   DATA     BYTE      PSW
      0200FF91H   XDATA    BYTE      PWM01_MAP
      0200FF90H   XDATA    BYTE      PWM0_MAP
*SFR* 000000DAH   DATA     BYTE      PWM0C
      0200FEF0H   XDATA    BYTE      PWM0CMPH
      0200FEF1H   XDATA    BYTE      PWM0CMPL
*SFR* 000000E4H   DATA     WORD      PWM0D
*SFR* 000000E5H   DATA     BYTE      PWM0DH
*SFR* 000000E4H   DATA     BYTE      PWM0DL
*SFR* 000000E6H   DATA     WORD      PWM0DT
*SFR* 000000E7H   DATA     BYTE      PWM0DTH
*SFR* 000000E6H   DATA     BYTE      PWM0DTL
*SFR* 000000E1H   DATA     BYTE      PWM0EN
      0200FEE8H   XDATA    BYTE      PWM0INTDIV
*SFR* 000000E2H   DATA     WORD      PWM0P
*SFR* 000000E3H   DATA     BYTE      PWM0PH
      0200FEE0H   XDATA    BYTE      PWM0PHASEH
      0200FEE1H   XDATA    BYTE      PWM0PHASEL
*SFR* 000000E2H   DATA     BYTE      PWM0PL
      0200FF95H   XDATA    BYTE      PWM11_MAP
      0200FF94H   XDATA    BYTE      PWM1_MAP
*SFR* 000000DBH   DATA     BYTE      PWM1C
*SFR* 000000ECH   DATA     WORD      PWM1D
*SFR* 000000EDH   DATA     BYTE      PWM1DH
*SFR* 000000ECH   DATA     BYTE      PWM1DL
*SFR* 000000EEH   DATA     WORD      PWM1DT
*SFR* 000000EFH   DATA     BYTE      PWM1DTH
*SFR* 000000EEH   DATA     BYTE      PWM1DTL
*SFR* 000000E9H   DATA     BYTE      PWM1EN
      0200FEE9H   XDATA    BYTE      PWM1INTDIV
*SFR* 000000EAH   DATA     WORD      PWM1P
*SFR* 000000EBH   DATA     BYTE      PWM1PH
      0200FEE2H   XDATA    BYTE      PWM1PHASEH
      0200FEE3H   XDATA    BYTE      PWM1PHASEL
*SFR* 000000EAH   DATA     BYTE      PWM1PL
      0200FF99H   XDATA    BYTE      PWM21_MAP
      0200FF98H   XDATA    BYTE      PWM2_MAP
*SFR* 000000DCH   DATA     BYTE      PWM2C
*SFR* 000000F4H   DATA     WORD      PWM2D
*SFR* 000000F5H   DATA     BYTE      PWM2DH
*SFR* 000000F4H   DATA     BYTE      PWM2DL
*SFR* 000000F6H   DATA     WORD      PWM2DT
LX51 LINKER/LOCATER V4.66.41.0                                                        06/16/2023  10:23:34  PAGE 16


*SFR* 000000F7H   DATA     BYTE      PWM2DTH
*SFR* 000000F6H   DATA     BYTE      PWM2DTL
*SFR* 000000F1H   DATA     BYTE      PWM2EN
      0200FEEAH   XDATA    BYTE      PWM2INTDIV
*SFR* 000000F2H   DATA     WORD      PWM2P
*SFR* 000000F3H   DATA     BYTE      PWM2PH
      0200FEE4H   XDATA    BYTE      PWM2PHASEH
      0200FEE5H   XDATA    BYTE      PWM2PHASEL
*SFR* 000000F2H   DATA     BYTE      PWM2PL
      0200FF9CH   XDATA    BYTE      PWM3_MAP
*SFR* 000000DDH   DATA     BYTE      PWM3C
      0200FEEEH   XDATA    BYTE      PWM3CLKS
*SFR* 000000DFH   DATA     BYTE      PWM3D
*SFR* 000000DEH   DATA     BYTE      PWM3P
      01001196H   CODE     ---       pwm_rpt
      0200FEF9H   XDATA    BYTE      PWMCON0
      0200FEFAH   XDATA    BYTE      PWMCON1
      0200FEFBH   XDATA    BYTE      PWMCON2
      0200FEF8H   XDATA    BYTE      PWMENA
*SFR* 00000098H.2 DATA     BIT       RB8
*SFR* 000000C4H   DATA     WORD      RCAP5
*SFR* 000000C5H   DATA     BYTE      RCAP5H
*SFR* 000000C4H   DATA     BYTE      RCAP5L
*SFR* 00000098H.4 DATA     BIT       REN
      01000FB3H   CODE     ---       reset_check
      0200004CH   XDATA    ---       rf
      020000B5H   XDATA    WORD      rf_reset_cnt
      020000B7H   XDATA    BYTE      rf_sleep_cnt
*SFR* 00000098H   DATA     BIT       RI
*SFR* 000000D0H.3 DATA     BIT       RS0
*SFR* 000000D0H.4 DATA     BIT       RS1
      0200FEAAH   XDATA    BYTE      RSTDBC
*SFR* 000000F8H   DATA     BYTE      RSTFR
      0200FFA9H   XDATA    BYTE      RXD2_MAP
      0200FFA1H   XDATA    BYTE      RXD_MAP
*SFR* 00000098H.6 DATA     BIT       RXROV
      0200FE8AH   XDATA    BYTE      S2BUF
      0200FE88H   XDATA    BYTE      S2CON
      0200FE89H   XDATA    BYTE      S2CON2
*SFR* 0000009AH   DATA     BYTE      SADDR
*SFR* 0000009BH   DATA     BYTE      SADEN
*SFR* 00000099H   DATA     BYTE      SBUF
      0200FFA5H   XDATA    BYTE      SCK_MAP
      0200FFA2H   XDATA    BYTE      SCL_MAP
*SFR* 00000098H   DATA     BYTE      SCON
*SFR* 0000009EH   DATA     BYTE      SCON2
      0200FEC0H   XDATA    BYTE      SCRH0
      0200FEC2H   XDATA    BYTE      SCRH1
      0200FEC4H   XDATA    BYTE      SCRH2
      0200FEC6H   XDATA    BYTE      SCRH3
      0200FEC8H   XDATA    BYTE      SCRH4
      0200FECAH   XDATA    BYTE      SCRH5
      0200FECCH   XDATA    BYTE      SCRH6
      0200FECEH   XDATA    BYTE      SCRH7
      0200FEC1H   XDATA    BYTE      SCRL0
      0200FEC3H   XDATA    BYTE      SCRL1
      0200FEC5H   XDATA    BYTE      SCRL2
      0200FEC7H   XDATA    BYTE      SCRL3
      0200FEC9H   XDATA    BYTE      SCRL4
      0200FECBH   XDATA    BYTE      SCRL5
      0200FECDH   XDATA    BYTE      SCRL6
      0200FECFH   XDATA    BYTE      SCRL7
      0200FFA3H   XDATA    BYTE      SDA_MAP
*SFR* 00000081H   DATA     BYTE      SP
*SFR* 000000ACH   DATA     BYTE      SPCTL
LX51 LINKER/LOCATER V4.66.41.0                                                        06/16/2023  10:23:34  PAGE 17


*SFR* 000000ABH   DATA     BYTE      SPDAT
*DEL*:00000000H   CODE     ---       SPI_3wire_readByte
*DEL*:00000000H   CODE     ---       spi_master_test_code
*DEL*:00000000H   CODE     ---       SPI_ReadByte
      01000E30H   CODE     ---       SPI_Rpt
      0200FE95H   XDATA    BYTE      SPOV_RSTEN
*SFR* 000000F8H.1 DATA     BIT       SPOVF
*SFR* 000000ADH   DATA     BYTE      SPSTAT
      0200FFA4H   XDATA    BYTE      SS_MAP
*SFR* 000000F8H.3 DATA     BIT       SWRF
      0100003EH   CODE     ---       system_flow_control
      01000D29H   CODE     ---       system_power_down
      01000B30H   CODE     ---       system_timer_pro
      0200FF80H   XDATA    BYTE      T0_MAP
      0200FF81H   XDATA    BYTE      T1_MAP
*SFR* 000000CAH   DATA     WORD      T3
      0200FF83H   XDATA    BYTE      T3_MAP
*SFR* 000000C9H   DATA     BYTE      T3CON
*SFR* 000000CDH   DATA     WORD      T4
      0200FF84H   XDATA    BYTE      T4_MAP
*SFR* 000000CCH   DATA     BYTE      T4CON
      0200FE84H   XDATA    BYTE      T4CON1
*SFR* 000000C2H   DATA     WORD      T5
      0200FF85H   XDATA    BYTE      T5_MAP
*SFR* 000000C1H   DATA     BYTE      T5CON
      0200FE85H   XDATA    BYTE      T5CON1
      0200FE86H   XDATA    BYTE      T5CON2
      01000789H   CODE     ---       task_key_scan
*SFR* 00000098H.3 DATA     BIT       TB8
*SFR* 00000088H   DATA     BYTE      TCON
      0200FE80H   XDATA    BYTE      TCON1
*SFR* 00000088H.5 DATA     BIT       TF0
*SFR* 00000088H.7 DATA     BIT       TF1
*SFR* 0000008CH   DATA     BYTE      TH0
*SFR* 0000008DH   DATA     BYTE      TH1
*SFR* 000000CBH   DATA     BYTE      TH3
*SFR* 000000CEH   DATA     BYTE      TH4
*SFR* 000000C3H   DATA     BYTE      TH5
*SFR* 00000098H.1 DATA     BIT       TI
*SFR* 00000091H   DATA     BYTE      TICKCON
*SFR* 00000093H   DATA     BYTE      TICKH
*SFR* 00000092H   DATA     BYTE      TICKL
      0100113DH   CODE     ---       timer0_service
      0100001AH   CODE     ---       timer1_service
      01001031H   CODE     ---       timer3_service
      01000022H   CODE     ---       timer4_service
      01000D82H   CODE     ---       timer5_service
*SFR* 0000008AH   DATA     BYTE      TL0
*SFR* 0000008BH   DATA     BYTE      TL1
*SFR* 000000CAH   DATA     BYTE      TL3
*SFR* 000000CDH   DATA     BYTE      TL4
*SFR* 000000C2H   DATA     BYTE      TL5
*SFR* 00000089H   DATA     BYTE      TMOD
*SFR* 00000088H.4 DATA     BIT       TR0
*SFR* 00000088H.6 DATA     BIT       TR1
      0200FEBDH   XDATA    BYTE      TRMEN
      0200FEBEH   XDATA    BYTE      TRMV
*DEL*:00000000H   CODE     ---       turn_off_pwm3
*SFR* 00000098H.5 DATA     BIT       TXCOL
      0200FFA8H   XDATA    BYTE      TXD2_MAP
      0200FFA0H   XDATA    BYTE      TXD_MAP
      02000044H   XDATA    WORD      u16_ad_val
      02000047H   XDATA    WORD      u16_cnt_3_int
      02000082H   XDATA    WORD      u16_pwm0_ch0_duty
      02000086H   XDATA    WORD      u16_pwm0_ch1_duty
LX51 LINKER/LOCATER V4.66.41.0                                                        06/16/2023  10:23:34  PAGE 18


      02000084H   XDATA    WORD      u16_pwm1_ch0_duty
      0200008AH   XDATA    WORD      u16_pwm1_ch1_duty
      02000088H   XDATA    WORD      u16_pwm2_ch0_duty
      0200008CH   XDATA    WORD      u16_pwm2_ch1_duty
      020000B8H   XDATA    WORD      u16_t5_catch_val
      0200003AH   XDATA    WORD      u16_wave_time
      0200003CH   XDATA    DWORD     u32_tmp
      02000040H   XDATA    BYTE      u8_cnt_1_int
      02000041H   XDATA    BYTE      u8_cnt_2_int
      020000B3H   XDATA    ---       u8_debug_rx_data
      020000B2H   XDATA    BYTE      u8_debug_rx_index
      0200004AH   XDATA    BYTE      u8_delay_int
      0200008EH   XDATA    ---       u8_iic_rece_buf
      02000092H   XDATA    BYTE      u8_iic_rece_cnt
      02000093H   XDATA    ---       u8_iic_send_buf
      02000097H   XDATA    BYTE      u8_iic_send_cnt
      02000042H   XDATA    BYTE      u8_led1_cnt
      02000043H   XDATA    BYTE      u8_led2_cnt
      02000081H   XDATA    BYTE      u8_pwm3_duty
      0200006FH   XDATA    BYTE      u8_rtc_hour
      0200004BH   XDATA    BYTE      u8_rtc_minute
      02000046H   XDATA    BYTE      u8_rtc_second
      02000099H   XDATA    ---       u8_spi_receive_buf
      0200009FH   XDATA    BYTE      u8_spi_rx_cnt
      02000098H   XDATA    BYTE      u8_spi_rx_flag
      020000A9H   XDATA    ---       u8_uart1_rx_data
      020000A8H   XDATA    BYTE      u8_uart1_rx_data_index
      020000A7H   XDATA    BYTE      u8_uart1_rx_ok
      02000049H   XDATA    BYTE      u8_wake_time
      01000ED1H   CODE     ---       uart1_rpt
      01000F20H   CODE     ---       user_gpio_initial
      010010A1H   CODE     ---       user_key_pro
      0100122EH   CODE     ---       user_register_initial
*DEL*:00000000H   CODE     ---       user_rfrx_pro
*DEL*:00000000H   CODE     ---       user_rftx_pro
      0100000EH   CODE     ---       wdt_rpt
*SFR* 000000BDH   DATA     BYTE      WDTC
      0200FEA0H   XDATA    BYTE      WDTCCR
*SFR* 000000F8H.4 DATA     BIT       WDTRF
      0200FE94H   XDATA    BYTE      XTALCFG



SYMBOL TABLE OF MODULE:  .\release\BL003C4 (?C_STARTUP)

      VALUE       REP       CLASS    TYPE      SYMBOL NAME
      ====================================================
      ---         MODULE    ---      ---       ?C_STARTUP
      01000000H   PUBLIC    CODE     ---       ?C_STARTUP
      000000E0H   SYMBOL    DATA     ---       ACC
      000000F0H   SYMBOL    DATA     ---       B
      00000083H   SYMBOL    DATA     ---       DPH
      00000082H   SYMBOL    DATA     ---       DPL
      00000000H   SYMBOL    NUMBER   ---       IBPSTACK
      00000100H   SYMBOL    NUMBER   ---       IBPSTACKTOP
      00000080H   SYMBOL    NUMBER   ---       IDATALEN
      01000BCAH   SYMBOL    CODE     ---       IDATALOOP
      00000000H   SYMBOL    NUMBER   ---       PBPSTACK
      00000100H   SYMBOL    NUMBER   ---       PBPSTACKTOP
      00000000H   SYMBOL    NUMBER   ---       PDATALEN
      00000000H   SYMBOL    NUMBER   ---       PDATASTART
      00000000H   SYMBOL    NUMBER   ---       PPAGE
      00000000H   SYMBOL    NUMBER   ---       PPAGEENABLE
      000000A0H   SYMBOL    DATA     ---       PPAGE_SFR
      00000081H   SYMBOL    DATA     ---       SP
LX51 LINKER/LOCATER V4.66.41.0                                                        06/16/2023  10:23:34  PAGE 19


      01000BC7H   SYMBOL    CODE     ---       STARTUP1
      00000000H   SYMBOL    NUMBER   ---       XBPSTACK
      00000000H   SYMBOL    NUMBER   ---       XBPSTACKTOP
      00000000H   SYMBOL    NUMBER   ---       XDATALEN
      00000000H   SYMBOL    NUMBER   ---       XDATASTART
      01000000H   LINE      CODE     ---       #126
      01000BC7H   LINE      CODE     ---       #133
      01000BC9H   LINE      CODE     ---       #134
      01000BCAH   LINE      CODE     ---       #135
      01000BCBH   LINE      CODE     ---       #136
      01000BCDH   LINE      CODE     ---       #185
      01000BD0H   LINE      CODE     ---       #196

      ---         MODULE    ---      ---       MAIN
      0200FF00H   PUBLIC    XDATA    BYTE      P0M0
      0200FF42H   PUBLIC    XDATA    BYTE      P02DBC
      0200FE9CH   PUBLIC    XDATA    BYTE      ADCDLYH
      0200FF41H   PUBLIC    XDATA    BYTE      P01DBC
      0200FF52H   PUBLIC    XDATA    BYTE      P2OUT
      0200FF40H   PUBLIC    XDATA    BYTE      P00DBC
      0200FF51H   PUBLIC    XDATA    BYTE      P1OUT
      0200FF50H   PUBLIC    XDATA    BYTE      P0OUT
      0200FE9FH   PUBLIC    XDATA    BYTE      ADCGAPV
      0200FEEAH   PUBLIC    XDATA    BYTE      PWM2INTDIV
      0200FFA6H   PUBLIC    XDATA    BYTE      MOSI_MAP
      0200FFA7H   PUBLIC    XDATA    BYTE      MISO_MAP
      0200FEE9H   PUBLIC    XDATA    BYTE      PWM1INTDIV
      0200FEE8H   PUBLIC    XDATA    BYTE      PWM0INTDIV
      0200FF62H   PUBLIC    XDATA    BYTE      COMP2EN
      0200FF61H   PUBLIC    XDATA    BYTE      COMP1EN
      0200FEB3H   PUBLIC    XDATA    BYTE      PITS3
      0200FF60H   PUBLIC    XDATA    BYTE      COMP0EN
      0200FEB2H   PUBLIC    XDATA    BYTE      PITS2
      0200FEB1H   PUBLIC    XDATA    BYTE      PITS1
      0200FF05H   PUBLIC    XDATA    BYTE      P0LPU
      0200FEB0H   PUBLIC    XDATA    BYTE      PITS0
      0200FE96H   PUBLIC    XDATA    BYTE      LXTALSPD
      0200FECFH   PUBLIC    XDATA    BYTE      SCRL7
      0200FECDH   PUBLIC    XDATA    BYTE      SCRL6
      0200FE92H   PUBLIC    XDATA    BYTE      FREQ_CLK
      0200FECBH   PUBLIC    XDATA    BYTE      SCRL5
      0200FE97H   PUBLIC    XDATA    BYTE      DBGFLAG
      0200FEBCH   PUBLIC    XDATA    BYTE      INT01_PINS
      0200FEC9H   PUBLIC    XDATA    BYTE      SCRL4
      0200FF8FH   PUBLIC    XDATA    BYTE      CLKO_MAP
      0200FEC7H   PUBLIC    XDATA    BYTE      SCRL3
      0200FECEH   PUBLIC    XDATA    BYTE      SCRH7
      0200FEC5H   PUBLIC    XDATA    BYTE      SCRL2
      0200FECCH   PUBLIC    XDATA    BYTE      SCRH6
      0200FED9H   PUBLIC    XDATA    BYTE      CAPCON1
      0200FEE5H   PUBLIC    XDATA    BYTE      PWM2PHASEL
      0200FF9CH   PUBLIC    XDATA    BYTE      PWM3_MAP
      0200FE80H   PUBLIC    XDATA    BYTE      TCON1
      0200FE88H   PUBLIC    XDATA    BYTE      S2CON
      0200FEC3H   PUBLIC    XDATA    BYTE      SCRL1
      0200FECAH   PUBLIC    XDATA    BYTE      SCRH5
      0200FED8H   PUBLIC    XDATA    BYTE      CAPCON0
      0200FEE3H   PUBLIC    XDATA    BYTE      PWM1PHASEL
      0200FF98H   PUBLIC    XDATA    BYTE      PWM2_MAP
      0200FEC1H   PUBLIC    XDATA    BYTE      SCRL0
      0200FEC8H   PUBLIC    XDATA    BYTE      SCRH4
      0200FEE1H   PUBLIC    XDATA    BYTE      PWM0PHASEL
      0200FF94H   PUBLIC    XDATA    BYTE      PWM1_MAP
      0200FFA4H   PUBLIC    XDATA    BYTE      SS_MAP
      0200FEC6H   PUBLIC    XDATA    BYTE      SCRH3
LX51 LINKER/LOCATER V4.66.41.0                                                        06/16/2023  10:23:34  PAGE 20


      0200FF90H   PUBLIC    XDATA    BYTE      PWM0_MAP
      0200FE8AH   PUBLIC    XDATA    BYTE      S2BUF
      0200FE98H   PUBLIC    XDATA    BYTE      ADCWC
      0200FEC4H   PUBLIC    XDATA    BYTE      SCRH2
      0200FEE4H   PUBLIC    XDATA    BYTE      PWM2PHASEH
      0200FEC2H   PUBLIC    XDATA    BYTE      SCRH1
      0200FEE2H   PUBLIC    XDATA    BYTE      PWM1PHASEH
      0200FFA8H   PUBLIC    XDATA    BYTE      TXD2_MAP
      0200FEC0H   PUBLIC    XDATA    BYTE      SCRH0
      0200FEE0H   PUBLIC    XDATA    BYTE      PWM0PHASEH
      0200FFA9H   PUBLIC    XDATA    BYTE      RXD2_MAP
      0200FEEEH   PUBLIC    XDATA    BYTE      PWM3CLKS
      0200FE9EH   PUBLIC    XDATA    BYTE      ADCCONTV
      0200FE93H   PUBLIC    XDATA    BYTE      CLKOUT
      0200FEF1H   PUBLIC    XDATA    BYTE      PWM0CMPL
      0200FED3H   PUBLIC    XDATA    BYTE      CAPL1
      0200FED1H   PUBLIC    XDATA    BYTE      CAPL0
      0200FEF0H   PUBLIC    XDATA    BYTE      PWM0CMPH
      0200FE8BH   PUBLIC    XDATA    BYTE      BRTSEL
      0200FED2H   PUBLIC    XDATA    BYTE      CAPH1
      0200FED0H   PUBLIC    XDATA    BYTE      CAPH0
      0200FEBEH   PUBLIC    XDATA    BYTE      TRMV
      0200FEF8H   PUBLIC    XDATA    BYTE      PWMENA
      0200FEA0H   PUBLIC    XDATA    BYTE      WDTCCR
      0200FF85H   PUBLIC    XDATA    BYTE      T5_MAP
      0200FF84H   PUBLIC    XDATA    BYTE      T4_MAP
      0200FF83H   PUBLIC    XDATA    BYTE      T3_MAP
      0200FF89H   PUBLIC    XDATA    BYTE      CAP1_MAP
      0200FEAAH   PUBLIC    XDATA    BYTE      RSTDBC
      0200FF81H   PUBLIC    XDATA    BYTE      T1_MAP
      0200FF88H   PUBLIC    XDATA    BYTE      CAP0_MAP
      0200FF80H   PUBLIC    XDATA    BYTE      T0_MAP
      0200FE91H   PUBLIC    XDATA    BYTE      CLKDIV
      0200FE9AH   PUBLIC    XDATA    BYTE      ADCC3
      0200FE9BH   PUBLIC    XDATA    BYTE      ADCC2
      0200FEABH   PUBLIC    XDATA    BYTE      AWDCON
      0200FE95H   PUBLIC    XDATA    BYTE      SPOV_RSTEN
      0200FEB9H   PUBLIC    XDATA    BYTE      PINTE1
      0200FEB8H   PUBLIC    XDATA    BYTE      PINTE0
      0200FEA7H   PUBLIC    XDATA    BYTE      LVDDBC
      0200FF8DH   PUBLIC    XDATA    BYTE      ADCST_MAP
      0200FFA0H   PUBLIC    XDATA    BYTE      TXD_MAP
      0200FEA5H   PUBLIC    XDATA    BYTE      BORDBC
      0200FFA1H   PUBLIC    XDATA    BYTE      RXD_MAP
      0200FEA4H   PUBLIC    XDATA    BYTE      BORC
      0200FFA2H   PUBLIC    XDATA    BYTE      SCL_MAP
      0200FFA5H   PUBLIC    XDATA    BYTE      SCK_MAP
      0200FE86H   PUBLIC    XDATA    BYTE      T5CON2
      0200FE85H   PUBLIC    XDATA    BYTE      T5CON1
      0200FEA2H   PUBLIC    XDATA    BYTE      CRCC
      0200FE84H   PUBLIC    XDATA    BYTE      T4CON1
      0200FE89H   PUBLIC    XDATA    BYTE      S2CON2
      0200FF99H   PUBLIC    XDATA    BYTE      PWM21_MAP
      0200FFA3H   PUBLIC    XDATA    BYTE      SDA_MAP
      0200FF95H   PUBLIC    XDATA    BYTE      PWM11_MAP
      0200FF91H   PUBLIC    XDATA    BYTE      PWM01_MAP
      0200FE94H   PUBLIC    XDATA    BYTE      XTALCFG
      0200FEAFH   PUBLIC    XDATA    BYTE      ADCLTRL
      0200FEFBH   PUBLIC    XDATA    BYTE      PWMCON2
      0200FEBDH   PUBLIC    XDATA    BYTE      TRMEN
      0200FEFAH   PUBLIC    XDATA    BYTE      PWMCON1
      0200FEF9H   PUBLIC    XDATA    BYTE      PWMCON0
      0200FEADH   PUBLIC    XDATA    BYTE      ADCHTRL
      0200FEAEH   PUBLIC    XDATA    BYTE      ADCLTRH
      0200FF13H   PUBLIC    XDATA    BYTE      P2M3
LX51 LINKER/LOCATER V4.66.41.0                                                        06/16/2023  10:23:34  PAGE 21


      0200FF12H   PUBLIC    XDATA    BYTE      P2M2
      0200FEACH   PUBLIC    XDATA    BYTE      ADCHTRH
      0200FF03H   PUBLIC    XDATA    BYTE      P0M3
      0200FF11H   PUBLIC    XDATA    BYTE      P2M1
      0200FE9DH   PUBLIC    XDATA    BYTE      ADCDLYL
      0200FF02H   PUBLIC    XDATA    BYTE      P0M2
      0200FF10H   PUBLIC    XDATA    BYTE      P2M0
      0200FF01H   PUBLIC    XDATA    BYTE      P0M1
      0200FF08H   PUBLIC    XDATA    BYTE      P1M0
      01000E82H   PUBLIC    CODE     ---       main
      00000080H   SFRSYM    DATA     BYTE      P0
      00000090H   SFRSYM    DATA     BYTE      P1
      000000A0H   SFRSYM    DATA     BYTE      P2
      000000D0H.6 SFRSYM    DATA     BIT       AC
      000000A8H.7 SFRSYM    DATA     BIT       EA
      000000E7H   SFRSYM    DATA     BYTE      PWM0DTH
      000000CAH   SFRSYM    DATA     WORD      T3
      000000EFH   SFRSYM    DATA     BYTE      PWM1DTH
      000000ACH   SFRSYM    DATA     BYTE      SPCTL
      000000CDH   SFRSYM    DATA     WORD      T4
      000000F8H.4 SFRSYM    DATA     BIT       WDTRF
      000000F7H   SFRSYM    DATA     BYTE      PWM2DTH
      000000C2H   SFRSYM    DATA     WORD      T5
      00000098H.7 SFRSYM    DATA     BIT       FE
      000000E6H   SFRSYM    DATA     BYTE      PWM0DTL
      00000098H.5 SFRSYM    DATA     BIT       TXCOL
      000000EEH   SFRSYM    DATA     BYTE      PWM1DTL
      000000F6H   SFRSYM    DATA     BYTE      PWM2DTL
      000000B8H.5 SFRSYM    DATA     BIT       EADC
      00000091H   SFRSYM    DATA     BYTE      TICKCON
      000000A8H   SFRSYM    DATA     BYTE      IE
      00000080H   SFRSYM    DATA     BIT       P0_0
      000000F8H.1 SFRSYM    DATA     BIT       SPOVF
      000000FCH   SFRSYM    DATA     WORD      IAP_CMD
      00000090H   SFRSYM    DATA     BIT       P1_0
      00000080H.1 SFRSYM    DATA     BIT       P0_1
      000000A0H   SFRSYM    DATA     BIT       P2_0
      00000090H.1 SFRSYM    DATA     BIT       P1_1
      00000080H.2 SFRSYM    DATA     BIT       P0_2
      000000A0H.1 SFRSYM    DATA     BIT       P2_1
      00000080H.3 SFRSYM    DATA     BIT       P0_3
      000000F8H   SFRSYM    DATA     BYTE      RSTFR
      000000A0H.2 SFRSYM    DATA     BIT       P2_2
      00000080H.4 SFRSYM    DATA     BIT       P0_4
      000000A0H.3 SFRSYM    DATA     BIT       P2_3
      00000080H.5 SFRSYM    DATA     BIT       P0_5
      000000A0H.4 SFRSYM    DATA     BIT       P2_4
      00000080H.6 SFRSYM    DATA     BIT       P0_6
      000000A0H.5 SFRSYM    DATA     BIT       P2_5
      00000080H.7 SFRSYM    DATA     BIT       P0_7
      000000A0H.6 SFRSYM    DATA     BIT       P2_6
      000000A0H.7 SFRSYM    DATA     BIT       P2_7
      00000098H   SFRSYM    DATA     BIT       RI
      000000B8H.3 SFRSYM    DATA     BIT       EIIC
      000000B6H   SFRSYM    DATA     WORD      ADCR
      000000B8H.7 SFRSYM    DATA     BIT       EX8_15
      000000D0H.7 SFRSYM    DATA     BIT       CY
      00000098H.1 SFRSYM    DATA     BIT       TI
      000000FAH   SFRSYM    DATA     BYTE      IAP_ADDRH
      000000BFH   SFRSYM    DATA     BYTE      CRCH
      00000098H.6 SFRSYM    DATA     BIT       RXROV
      00000081H   SFRSYM    DATA     BYTE      SP
      000000F9H   SFRSYM    DATA     BYTE      IAP_ADDRL
      000000D0H.2 SFRSYM    DATA     BIT       OV
      000000BEH   SFRSYM    DATA     BYTE      CRCL
LX51 LINKER/LOCATER V4.66.41.0                                                        06/16/2023  10:23:34  PAGE 22


      000000C5H   SFRSYM    DATA     BYTE      RCAP5H
      000000C4H   SFRSYM    DATA     BYTE      RCAP5L
      000000F8H.5 SFRSYM    DATA     BIT       BORF
      000000BBH   SFRSYM    DATA     BYTE      LVDC
      000000BEH   SFRSYM    DATA     WORD      CRCR
      000000AFH   SFRSYM    DATA     BYTE      IICADR
      000000AEH   SFRSYM    DATA     BYTE      IICDAT
      00000099H   SFRSYM    DATA     BYTE      SBUF
      00000087H   SFRSYM    DATA     BYTE      PCON
      000000B8H   SFRSYM    DATA     BIT       ESPI
      000000E5H   SFRSYM    DATA     BYTE      PWM0DH
      000000EDH   SFRSYM    DATA     BYTE      PWM1DH
      00000096H   SFRSYM    DATA     BYTE      PINTF0
      000000BDH   SFRSYM    DATA     BYTE      WDTC
      000000F8H   SFRSYM    DATA     BIT       PLVRSTF
      000000F5H   SFRSYM    DATA     BYTE      PWM2DH
      00000098H   SFRSYM    DATA     BYTE      SCON
      00000097H   SFRSYM    DATA     BYTE      PINTF1
      000000A8H.5 SFRSYM    DATA     BIT       EWDT
      000000D1H   SFRSYM    DATA     BYTE      LCDCON
      00000089H   SFRSYM    DATA     BYTE      TMOD
      00000088H   SFRSYM    DATA     BYTE      TCON
      000000E4H   SFRSYM    DATA     BYTE      PWM0DL
      000000ECH   SFRSYM    DATA     BYTE      PWM1DL
      000000A6H   SFRSYM    DATA     BYTE      IICCON
      000000F8H.7 SFRSYM    DATA     BIT       PORF
      000000F4H   SFRSYM    DATA     BYTE      PWM2DL
      000000E1H   SFRSYM    DATA     BYTE      PWM0EN
      000000E9H   SFRSYM    DATA     BYTE      PWM1EN
      000000F1H   SFRSYM    DATA     BYTE      PWM2EN
      00000082H   SFRSYM    DATA     WORD      DPTR
      000000B4H   SFRSYM    DATA     BYTE      ADCC0
      0000008FH   SFRSYM    DATA     BYTE      CLKCON
      000000B5H   SFRSYM    DATA     BYTE      ADCC1
      000000E6H   SFRSYM    DATA     WORD      PWM0DT
      000000E3H   SFRSYM    DATA     BYTE      PWM0PH
      000000EEH   SFRSYM    DATA     WORD      PWM1DT
      000000EBH   SFRSYM    DATA     BYTE      PWM1PH
      000000A7H   SFRSYM    DATA     BYTE      IICSTA
      000000B8H   SFRSYM    DATA     BYTE      IE1
      000000F6H   SFRSYM    DATA     WORD      PWM2DT
      000000F3H   SFRSYM    DATA     BYTE      PWM2PH
      000000F0H   SFRSYM    DATA     BYTE      B
      000000E2H   SFRSYM    DATA     BYTE      PWM0PL
      000000F8H.3 SFRSYM    DATA     BIT       SWRF
      000000EAH   SFRSYM    DATA     BYTE      PWM1PL
      000000F2H   SFRSYM    DATA     BYTE      PWM2PL
      000000E0H   SFRSYM    DATA     BYTE      ACC
      000000BCH   SFRSYM    DATA     BYTE      LVDCMP
      000000A8H.1 SFRSYM    DATA     BIT       ET0
      000000A8H.4 SFRSYM    DATA     BIT       ES1
      000000A9H   SFRSYM    DATA     BYTE      IP0
      00000088H.5 SFRSYM    DATA     BIT       TF0
      000000A8H.3 SFRSYM    DATA     BIT       ET1
      000000A8H.6 SFRSYM    DATA     BIT       ES2
      000000AAH   SFRSYM    DATA     BYTE      IP1
      00000088H.7 SFRSYM    DATA     BIT       TF1
      000000B9H   SFRSYM    DATA     BYTE      IP2
      00000098H.2 SFRSYM    DATA     BIT       RB8
      000000B8H.1 SFRSYM    DATA     BIT       ET3
      0000008CH   SFRSYM    DATA     BYTE      TH0
      000000BAH   SFRSYM    DATA     BYTE      IP3
      000000A2H   SFRSYM    DATA     BYTE      INSCON
      000000B8H.2 SFRSYM    DATA     BIT       ET4
      000000A8H   SFRSYM    DATA     BIT       EX0
LX51 LINKER/LOCATER V4.66.41.0                                                        06/16/2023  10:23:34  PAGE 23


      0000008DH   SFRSYM    DATA     BYTE      TH1
      000000B1H   SFRSYM    DATA     BYTE      IP4
      00000098H.3 SFRSYM    DATA     BIT       TB8
      000000B8H.4 SFRSYM    DATA     BIT       ET5
      000000A8H.2 SFRSYM    DATA     BIT       EX1
      000000D0H   SFRSYM    DATA     BIT       P
      000000CBH   SFRSYM    DATA     BYTE      TH3
      000000CEH   SFRSYM    DATA     BYTE      TH4
      0000008AH   SFRSYM    DATA     BYTE      TL0
      000000C3H   SFRSYM    DATA     BYTE      TH5
      0000008BH   SFRSYM    DATA     BYTE      TL1
      000000CAH   SFRSYM    DATA     BYTE      TL3
      000000CDH   SFRSYM    DATA     BYTE      TL4
      000000D0H.3 SFRSYM    DATA     BIT       RS0
      000000C2H   SFRSYM    DATA     BYTE      TL5
      00000088H.4 SFRSYM    DATA     BIT       TR0
      000000D0H.4 SFRSYM    DATA     BIT       RS1
      000000FBH   SFRSYM    DATA     BYTE      IAP_DATA
      00000088H.6 SFRSYM    DATA     BIT       TR1
      000000F9H   SFRSYM    DATA     WORD      IAP_ADDR
      000000FDH   SFRSYM    DATA     BYTE      IAP_CMDH
      0000008EH   SFRSYM    DATA     BYTE      CLKSWR
      000000C4H   SFRSYM    DATA     WORD      RCAP5
      000000FCH   SFRSYM    DATA     BYTE      IAP_CMDL
      00000083H   SFRSYM    DATA     BYTE      DPH
      000000F8H.6 SFRSYM    DATA     BIT       EXRSTF
      00000082H   SFRSYM    DATA     BYTE      DPL
      000000ADH   SFRSYM    DATA     BYTE      SPSTAT
      000000B7H   SFRSYM    DATA     BYTE      ADCRH
      00000098H.4 SFRSYM    DATA     BIT       REN
      000000B8H.6 SFRSYM    DATA     BIT       EX2_7
      0000009EH   SFRSYM    DATA     BYTE      SCON2
      000000B6H   SFRSYM    DATA     BYTE      ADCRL
      000000DAH   SFRSYM    DATA     BYTE      PWM0C
      000000C9H   SFRSYM    DATA     BYTE      T3CON
      000000E4H   SFRSYM    DATA     WORD      PWM0D
      000000DBH   SFRSYM    DATA     BYTE      PWM1C
      000000CCH   SFRSYM    DATA     BYTE      T4CON
      000000ECH   SFRSYM    DATA     WORD      PWM1D
      000000DCH   SFRSYM    DATA     BYTE      PWM2C
      000000C1H   SFRSYM    DATA     BYTE      T5CON
      000000F4H   SFRSYM    DATA     WORD      PWM2D
      000000DDH   SFRSYM    DATA     BYTE      PWM3C
      000000DFH   SFRSYM    DATA     BYTE      PWM3D
      0000009BH   SFRSYM    DATA     BYTE      SADEN
      0000009AH   SFRSYM    DATA     BYTE      SADDR
      00000093H   SFRSYM    DATA     BYTE      TICKH
      000000D0H.5 SFRSYM    DATA     BIT       F0
      000000E2H   SFRSYM    DATA     WORD      PWM0P
      000000D0H.1 SFRSYM    DATA     BIT       F1
      000000EAH   SFRSYM    DATA     WORD      PWM1P
      000000F2H   SFRSYM    DATA     WORD      PWM2P
      000000DEH   SFRSYM    DATA     BYTE      PWM3P
      00000092H   SFRSYM    DATA     BYTE      TICKL
      000000D0H   SFRSYM    DATA     BYTE      PSW
      000000ABH   SFRSYM    DATA     BYTE      SPDAT

      01000E82H   BLOCK     CODE     ---       LVL=0
      01000E82H   LINE      CODE     ---       #50
      01000E82H   LINE      CODE     ---       #51
      01000E82H   LINE      CODE     ---       #52
      01000E85H   LINE      CODE     ---       #53
      01000E88H   LINE      CODE     ---       #54
      01000E8BH   LINE      CODE     ---       #56
      01000E8EH   LINE      CODE     ---       #57
LX51 LINKER/LOCATER V4.66.41.0                                                        06/16/2023  10:23:34  PAGE 24


      01000E97H   LINE      CODE     ---       #79
      01000E99H   LINE      CODE     ---       #81
      01000E99H   LINE      CODE     ---       #82
      01000E99H   LINE      CODE     ---       #83
      01000E9CH   LINE      CODE     ---       #84
      01000E9FH   LINE      CODE     ---       #85
      01000EA2H   LINE      CODE     ---       #87
      01000EA2H   LINE      CODE     ---       #88
      01000EA2H   LINE      CODE     ---       #89
      01000EA2H   LINE      CODE     ---       #90
      01000EA2H   LINE      CODE     ---       #92
      01000EB4H   LINE      CODE     ---       #93
      01000EB4H   LINE      CODE     ---       #94
      01000EB4H   LINE      CODE     ---       #95
      01000EB4H   LINE      CODE     ---       #97
      01000EBDH   LINE      CODE     ---       #99
      01000EC0H   LINE      CODE     ---       #100
      01000EC6H   LINE      CODE     ---       #102
      01000ECFH   LINE      CODE     ---       #104
      ---         BLOCKEND  ---      ---       LVL=0

      ---         MODULE    ---      ---       USER
      0200006FH   PUBLIC    XDATA    BYTE      u8_rtc_hour
      00000021H.7 PUBLIC    BIT      BIT       b_pwmen_flag
      00000021H.6 PUBLIC    BIT      BIT       b_aden_flag
      0200004CH   PUBLIC    XDATA    ---       rf
      0200004BH   PUBLIC    XDATA    BYTE      u8_rtc_minute
      0200004AH   PUBLIC    XDATA    BYTE      u8_delay_int
      02000049H   PUBLIC    XDATA    BYTE      u8_wake_time
      02000047H   PUBLIC    XDATA    WORD      u16_cnt_3_int
      02000046H   PUBLIC    XDATA    BYTE      u8_rtc_second
      02000044H   PUBLIC    XDATA    WORD      u16_ad_val
      02000043H   PUBLIC    XDATA    BYTE      u8_led2_cnt
      02000042H   PUBLIC    XDATA    BYTE      u8_led1_cnt
      02000041H   PUBLIC    XDATA    BYTE      u8_cnt_2_int
      02000040H   PUBLIC    XDATA    BYTE      u8_cnt_1_int
      0200003CH   PUBLIC    XDATA    DWORD     u32_tmp
      0200003AH   PUBLIC    XDATA    WORD      u16_wave_time
      00000021H.5 PUBLIC    BIT      BIT       b_base_1ms_int
      01000B30H   PUBLIC    CODE     ---       system_timer_pro
      0100003EH   PUBLIC    CODE     ---       system_flow_control
      010010A1H   PUBLIC    CODE     ---       user_key_pro
      0100122EH   PUBLIC    CODE     ---       user_register_initial
      01000F20H   PUBLIC    CODE     ---       user_gpio_initial
      00000080H   SFRSYM    DATA     BYTE      P0
      00000090H   SFRSYM    DATA     BYTE      P1
      000000A0H   SFRSYM    DATA     BYTE      P2
      000000D0H.6 SFRSYM    DATA     BIT       AC
      000000A8H.7 SFRSYM    DATA     BIT       EA
      000000E7H   SFRSYM    DATA     BYTE      PWM0DTH
      000000CAH   SFRSYM    DATA     WORD      T3
      000000EFH   SFRSYM    DATA     BYTE      PWM1DTH
      000000ACH   SFRSYM    DATA     BYTE      SPCTL
      000000CDH   SFRSYM    DATA     WORD      T4
      000000F8H.4 SFRSYM    DATA     BIT       WDTRF
      000000F7H   SFRSYM    DATA     BYTE      PWM2DTH
      000000C2H   SFRSYM    DATA     WORD      T5
      00000098H.7 SFRSYM    DATA     BIT       FE
      000000E6H   SFRSYM    DATA     BYTE      PWM0DTL
      00000098H.5 SFRSYM    DATA     BIT       TXCOL
      000000EEH   SFRSYM    DATA     BYTE      PWM1DTL
      000000F6H   SFRSYM    DATA     BYTE      PWM2DTL
      000000B8H.5 SFRSYM    DATA     BIT       EADC
      00000091H   SFRSYM    DATA     BYTE      TICKCON
      000000A8H   SFRSYM    DATA     BYTE      IE
LX51 LINKER/LOCATER V4.66.41.0                                                        06/16/2023  10:23:34  PAGE 25


      00000080H   SFRSYM    DATA     BIT       P0_0
      000000F8H.1 SFRSYM    DATA     BIT       SPOVF
      000000FCH   SFRSYM    DATA     WORD      IAP_CMD
      00000090H   SFRSYM    DATA     BIT       P1_0
      00000080H.1 SFRSYM    DATA     BIT       P0_1
      000000A0H   SFRSYM    DATA     BIT       P2_0
      00000090H.1 SFRSYM    DATA     BIT       P1_1
      00000080H.2 SFRSYM    DATA     BIT       P0_2
      000000A0H.1 SFRSYM    DATA     BIT       P2_1
      00000080H.3 SFRSYM    DATA     BIT       P0_3
      000000F8H   SFRSYM    DATA     BYTE      RSTFR
      000000A0H.2 SFRSYM    DATA     BIT       P2_2
      00000080H.4 SFRSYM    DATA     BIT       P0_4
      000000A0H.3 SFRSYM    DATA     BIT       P2_3
      00000080H.5 SFRSYM    DATA     BIT       P0_5
      000000A0H.4 SFRSYM    DATA     BIT       P2_4
      00000080H.6 SFRSYM    DATA     BIT       P0_6
      000000A0H.5 SFRSYM    DATA     BIT       P2_5
      00000080H.7 SFRSYM    DATA     BIT       P0_7
      000000A0H.6 SFRSYM    DATA     BIT       P2_6
      000000A0H.7 SFRSYM    DATA     BIT       P2_7
      00000098H   SFRSYM    DATA     BIT       RI
      000000B8H.3 SFRSYM    DATA     BIT       EIIC
      000000B6H   SFRSYM    DATA     WORD      ADCR
      000000B8H.7 SFRSYM    DATA     BIT       EX8_15
      000000D0H.7 SFRSYM    DATA     BIT       CY
      00000098H.1 SFRSYM    DATA     BIT       TI
      000000FAH   SFRSYM    DATA     BYTE      IAP_ADDRH
      000000BFH   SFRSYM    DATA     BYTE      CRCH
      00000098H.6 SFRSYM    DATA     BIT       RXROV
      00000081H   SFRSYM    DATA     BYTE      SP
      000000F9H   SFRSYM    DATA     BYTE      IAP_ADDRL
      000000D0H.2 SFRSYM    DATA     BIT       OV
      000000BEH   SFRSYM    DATA     BYTE      CRCL
      000000C5H   SFRSYM    DATA     BYTE      RCAP5H
      000000C4H   SFRSYM    DATA     BYTE      RCAP5L
      000000F8H.5 SFRSYM    DATA     BIT       BORF
      000000BBH   SFRSYM    DATA     BYTE      LVDC
      000000BEH   SFRSYM    DATA     WORD      CRCR
      000000AFH   SFRSYM    DATA     BYTE      IICADR
      000000AEH   SFRSYM    DATA     BYTE      IICDAT
      00000099H   SFRSYM    DATA     BYTE      SBUF
      00000087H   SFRSYM    DATA     BYTE      PCON
      000000B8H   SFRSYM    DATA     BIT       ESPI
      000000E5H   SFRSYM    DATA     BYTE      PWM0DH
      000000EDH   SFRSYM    DATA     BYTE      PWM1DH
      00000096H   SFRSYM    DATA     BYTE      PINTF0
      000000BDH   SFRSYM    DATA     BYTE      WDTC
      000000F8H   SFRSYM    DATA     BIT       PLVRSTF
      000000F5H   SFRSYM    DATA     BYTE      PWM2DH
      00000098H   SFRSYM    DATA     BYTE      SCON
      00000097H   SFRSYM    DATA     BYTE      PINTF1
      000000A8H.5 SFRSYM    DATA     BIT       EWDT
      000000D1H   SFRSYM    DATA     BYTE      LCDCON
      00000089H   SFRSYM    DATA     BYTE      TMOD
      00000088H   SFRSYM    DATA     BYTE      TCON
      000000E4H   SFRSYM    DATA     BYTE      PWM0DL
      000000ECH   SFRSYM    DATA     BYTE      PWM1DL
      000000A6H   SFRSYM    DATA     BYTE      IICCON
      000000F8H.7 SFRSYM    DATA     BIT       PORF
      000000F4H   SFRSYM    DATA     BYTE      PWM2DL
      000000E1H   SFRSYM    DATA     BYTE      PWM0EN
      000000E9H   SFRSYM    DATA     BYTE      PWM1EN
      000000F1H   SFRSYM    DATA     BYTE      PWM2EN
      00000082H   SFRSYM    DATA     WORD      DPTR
LX51 LINKER/LOCATER V4.66.41.0                                                        06/16/2023  10:23:34  PAGE 26


      000000B4H   SFRSYM    DATA     BYTE      ADCC0
      0000008FH   SFRSYM    DATA     BYTE      CLKCON
      000000B5H   SFRSYM    DATA     BYTE      ADCC1
      000000E6H   SFRSYM    DATA     WORD      PWM0DT
      000000E3H   SFRSYM    DATA     BYTE      PWM0PH
      000000EEH   SFRSYM    DATA     WORD      PWM1DT
      000000EBH   SFRSYM    DATA     BYTE      PWM1PH
      000000A7H   SFRSYM    DATA     BYTE      IICSTA
      000000B8H   SFRSYM    DATA     BYTE      IE1
      000000F6H   SFRSYM    DATA     WORD      PWM2DT
      000000F3H   SFRSYM    DATA     BYTE      PWM2PH
      000000F0H   SFRSYM    DATA     BYTE      B
      000000E2H   SFRSYM    DATA     BYTE      PWM0PL
      000000F8H.3 SFRSYM    DATA     BIT       SWRF
      000000EAH   SFRSYM    DATA     BYTE      PWM1PL
      000000F2H   SFRSYM    DATA     BYTE      PWM2PL
      000000E0H   SFRSYM    DATA     BYTE      ACC
      000000BCH   SFRSYM    DATA     BYTE      LVDCMP
      000000A8H.1 SFRSYM    DATA     BIT       ET0
      000000A8H.4 SFRSYM    DATA     BIT       ES1
      000000A9H   SFRSYM    DATA     BYTE      IP0
      00000088H.5 SFRSYM    DATA     BIT       TF0
      000000A8H.3 SFRSYM    DATA     BIT       ET1
      000000A8H.6 SFRSYM    DATA     BIT       ES2
      000000AAH   SFRSYM    DATA     BYTE      IP1
      00000088H.7 SFRSYM    DATA     BIT       TF1
      000000B9H   SFRSYM    DATA     BYTE      IP2
      00000098H.2 SFRSYM    DATA     BIT       RB8
      000000B8H.1 SFRSYM    DATA     BIT       ET3
      0000008CH   SFRSYM    DATA     BYTE      TH0
      000000BAH   SFRSYM    DATA     BYTE      IP3
      000000A2H   SFRSYM    DATA     BYTE      INSCON
      000000B8H.2 SFRSYM    DATA     BIT       ET4
      000000A8H   SFRSYM    DATA     BIT       EX0
      0000008DH   SFRSYM    DATA     BYTE      TH1
      000000B1H   SFRSYM    DATA     BYTE      IP4
      00000098H.3 SFRSYM    DATA     BIT       TB8
      000000B8H.4 SFRSYM    DATA     BIT       ET5
      000000A8H.2 SFRSYM    DATA     BIT       EX1
      000000D0H   SFRSYM    DATA     BIT       P
      000000CBH   SFRSYM    DATA     BYTE      TH3
      000000CEH   SFRSYM    DATA     BYTE      TH4
      0000008AH   SFRSYM    DATA     BYTE      TL0
      000000C3H   SFRSYM    DATA     BYTE      TH5
      0000008BH   SFRSYM    DATA     BYTE      TL1
      000000CAH   SFRSYM    DATA     BYTE      TL3
      000000CDH   SFRSYM    DATA     BYTE      TL4
      000000D0H.3 SFRSYM    DATA     BIT       RS0
      000000C2H   SFRSYM    DATA     BYTE      TL5
      00000088H.4 SFRSYM    DATA     BIT       TR0
      000000D0H.4 SFRSYM    DATA     BIT       RS1
      000000FBH   SFRSYM    DATA     BYTE      IAP_DATA
      00000088H.6 SFRSYM    DATA     BIT       TR1
      000000F9H   SFRSYM    DATA     WORD      IAP_ADDR
      000000FDH   SFRSYM    DATA     BYTE      IAP_CMDH
      0000008EH   SFRSYM    DATA     BYTE      CLKSWR
      000000C4H   SFRSYM    DATA     WORD      RCAP5
      000000FCH   SFRSYM    DATA     BYTE      IAP_CMDL
      00000083H   SFRSYM    DATA     BYTE      DPH
      000000F8H.6 SFRSYM    DATA     BIT       EXRSTF
      00000082H   SFRSYM    DATA     BYTE      DPL
      000000ADH   SFRSYM    DATA     BYTE      SPSTAT
      000000B7H   SFRSYM    DATA     BYTE      ADCRH
      00000098H.4 SFRSYM    DATA     BIT       REN
      000000B8H.6 SFRSYM    DATA     BIT       EX2_7
LX51 LINKER/LOCATER V4.66.41.0                                                        06/16/2023  10:23:34  PAGE 27


      0000009EH   SFRSYM    DATA     BYTE      SCON2
      000000B6H   SFRSYM    DATA     BYTE      ADCRL
      000000DAH   SFRSYM    DATA     BYTE      PWM0C
      000000C9H   SFRSYM    DATA     BYTE      T3CON
      000000E4H   SFRSYM    DATA     WORD      PWM0D
      000000DBH   SFRSYM    DATA     BYTE      PWM1C
      000000CCH   SFRSYM    DATA     BYTE      T4CON
      000000ECH   SFRSYM    DATA     WORD      PWM1D
      000000DCH   SFRSYM    DATA     BYTE      PWM2C
      000000C1H   SFRSYM    DATA     BYTE      T5CON
      000000F4H   SFRSYM    DATA     WORD      PWM2D
      000000DDH   SFRSYM    DATA     BYTE      PWM3C
      000000DFH   SFRSYM    DATA     BYTE      PWM3D
      0000009BH   SFRSYM    DATA     BYTE      SADEN
      0000009AH   SFRSYM    DATA     BYTE      SADDR
      00000093H   SFRSYM    DATA     BYTE      TICKH
      000000D0H.5 SFRSYM    DATA     BIT       F0
      000000E2H   SFRSYM    DATA     WORD      PWM0P
      000000D0H.1 SFRSYM    DATA     BIT       F1
      000000EAH   SFRSYM    DATA     WORD      PWM1P
      000000F2H   SFRSYM    DATA     WORD      PWM2P
      000000DEH   SFRSYM    DATA     BYTE      PWM3P
      00000092H   SFRSYM    DATA     BYTE      TICKL
      000000D0H   SFRSYM    DATA     BYTE      PSW
      000000ABH   SFRSYM    DATA     BYTE      SPDAT

      01000F20H   BLOCK     CODE     ---       LVL=0
      01000F20H   LINE      CODE     ---       #26
      01000F20H   LINE      CODE     ---       #27
      01000F20H   LINE      CODE     ---       #28
      01000F29H   LINE      CODE     ---       #29
      01000F2BH   LINE      CODE     ---       #31
      01000F34H   LINE      CODE     ---       #32
      01000F36H   LINE      CODE     ---       #34
      01000F3CH   LINE      CODE     ---       #35
      01000F3EH   LINE      CODE     ---       #37
      01000F47H   LINE      CODE     ---       #38
      01000F49H   LINE      CODE     ---       #40
      01000F4FH   LINE      CODE     ---       #41
      01000F51H   LINE      CODE     ---       #43
      01000F5AH   LINE      CODE     ---       #45
      01000F63H   LINE      CODE     ---       #47
      01000F69H   LINE      CODE     ---       #48
      ---         BLOCKEND  ---      ---       LVL=0

      0100122EH   BLOCK     CODE     ---       LVL=0
      0100122EH   LINE      CODE     ---       #59
      0100122EH   LINE      CODE     ---       #60
      0100122EH   LINE      CODE     ---       #61
      01001230H   LINE      CODE     ---       #62
      01001232H   LINE      CODE     ---       #63
      01001237H   LINE      CODE     ---       #64
      01001239H   LINE      CODE     ---       #65
      0100123FH   LINE      CODE     ---       #66
      ---         BLOCKEND  ---      ---       LVL=0

      010010A1H   BLOCK     CODE     ---       LVL=0
      010010A1H   LINE      CODE     ---       #78
      010010A1H   LINE      CODE     ---       #79
      010010A1H   LINE      CODE     ---       #80
      010010A4H   LINE      CODE     ---       #81
      010010A4H   LINE      CODE     ---       #82
      010010A6H   LINE      CODE     ---       #84
      010010A9H   LINE      CODE     ---       #85
      010010A9H   LINE      CODE     ---       #86
LX51 LINKER/LOCATER V4.66.41.0                                                        06/16/2023  10:23:34  PAGE 28


      010010ABH   LINE      CODE     ---       #87
      010010B8H   LINE      CODE     ---       #89
      010010B8H   LINE      CODE     ---       #90
      010010B8H   LINE      CODE     ---       #92
      010010BBH   LINE      CODE     ---       #93
      010010BBH   LINE      CODE     ---       #94
      010010BDH   LINE      CODE     ---       #96
      010010C0H   LINE      CODE     ---       #97
      010010C0H   LINE      CODE     ---       #98
      010010C2H   LINE      CODE     ---       #99
      010010C7H   LINE      CODE     ---       #100
      010010C7H   LINE      CODE     ---       #101
      010010C7H   LINE      CODE     ---       #103
      010010CAH   LINE      CODE     ---       #104
      010010CAH   LINE      CODE     ---       #105
      010010CCH   LINE      CODE     ---       #107
      010010CEH   LINE      CODE     ---       #108
      010010CEH   LINE      CODE     ---       #110
      010010D1H   LINE      CODE     ---       #111
      010010D1H   LINE      CODE     ---       #112
      010010D3H   LINE      CODE     ---       #114
      010010D5H   LINE      CODE     ---       #115
      010010D5H   LINE      CODE     ---       #116
      ---         BLOCKEND  ---      ---       LVL=0

      0100003EH   BLOCK     CODE     ---       LVL=0
      0100003EH   LINE      CODE     ---       #206
      0100003EH   LINE      CODE     ---       #207
      0100003EH   LINE      CODE     ---       #208
      ---         BLOCKEND  ---      ---       LVL=0

      01000B30H   BLOCK     CODE     ---       LVL=0
      01000B30H   LINE      CODE     ---       #227
      01000B30H   LINE      CODE     ---       #228
      01000B30H   LINE      CODE     ---       #230
      01000B33H   LINE      CODE     ---       #231
      01000B33H   LINE      CODE     ---       #232
      01000B35H   LINE      CODE     ---       #234
      01000B37H   LINE      CODE     ---       #238
      01000B37H   LINE      CODE     ---       #242
      01000B40H   LINE      CODE     ---       #243
      01000B40H   LINE      CODE     ---       #244
      01000B42H   LINE      CODE     ---       #246
      01000B45H   LINE      CODE     ---       #248
      01000B4BH   LINE      CODE     ---       #249
      01000B4BH   LINE      CODE     ---       #253
      01000B54H   LINE      CODE     ---       #254
      01000B54H   LINE      CODE     ---       #255
      01000B56H   LINE      CODE     ---       #257
      01000B5AH   LINE      CODE     ---       #258
      01000B5FH   LINE      CODE     ---       #259
      01000B5FH   LINE      CODE     ---       #260
      01000B61H   LINE      CODE     ---       #261
      01000B63H   LINE      CODE     ---       #262
      01000B63H   LINE      CODE     ---       #264
      01000B69H   LINE      CODE     ---       #265
      01000B69H   LINE      CODE     ---       #266
      01000B6BH   LINE      CODE     ---       #267
      01000B6BH   LINE      CODE     ---       #268
      01000B6BH   LINE      CODE     ---       #272
      01000B7AH   LINE      CODE     ---       #273
      01000B7AH   LINE      CODE     ---       #274
      01000B7EH   LINE      CODE     ---       #276
      01000B81H   LINE      CODE     ---       #277
      01000B81H   LINE      CODE     ---       #278
LX51 LINKER/LOCATER V4.66.41.0                                                        06/16/2023  10:23:34  PAGE 29


      01000B8EH   LINE      CODE     ---       #280
      01000BACH   LINE      CODE     ---       #281
      01000BC6H   LINE      CODE     ---       #283
      01000BC6H   LINE      CODE     ---       #284
      01000BC6H   LINE      CODE     ---       #285
      ---         BLOCKEND  ---      ---       LVL=0

      ---         MODULE    ---      ---       KEY
      00000021H.4 PUBLIC    BIT      BIT       b_key2_short_trig
      00000021H.3 PUBLIC    BIT      BIT       b_key1_short_trig
      00000021H.2 PUBLIC    BIT      BIT       b_key2_long_trig
      00000021H.1 PUBLIC    BIT      BIT       b_key1_long_trig
      01000789H   PUBLIC    CODE     ---       task_key_scan
      00000080H   SFRSYM    DATA     BYTE      P0
      00000090H   SFRSYM    DATA     BYTE      P1
      000000A0H   SFRSYM    DATA     BYTE      P2
      000000D0H.6 SFRSYM    DATA     BIT       AC
      000000A8H.7 SFRSYM    DATA     BIT       EA
      000000E7H   SFRSYM    DATA     BYTE      PWM0DTH
      000000CAH   SFRSYM    DATA     WORD      T3
      000000EFH   SFRSYM    DATA     BYTE      PWM1DTH
      000000ACH   SFRSYM    DATA     BYTE      SPCTL
      000000CDH   SFRSYM    DATA     WORD      T4
      000000F8H.4 SFRSYM    DATA     BIT       WDTRF
      000000F7H   SFRSYM    DATA     BYTE      PWM2DTH
      000000C2H   SFRSYM    DATA     WORD      T5
      00000098H.7 SFRSYM    DATA     BIT       FE
      000000E6H   SFRSYM    DATA     BYTE      PWM0DTL
      00000098H.5 SFRSYM    DATA     BIT       TXCOL
      000000EEH   SFRSYM    DATA     BYTE      PWM1DTL
      000000F6H   SFRSYM    DATA     BYTE      PWM2DTL
      000000B8H.5 SFRSYM    DATA     BIT       EADC
      00000091H   SFRSYM    DATA     BYTE      TICKCON
      000000A8H   SFRSYM    DATA     BYTE      IE
      00000080H   SFRSYM    DATA     BIT       P0_0
      000000F8H.1 SFRSYM    DATA     BIT       SPOVF
      000000FCH   SFRSYM    DATA     WORD      IAP_CMD
      00000090H   SFRSYM    DATA     BIT       P1_0
      00000080H.1 SFRSYM    DATA     BIT       P0_1
      000000A0H   SFRSYM    DATA     BIT       P2_0
      00000090H.1 SFRSYM    DATA     BIT       P1_1
      00000080H.2 SFRSYM    DATA     BIT       P0_2
      000000A0H.1 SFRSYM    DATA     BIT       P2_1
      00000080H.3 SFRSYM    DATA     BIT       P0_3
      000000F8H   SFRSYM    DATA     BYTE      RSTFR
      000000A0H.2 SFRSYM    DATA     BIT       P2_2
      00000080H.4 SFRSYM    DATA     BIT       P0_4
      000000A0H.3 SFRSYM    DATA     BIT       P2_3
      00000080H.5 SFRSYM    DATA     BIT       P0_5
      000000A0H.4 SFRSYM    DATA     BIT       P2_4
      00000080H.6 SFRSYM    DATA     BIT       P0_6
      000000A0H.5 SFRSYM    DATA     BIT       P2_5
      00000080H.7 SFRSYM    DATA     BIT       P0_7
      000000A0H.6 SFRSYM    DATA     BIT       P2_6
      000000A0H.7 SFRSYM    DATA     BIT       P2_7
      00000098H   SFRSYM    DATA     BIT       RI
      000000B8H.3 SFRSYM    DATA     BIT       EIIC
      000000B6H   SFRSYM    DATA     WORD      ADCR
      000000B8H.7 SFRSYM    DATA     BIT       EX8_15
      000000D0H.7 SFRSYM    DATA     BIT       CY
      00000098H.1 SFRSYM    DATA     BIT       TI
      000000FAH   SFRSYM    DATA     BYTE      IAP_ADDRH
      000000BFH   SFRSYM    DATA     BYTE      CRCH
      00000098H.6 SFRSYM    DATA     BIT       RXROV
      00000081H   SFRSYM    DATA     BYTE      SP
LX51 LINKER/LOCATER V4.66.41.0                                                        06/16/2023  10:23:34  PAGE 30


      000000F9H   SFRSYM    DATA     BYTE      IAP_ADDRL
      000000D0H.2 SFRSYM    DATA     BIT       OV
      000000BEH   SFRSYM    DATA     BYTE      CRCL
      000000C5H   SFRSYM    DATA     BYTE      RCAP5H
      000000C4H   SFRSYM    DATA     BYTE      RCAP5L
      000000F8H.5 SFRSYM    DATA     BIT       BORF
      000000BBH   SFRSYM    DATA     BYTE      LVDC
      000000BEH   SFRSYM    DATA     WORD      CRCR
      000000AFH   SFRSYM    DATA     BYTE      IICADR
      000000AEH   SFRSYM    DATA     BYTE      IICDAT
      00000099H   SFRSYM    DATA     BYTE      SBUF
      00000087H   SFRSYM    DATA     BYTE      PCON
      000000B8H   SFRSYM    DATA     BIT       ESPI
      000000E5H   SFRSYM    DATA     BYTE      PWM0DH
      000000EDH   SFRSYM    DATA     BYTE      PWM1DH
      00000096H   SFRSYM    DATA     BYTE      PINTF0
      000000BDH   SFRSYM    DATA     BYTE      WDTC
      000000F8H   SFRSYM    DATA     BIT       PLVRSTF
      000000F5H   SFRSYM    DATA     BYTE      PWM2DH
      00000098H   SFRSYM    DATA     BYTE      SCON
      00000097H   SFRSYM    DATA     BYTE      PINTF1
      000000A8H.5 SFRSYM    DATA     BIT       EWDT
      000000D1H   SFRSYM    DATA     BYTE      LCDCON
      00000089H   SFRSYM    DATA     BYTE      TMOD
      00000088H   SFRSYM    DATA     BYTE      TCON
      000000E4H   SFRSYM    DATA     BYTE      PWM0DL
      000000ECH   SFRSYM    DATA     BYTE      PWM1DL
      000000A6H   SFRSYM    DATA     BYTE      IICCON
      000000F8H.7 SFRSYM    DATA     BIT       PORF
      000000F4H   SFRSYM    DATA     BYTE      PWM2DL
      000000E1H   SFRSYM    DATA     BYTE      PWM0EN
      000000E9H   SFRSYM    DATA     BYTE      PWM1EN
      000000F1H   SFRSYM    DATA     BYTE      PWM2EN
      00000082H   SFRSYM    DATA     WORD      DPTR
      000000B4H   SFRSYM    DATA     BYTE      ADCC0
      0000008FH   SFRSYM    DATA     BYTE      CLKCON
      000000B5H   SFRSYM    DATA     BYTE      ADCC1
      000000E6H   SFRSYM    DATA     WORD      PWM0DT
      000000E3H   SFRSYM    DATA     BYTE      PWM0PH
      000000EEH   SFRSYM    DATA     WORD      PWM1DT
      000000EBH   SFRSYM    DATA     BYTE      PWM1PH
      000000A7H   SFRSYM    DATA     BYTE      IICSTA
      000000B8H   SFRSYM    DATA     BYTE      IE1
      000000F6H   SFRSYM    DATA     WORD      PWM2DT
      000000F3H   SFRSYM    DATA     BYTE      PWM2PH
      000000F0H   SFRSYM    DATA     BYTE      B
      000000E2H   SFRSYM    DATA     BYTE      PWM0PL
      000000F8H.3 SFRSYM    DATA     BIT       SWRF
      000000EAH   SFRSYM    DATA     BYTE      PWM1PL
      000000F2H   SFRSYM    DATA     BYTE      PWM2PL
      000000E0H   SFRSYM    DATA     BYTE      ACC
      000000BCH   SFRSYM    DATA     BYTE      LVDCMP
      000000A8H.1 SFRSYM    DATA     BIT       ET0
      000000A8H.4 SFRSYM    DATA     BIT       ES1
      000000A9H   SFRSYM    DATA     BYTE      IP0
      00000088H.5 SFRSYM    DATA     BIT       TF0
      000000A8H.3 SFRSYM    DATA     BIT       ET1
      000000A8H.6 SFRSYM    DATA     BIT       ES2
      000000AAH   SFRSYM    DATA     BYTE      IP1
      00000088H.7 SFRSYM    DATA     BIT       TF1
      000000B9H   SFRSYM    DATA     BYTE      IP2
      00000098H.2 SFRSYM    DATA     BIT       RB8
      000000B8H.1 SFRSYM    DATA     BIT       ET3
      0000008CH   SFRSYM    DATA     BYTE      TH0
      000000BAH   SFRSYM    DATA     BYTE      IP3
LX51 LINKER/LOCATER V4.66.41.0                                                        06/16/2023  10:23:34  PAGE 31


      000000A2H   SFRSYM    DATA     BYTE      INSCON
      000000B8H.2 SFRSYM    DATA     BIT       ET4
      000000A8H   SFRSYM    DATA     BIT       EX0
      0000008DH   SFRSYM    DATA     BYTE      TH1
      000000B1H   SFRSYM    DATA     BYTE      IP4
      00000098H.3 SFRSYM    DATA     BIT       TB8
      000000B8H.4 SFRSYM    DATA     BIT       ET5
      000000A8H.2 SFRSYM    DATA     BIT       EX1
      000000D0H   SFRSYM    DATA     BIT       P
      000000CBH   SFRSYM    DATA     BYTE      TH3
      000000CEH   SFRSYM    DATA     BYTE      TH4
      0000008AH   SFRSYM    DATA     BYTE      TL0
      000000C3H   SFRSYM    DATA     BYTE      TH5
      0000008BH   SFRSYM    DATA     BYTE      TL1
      000000CAH   SFRSYM    DATA     BYTE      TL3
      000000CDH   SFRSYM    DATA     BYTE      TL4
      000000D0H.3 SFRSYM    DATA     BIT       RS0
      000000C2H   SFRSYM    DATA     BYTE      TL5
      00000088H.4 SFRSYM    DATA     BIT       TR0
      000000D0H.4 SFRSYM    DATA     BIT       RS1
      000000FBH   SFRSYM    DATA     BYTE      IAP_DATA
      00000088H.6 SFRSYM    DATA     BIT       TR1
      000000F9H   SFRSYM    DATA     WORD      IAP_ADDR
      000000FDH   SFRSYM    DATA     BYTE      IAP_CMDH
      0000008EH   SFRSYM    DATA     BYTE      CLKSWR
      000000C4H   SFRSYM    DATA     WORD      RCAP5
      000000FCH   SFRSYM    DATA     BYTE      IAP_CMDL
      00000083H   SFRSYM    DATA     BYTE      DPH
      000000F8H.6 SFRSYM    DATA     BIT       EXRSTF
      00000082H   SFRSYM    DATA     BYTE      DPL
      000000ADH   SFRSYM    DATA     BYTE      SPSTAT
      000000B7H   SFRSYM    DATA     BYTE      ADCRH
      00000098H.4 SFRSYM    DATA     BIT       REN
      000000B8H.6 SFRSYM    DATA     BIT       EX2_7
      0000009EH   SFRSYM    DATA     BYTE      SCON2
      000000B6H   SFRSYM    DATA     BYTE      ADCRL
      000000DAH   SFRSYM    DATA     BYTE      PWM0C
      000000C9H   SFRSYM    DATA     BYTE      T3CON
      000000E4H   SFRSYM    DATA     WORD      PWM0D
      000000DBH   SFRSYM    DATA     BYTE      PWM1C
      000000CCH   SFRSYM    DATA     BYTE      T4CON
      000000ECH   SFRSYM    DATA     WORD      PWM1D
      000000DCH   SFRSYM    DATA     BYTE      PWM2C
      000000C1H   SFRSYM    DATA     BYTE      T5CON
      000000F4H   SFRSYM    DATA     WORD      PWM2D
      000000DDH   SFRSYM    DATA     BYTE      PWM3C
      000000DFH   SFRSYM    DATA     BYTE      PWM3D
      0000009BH   SFRSYM    DATA     BYTE      SADEN
      0000009AH   SFRSYM    DATA     BYTE      SADDR
      00000093H   SFRSYM    DATA     BYTE      TICKH
      000000D0H.5 SFRSYM    DATA     BIT       F0
      000000E2H   SFRSYM    DATA     WORD      PWM0P
      000000D0H.1 SFRSYM    DATA     BIT       F1
      000000EAH   SFRSYM    DATA     WORD      PWM1P
      000000F2H   SFRSYM    DATA     WORD      PWM2P
      000000DEH   SFRSYM    DATA     BYTE      PWM3P
      00000092H   SFRSYM    DATA     BYTE      TICKL
      000000D0H   SFRSYM    DATA     BYTE      PSW
      000000ABH   SFRSYM    DATA     BYTE      SPDAT

      01000789H   BLOCK     CODE     ---       LVL=0
      01000789H   BLOCK     CODE     NEAR LAB  LVL=1
      020000A0H   SYMBOL    XDATA    BYTE      u8_key_bounce
      020000A1H   SYMBOL    XDATA    BYTE      u8_key_new
      020000A2H   SYMBOL    XDATA    BYTE      u8_key_old
LX51 LINKER/LOCATER V4.66.41.0                                                        06/16/2023  10:23:34  PAGE 32


      020000A3H   SYMBOL    XDATA    BYTE      u8_key_value
      020000A4H   SYMBOL    XDATA    BYTE      u8_key_tmp
      020000A5H   SYMBOL    XDATA    WORD      u16_key_cnt
      ---         BLOCKEND  ---      ---       LVL=1
      01000789H   LINE      CODE     ---       #19
      01000789H   LINE      CODE     ---       #20
      01000789H   LINE      CODE     ---       #29
      01000791H   LINE      CODE     ---       #30
      01000796H   LINE      CODE     ---       #32
      0100079EH   LINE      CODE     ---       #33
      0100079EH   LINE      CODE     ---       #34
      010007A4H   LINE      CODE     ---       #35
      010007A4H   LINE      CODE     ---       #36
      010007ABH   LINE      CODE     ---       #37
      010007ABH   LINE      CODE     ---       #38
      010007B1H   LINE      CODE     ---       #39
      010007B3H   LINE      CODE     ---       #40
      010007B3H   LINE      CODE     ---       #41
      010007C1H   LINE      CODE     ---       #42
      010007D0H   LINE      CODE     ---       #43
      010007D0H   LINE      CODE     ---       #44
      010007D6H   LINE      CODE     ---       #45
      010007D6H   LINE      CODE     ---       #46
      010007D8H   LINE      CODE     ---       #48
      010007D8H   LINE      CODE     ---       #49
      010007DEH   LINE      CODE     ---       #50
      010007DEH   LINE      CODE     ---       #51
      010007E0H   LINE      CODE     ---       #53
      010007E0H   LINE      CODE     ---       #54
      010007E8H   LINE      CODE     ---       #55
      010007EEH   LINE      CODE     ---       #56
      010007F5H   LINE      CODE     ---       #57
      010007F5H   LINE      CODE     ---       #59
      010007FBH   LINE      CODE     ---       #60
      010007FBH   LINE      CODE     ---       #61
      01000803H   LINE      CODE     ---       #62
      01000803H   LINE      CODE     ---       #63
      01000805H   LINE      CODE     ---       #64
      01000807H   LINE      CODE     ---       #65
      0100080BH   LINE      CODE     ---       #66
      0100080BH   LINE      CODE     ---       #67
      0100080DH   LINE      CODE     ---       #68
      0100080DH   LINE      CODE     ---       #69
      0100080DH   LINE      CODE     ---       #70
      0100080FH   LINE      CODE     ---       #72
      0100080FH   LINE      CODE     ---       #73
      01000815H   LINE      CODE     ---       #75
      0100081DH   LINE      CODE     ---       #76
      0100081DH   LINE      CODE     ---       #77
      0100082CH   LINE      CODE     ---       #78
      0100082CH   LINE      CODE     ---       #79
      0100082EH   LINE      CODE     ---       #80
      0100082EH   LINE      CODE     ---       #81
      0100082EH   LINE      CODE     ---       #82
      01000830H   LINE      CODE     ---       #83
      01000834H   LINE      CODE     ---       #84
      01000834H   LINE      CODE     ---       #85
      01000843H   LINE      CODE     ---       #86
      01000843H   LINE      CODE     ---       #87
      01000845H   LINE      CODE     ---       #88
      0100084AH   LINE      CODE     ---       #89
      0100084AH   LINE      CODE     ---       #90
      0100084BH   LINE      CODE     ---       #92
      0100084BH   LINE      CODE     ---       #93
      01000850H   LINE      CODE     ---       #94
LX51 LINKER/LOCATER V4.66.41.0                                                        06/16/2023  10:23:34  PAGE 33


      01000856H   LINE      CODE     ---       #95
      01000856H   LINE      CODE     ---       #96
      01000856H   LINE      CODE     ---       #97
      ---         BLOCKEND  ---      ---       LVL=0

      ---         MODULE    ---      ---       PORT_MCU
      020000B3H   PUBLIC    XDATA    ---       u8_debug_rx_data
      020000B2H   PUBLIC    XDATA    BYTE      u8_debug_rx_index
      00000022H.0 PUBLIC    BIT      BIT       b_debug_rx_end
      01001206H   PUBLIC    CODE     ---       hardware_init
      01000D29H   PUBLIC    CODE     ---       system_power_down
      0100002EH   PUBLIC    CODE     ---       _delay_us
      01000C53H   PUBLIC    CODE     ---       debug_rpt
      0100110AH   PUBLIC    CODE     ---       _user_printf
      01000FF3H   PUBLIC    CODE     ---       debug_init
      010011F2H   PUBLIC    CODE     ---       _debug_putchar
      010011DAH   PUBLIC    CODE     ---       _putchar
      00000080H   SFRSYM    DATA     BYTE      P0
      00000090H   SFRSYM    DATA     BYTE      P1
      000000A0H   SFRSYM    DATA     BYTE      P2
      000000D0H.6 SFRSYM    DATA     BIT       AC
      000000A8H.7 SFRSYM    DATA     BIT       EA
      000000E7H   SFRSYM    DATA     BYTE      PWM0DTH
      000000CAH   SFRSYM    DATA     WORD      T3
      000000EFH   SFRSYM    DATA     BYTE      PWM1DTH
      000000ACH   SFRSYM    DATA     BYTE      SPCTL
      000000CDH   SFRSYM    DATA     WORD      T4
      000000F8H.4 SFRSYM    DATA     BIT       WDTRF
      000000F7H   SFRSYM    DATA     BYTE      PWM2DTH
      000000C2H   SFRSYM    DATA     WORD      T5
      00000098H.7 SFRSYM    DATA     BIT       FE
      000000E6H   SFRSYM    DATA     BYTE      PWM0DTL
      00000098H.5 SFRSYM    DATA     BIT       TXCOL
      000000EEH   SFRSYM    DATA     BYTE      PWM1DTL
      000000F6H   SFRSYM    DATA     BYTE      PWM2DTL
      000000B8H.5 SFRSYM    DATA     BIT       EADC
      00000091H   SFRSYM    DATA     BYTE      TICKCON
      000000A8H   SFRSYM    DATA     BYTE      IE
      00000080H   SFRSYM    DATA     BIT       P0_0
      000000F8H.1 SFRSYM    DATA     BIT       SPOVF
      000000FCH   SFRSYM    DATA     WORD      IAP_CMD
      00000090H   SFRSYM    DATA     BIT       P1_0
      00000080H.1 SFRSYM    DATA     BIT       P0_1
      000000A0H   SFRSYM    DATA     BIT       P2_0
      00000090H.1 SFRSYM    DATA     BIT       P1_1
      00000080H.2 SFRSYM    DATA     BIT       P0_2
      000000A0H.1 SFRSYM    DATA     BIT       P2_1
      00000080H.3 SFRSYM    DATA     BIT       P0_3
      000000F8H   SFRSYM    DATA     BYTE      RSTFR
      000000A0H.2 SFRSYM    DATA     BIT       P2_2
      00000080H.4 SFRSYM    DATA     BIT       P0_4
      000000A0H.3 SFRSYM    DATA     BIT       P2_3
      00000080H.5 SFRSYM    DATA     BIT       P0_5
      000000A0H.4 SFRSYM    DATA     BIT       P2_4
      00000080H.6 SFRSYM    DATA     BIT       P0_6
      000000A0H.5 SFRSYM    DATA     BIT       P2_5
      00000080H.7 SFRSYM    DATA     BIT       P0_7
      000000A0H.6 SFRSYM    DATA     BIT       P2_6
      000000A0H.7 SFRSYM    DATA     BIT       P2_7
      00000098H   SFRSYM    DATA     BIT       RI
      000000B8H.3 SFRSYM    DATA     BIT       EIIC
      000000B6H   SFRSYM    DATA     WORD      ADCR
      000000B8H.7 SFRSYM    DATA     BIT       EX8_15
      000000D0H.7 SFRSYM    DATA     BIT       CY
      00000098H.1 SFRSYM    DATA     BIT       TI
LX51 LINKER/LOCATER V4.66.41.0                                                        06/16/2023  10:23:34  PAGE 34


      000000FAH   SFRSYM    DATA     BYTE      IAP_ADDRH
      000000BFH   SFRSYM    DATA     BYTE      CRCH
      00000098H.6 SFRSYM    DATA     BIT       RXROV
      00000081H   SFRSYM    DATA     BYTE      SP
      000000F9H   SFRSYM    DATA     BYTE      IAP_ADDRL
      000000D0H.2 SFRSYM    DATA     BIT       OV
      000000BEH   SFRSYM    DATA     BYTE      CRCL
      000000C5H   SFRSYM    DATA     BYTE      RCAP5H
      000000C4H   SFRSYM    DATA     BYTE      RCAP5L
      000000F8H.5 SFRSYM    DATA     BIT       BORF
      000000BBH   SFRSYM    DATA     BYTE      LVDC
      000000BEH   SFRSYM    DATA     WORD      CRCR
      000000AFH   SFRSYM    DATA     BYTE      IICADR
      000000AEH   SFRSYM    DATA     BYTE      IICDAT
      00000099H   SFRSYM    DATA     BYTE      SBUF
      00000087H   SFRSYM    DATA     BYTE      PCON
      000000B8H   SFRSYM    DATA     BIT       ESPI
      000000E5H   SFRSYM    DATA     BYTE      PWM0DH
      000000EDH   SFRSYM    DATA     BYTE      PWM1DH
      00000096H   SFRSYM    DATA     BYTE      PINTF0
      000000BDH   SFRSYM    DATA     BYTE      WDTC
      000000F8H   SFRSYM    DATA     BIT       PLVRSTF
      000000F5H   SFRSYM    DATA     BYTE      PWM2DH
      00000098H   SFRSYM    DATA     BYTE      SCON
      00000097H   SFRSYM    DATA     BYTE      PINTF1
      000000A8H.5 SFRSYM    DATA     BIT       EWDT
      000000D1H   SFRSYM    DATA     BYTE      LCDCON
      00000089H   SFRSYM    DATA     BYTE      TMOD
      00000088H   SFRSYM    DATA     BYTE      TCON
      000000E4H   SFRSYM    DATA     BYTE      PWM0DL
      000000ECH   SFRSYM    DATA     BYTE      PWM1DL
      000000A6H   SFRSYM    DATA     BYTE      IICCON
      000000F8H.7 SFRSYM    DATA     BIT       PORF
      000000F4H   SFRSYM    DATA     BYTE      PWM2DL
      000000E1H   SFRSYM    DATA     BYTE      PWM0EN
      000000E9H   SFRSYM    DATA     BYTE      PWM1EN
      000000F1H   SFRSYM    DATA     BYTE      PWM2EN
      00000082H   SFRSYM    DATA     WORD      DPTR
      000000B4H   SFRSYM    DATA     BYTE      ADCC0
      0000008FH   SFRSYM    DATA     BYTE      CLKCON
      000000B5H   SFRSYM    DATA     BYTE      ADCC1
      000000E6H   SFRSYM    DATA     WORD      PWM0DT
      000000E3H   SFRSYM    DATA     BYTE      PWM0PH
      000000EEH   SFRSYM    DATA     WORD      PWM1DT
      000000EBH   SFRSYM    DATA     BYTE      PWM1PH
      000000A7H   SFRSYM    DATA     BYTE      IICSTA
      000000B8H   SFRSYM    DATA     BYTE      IE1
      000000F6H   SFRSYM    DATA     WORD      PWM2DT
      000000F3H   SFRSYM    DATA     BYTE      PWM2PH
      000000F0H   SFRSYM    DATA     BYTE      B
      000000E2H   SFRSYM    DATA     BYTE      PWM0PL
      000000F8H.3 SFRSYM    DATA     BIT       SWRF
      000000EAH   SFRSYM    DATA     BYTE      PWM1PL
      000000F2H   SFRSYM    DATA     BYTE      PWM2PL
      000000E0H   SFRSYM    DATA     BYTE      ACC
      000000BCH   SFRSYM    DATA     BYTE      LVDCMP
      000000A8H.1 SFRSYM    DATA     BIT       ET0
      000000A8H.4 SFRSYM    DATA     BIT       ES1
      000000A9H   SFRSYM    DATA     BYTE      IP0
      00000088H.5 SFRSYM    DATA     BIT       TF0
      000000A8H.3 SFRSYM    DATA     BIT       ET1
      000000A8H.6 SFRSYM    DATA     BIT       ES2
      000000AAH   SFRSYM    DATA     BYTE      IP1
      00000088H.7 SFRSYM    DATA     BIT       TF1
      000000B9H   SFRSYM    DATA     BYTE      IP2
LX51 LINKER/LOCATER V4.66.41.0                                                        06/16/2023  10:23:34  PAGE 35


      00000098H.2 SFRSYM    DATA     BIT       RB8
      000000B8H.1 SFRSYM    DATA     BIT       ET3
      0000008CH   SFRSYM    DATA     BYTE      TH0
      000000BAH   SFRSYM    DATA     BYTE      IP3
      000000A2H   SFRSYM    DATA     BYTE      INSCON
      000000B8H.2 SFRSYM    DATA     BIT       ET4
      000000A8H   SFRSYM    DATA     BIT       EX0
      0000008DH   SFRSYM    DATA     BYTE      TH1
      000000B1H   SFRSYM    DATA     BYTE      IP4
      00000098H.3 SFRSYM    DATA     BIT       TB8
      000000B8H.4 SFRSYM    DATA     BIT       ET5
      000000A8H.2 SFRSYM    DATA     BIT       EX1
      000000D0H   SFRSYM    DATA     BIT       P
      000000CBH   SFRSYM    DATA     BYTE      TH3
      000000CEH   SFRSYM    DATA     BYTE      TH4
      0000008AH   SFRSYM    DATA     BYTE      TL0
      000000C3H   SFRSYM    DATA     BYTE      TH5
      0000008BH   SFRSYM    DATA     BYTE      TL1
      000000CAH   SFRSYM    DATA     BYTE      TL3
      000000CDH   SFRSYM    DATA     BYTE      TL4
      000000D0H.3 SFRSYM    DATA     BIT       RS0
      000000C2H   SFRSYM    DATA     BYTE      TL5
      00000088H.4 SFRSYM    DATA     BIT       TR0
      000000D0H.4 SFRSYM    DATA     BIT       RS1
      000000FBH   SFRSYM    DATA     BYTE      IAP_DATA
      00000088H.6 SFRSYM    DATA     BIT       TR1
      000000F9H   SFRSYM    DATA     WORD      IAP_ADDR
      000000FDH   SFRSYM    DATA     BYTE      IAP_CMDH
      0000008EH   SFRSYM    DATA     BYTE      CLKSWR
      000000C4H   SFRSYM    DATA     WORD      RCAP5
      000000FCH   SFRSYM    DATA     BYTE      IAP_CMDL
      00000083H   SFRSYM    DATA     BYTE      DPH
      000000F8H.6 SFRSYM    DATA     BIT       EXRSTF
      00000082H   SFRSYM    DATA     BYTE      DPL
      000000ADH   SFRSYM    DATA     BYTE      SPSTAT
      000000B7H   SFRSYM    DATA     BYTE      ADCRH
      00000098H.4 SFRSYM    DATA     BIT       REN
      000000B8H.6 SFRSYM    DATA     BIT       EX2_7
      0000009EH   SFRSYM    DATA     BYTE      SCON2
      000000B6H   SFRSYM    DATA     BYTE      ADCRL
      000000DAH   SFRSYM    DATA     BYTE      PWM0C
      000000C9H   SFRSYM    DATA     BYTE      T3CON
      000000E4H   SFRSYM    DATA     WORD      PWM0D
      000000DBH   SFRSYM    DATA     BYTE      PWM1C
      000000CCH   SFRSYM    DATA     BYTE      T4CON
      000000ECH   SFRSYM    DATA     WORD      PWM1D
      000000DCH   SFRSYM    DATA     BYTE      PWM2C
      000000C1H   SFRSYM    DATA     BYTE      T5CON
      000000F4H   SFRSYM    DATA     WORD      PWM2D
      000000DDH   SFRSYM    DATA     BYTE      PWM3C
      000000DFH   SFRSYM    DATA     BYTE      PWM3D
      0000009BH   SFRSYM    DATA     BYTE      SADEN
      0000009AH   SFRSYM    DATA     BYTE      SADDR
      00000093H   SFRSYM    DATA     BYTE      TICKH
      000000D0H.5 SFRSYM    DATA     BIT       F0
      000000E2H   SFRSYM    DATA     WORD      PWM0P
      000000D0H.1 SFRSYM    DATA     BIT       F1
      000000EAH   SFRSYM    DATA     WORD      PWM1P
      000000F2H   SFRSYM    DATA     WORD      PWM2P
      000000DEH   SFRSYM    DATA     BYTE      PWM3P
      00000092H   SFRSYM    DATA     BYTE      TICKL
      000000D0H   SFRSYM    DATA     BYTE      PSW
      000000ABH   SFRSYM    DATA     BYTE      SPDAT

      010011DAH   BLOCK     CODE     ---       LVL=0
LX51 LINKER/LOCATER V4.66.41.0                                                        06/16/2023  10:23:34  PAGE 36


      00000005H   SYMBOL    DATA     CHAR      c
      010011DAH   LINE      CODE     ---       #31
      010011DCH   LINE      CODE     ---       #32
      010011DCH   LINE      CODE     ---       #33
      010011E1H   LINE      CODE     ---       #34
      010011E8H   LINE      CODE     ---       #35
      010011EFH   LINE      CODE     ---       #37
      010011F1H   LINE      CODE     ---       #38
      ---         BLOCKEND  ---      ---       LVL=0

      010011F2H   BLOCK     CODE     ---       LVL=0
      00000007H   SYMBOL    DATA     BYTE      u8_data
      010011F2H   LINE      CODE     ---       #40
      010011F2H   LINE      CODE     ---       #41
      010011F2H   LINE      CODE     ---       #42
      010011F7H   LINE      CODE     ---       #43
      010011FEH   LINE      CODE     ---       #44
      01001205H   LINE      CODE     ---       #45
      ---         BLOCKEND  ---      ---       LVL=0

      01000FF3H   BLOCK     CODE     ---       LVL=0
      01000FF3H   LINE      CODE     ---       #47
      01000FF3H   LINE      CODE     ---       #48
      01000FF3H   LINE      CODE     ---       #49
      01000FFCH   LINE      CODE     ---       #50
      01000FFEH   LINE      CODE     ---       #51
      01001004H   LINE      CODE     ---       #54
      0100100DH   LINE      CODE     ---       #55
      01001013H   LINE      CODE     ---       #58
      01001016H   LINE      CODE     ---       #59
      01001019H   LINE      CODE     ---       #61
      0100101CH   LINE      CODE     ---       #62
      01001021H   LINE      CODE     ---       #65
      01001026H   LINE      CODE     ---       #67
      0100102DH   LINE      CODE     ---       #68
      01001030H   LINE      CODE     ---       #70
      ---         BLOCKEND  ---      ---       LVL=0

      0100110AH   BLOCK     CODE     ---       LVL=0
      02000000H   SYMBOL    XDATA    ---       p_data
      0100110AH   LINE      CODE     ---       #72
      01001115H   LINE      CODE     ---       #73
      01001115H   LINE      CODE     ---       #74
      01001125H   LINE      CODE     ---       #75
      01001125H   LINE      CODE     ---       #76
      0100113AH   LINE      CODE     ---       #77
      0100113CH   LINE      CODE     ---       #78
      ---         BLOCKEND  ---      ---       LVL=0

      01000C53H   BLOCK     CODE     ---       LVL=0
      01000C62H   BLOCK     CODE     NEAR LAB  LVL=1
      00000007H   SYMBOL    DATA     BYTE      buf
      ---         BLOCKEND  ---      ---       LVL=1
      01000C53H   LINE      CODE     ---       #87
      01000C62H   LINE      CODE     ---       #91
      01000C69H   LINE      CODE     ---       #92
      01000C69H   LINE      CODE     ---       #93
      01000C6DH   LINE      CODE     ---       #94
      01000C72H   LINE      CODE     ---       #96
      01000C75H   LINE      CODE     ---       #97
      01000C75H   LINE      CODE     ---       #98
      01000C7FH   LINE      CODE     ---       #99
      01000C7FH   LINE      CODE     ---       #100
      01000C81H   LINE      CODE     ---       #101
      01000C83H   LINE      CODE     ---       #102
LX51 LINKER/LOCATER V4.66.41.0                                                        06/16/2023  10:23:34  PAGE 37


      01000C8AH   LINE      CODE     ---       #103
      01000C8AH   LINE      CODE     ---       #104
      01000C90H   LINE      CODE     ---       #105
      01000C92H   LINE      CODE     ---       #107
      01000C92H   LINE      CODE     ---       #108
      01000C98H   LINE      CODE     ---       #109
      01000CA5H   LINE      CODE     ---       #110
      01000CABH   LINE      CODE     ---       #111
      01000CABH   LINE      CODE     ---       #112
      01000CADH   LINE      CODE     ---       #113
      01000CB2H   LINE      CODE     ---       #114
      01000CB2H   LINE      CODE     ---       #115
      01000CB2H   LINE      CODE     ---       #116
      01000CB2H   LINE      CODE     ---       #117
      01000CB2H   LINE      CODE     ---       #118
      ---         BLOCKEND  ---      ---       LVL=0
      00000006H   SYMBOL    DATA     WORD      ms
      00000004H   SYMBOL    DATA     WORD      i

      0100002EH   BLOCK     CODE     ---       LVL=0
      00000007H   SYMBOL    DATA     BYTE      us
      0100002EH   LINE      CODE     ---       #158
      0100002EH   LINE      CODE     ---       #159
      0100002EH   LINE      CODE     ---       #160
      01000034H   LINE      CODE     ---       #161
      01000034H   LINE      CODE     ---       #162
      01000035H   LINE      CODE     ---       #163
      01000036H   LINE      CODE     ---       #164
      01000037H   LINE      CODE     ---       #165
      0100003AH   LINE      CODE     ---       #166
      ---         BLOCKEND  ---      ---       LVL=0
      00000007H   SYMBOL    DATA     BYTE      ms

      01000D29H   BLOCK     CODE     ---       LVL=0
      01000D29H   LINE      CODE     ---       #199
      01000D29H   LINE      CODE     ---       #200
      01000D29H   LINE      CODE     ---       #202
      01000D32H   LINE      CODE     ---       #203
      01000D38H   LINE      CODE     ---       #204
      01000D3FH   LINE      CODE     ---       #205
      01000D44H   LINE      CODE     ---       #206
      01000D47H   LINE      CODE     ---       #207
      01000D4AH   LINE      CODE     ---       #209
      01000D4DH   LINE      CODE     ---       #211
      01000D50H   LINE      CODE     ---       #213
      01000D56H   LINE      CODE     ---       #215
      01000D5DH   LINE      CODE     ---       #217
      01000D60H   LINE      CODE     ---       #219
      01000D62H   LINE      CODE     ---       #221
      01000D65H   LINE      CODE     ---       #222
      01000D69H   LINE      CODE     ---       #223
      01000D6CH   LINE      CODE     ---       #225
      01000D6FH   LINE      CODE     ---       #226
      01000D72H   LINE      CODE     ---       #228
      01000D79H   LINE      CODE     ---       #229
      01000D7CH   LINE      CODE     ---       #230
      01000D7FH   LINE      CODE     ---       #231
      01000D81H   LINE      CODE     ---       #232
      ---         BLOCKEND  ---      ---       LVL=0

      01001206H   BLOCK     CODE     ---       LVL=0
      01001206H   LINE      CODE     ---       #244
      01001206H   LINE      CODE     ---       #245
      01001206H   LINE      CODE     ---       #246
      01001209H   LINE      CODE     ---       #247
LX51 LINKER/LOCATER V4.66.41.0                                                        06/16/2023  10:23:34  PAGE 38


      0100120CH   LINE      CODE     ---       #251
      0100120FH   LINE      CODE     ---       #252
      01001212H   LINE      CODE     ---       #253
      01001217H   LINE      CODE     ---       #254
      ---         BLOCKEND  ---      ---       LVL=0

      ---         MODULE    ---      ---       HS6220_RF
      020000B7H   PUBLIC    XDATA    BYTE      rf_sleep_cnt
      020000B5H   PUBLIC    XDATA    WORD      rf_reset_cnt
      00000080H   SFRSYM    DATA     BYTE      P0
      00000090H   SFRSYM    DATA     BYTE      P1
      000000A0H   SFRSYM    DATA     BYTE      P2
      000000D0H.6 SFRSYM    DATA     BIT       AC
      000000A8H.7 SFRSYM    DATA     BIT       EA
      000000E7H   SFRSYM    DATA     BYTE      PWM0DTH
      000000CAH   SFRSYM    DATA     WORD      T3
      000000EFH   SFRSYM    DATA     BYTE      PWM1DTH
      000000ACH   SFRSYM    DATA     BYTE      SPCTL
      000000CDH   SFRSYM    DATA     WORD      T4
      000000F8H.4 SFRSYM    DATA     BIT       WDTRF
      000000F7H   SFRSYM    DATA     BYTE      PWM2DTH
      000000C2H   SFRSYM    DATA     WORD      T5
      00000098H.7 SFRSYM    DATA     BIT       FE
      000000E6H   SFRSYM    DATA     BYTE      PWM0DTL
      00000098H.5 SFRSYM    DATA     BIT       TXCOL
      000000EEH   SFRSYM    DATA     BYTE      PWM1DTL
      000000F6H   SFRSYM    DATA     BYTE      PWM2DTL
      000000B8H.5 SFRSYM    DATA     BIT       EADC
      00000091H   SFRSYM    DATA     BYTE      TICKCON
      000000A8H   SFRSYM    DATA     BYTE      IE
      00000080H   SFRSYM    DATA     BIT       P0_0
      000000F8H.1 SFRSYM    DATA     BIT       SPOVF
      000000FCH   SFRSYM    DATA     WORD      IAP_CMD
      00000090H   SFRSYM    DATA     BIT       P1_0
      00000080H.1 SFRSYM    DATA     BIT       P0_1
      000000A0H   SFRSYM    DATA     BIT       P2_0
      00000090H.1 SFRSYM    DATA     BIT       P1_1
      00000080H.2 SFRSYM    DATA     BIT       P0_2
      000000A0H.1 SFRSYM    DATA     BIT       P2_1
      00000080H.3 SFRSYM    DATA     BIT       P0_3
      000000F8H   SFRSYM    DATA     BYTE      RSTFR
      000000A0H.2 SFRSYM    DATA     BIT       P2_2
      00000080H.4 SFRSYM    DATA     BIT       P0_4
      000000A0H.3 SFRSYM    DATA     BIT       P2_3
      00000080H.5 SFRSYM    DATA     BIT       P0_5
      000000A0H.4 SFRSYM    DATA     BIT       P2_4
      00000080H.6 SFRSYM    DATA     BIT       P0_6
      000000A0H.5 SFRSYM    DATA     BIT       P2_5
      00000080H.7 SFRSYM    DATA     BIT       P0_7
      000000A0H.6 SFRSYM    DATA     BIT       P2_6
      000000A0H.7 SFRSYM    DATA     BIT       P2_7
      00000098H   SFRSYM    DATA     BIT       RI
      000000B8H.3 SFRSYM    DATA     BIT       EIIC
      000000B6H   SFRSYM    DATA     WORD      ADCR
      000000B8H.7 SFRSYM    DATA     BIT       EX8_15
      000000D0H.7 SFRSYM    DATA     BIT       CY
      00000098H.1 SFRSYM    DATA     BIT       TI
      000000FAH   SFRSYM    DATA     BYTE      IAP_ADDRH
      000000BFH   SFRSYM    DATA     BYTE      CRCH
      00000098H.6 SFRSYM    DATA     BIT       RXROV
      00000081H   SFRSYM    DATA     BYTE      SP
      000000F9H   SFRSYM    DATA     BYTE      IAP_ADDRL
      000000D0H.2 SFRSYM    DATA     BIT       OV
      000000BEH   SFRSYM    DATA     BYTE      CRCL
      000000C5H   SFRSYM    DATA     BYTE      RCAP5H
LX51 LINKER/LOCATER V4.66.41.0                                                        06/16/2023  10:23:34  PAGE 39


      000000C4H   SFRSYM    DATA     BYTE      RCAP5L
      000000F8H.5 SFRSYM    DATA     BIT       BORF
      000000BBH   SFRSYM    DATA     BYTE      LVDC
      000000BEH   SFRSYM    DATA     WORD      CRCR
      000000AFH   SFRSYM    DATA     BYTE      IICADR
      000000AEH   SFRSYM    DATA     BYTE      IICDAT
      00000099H   SFRSYM    DATA     BYTE      SBUF
      00000087H   SFRSYM    DATA     BYTE      PCON
      000000B8H   SFRSYM    DATA     BIT       ESPI
      000000E5H   SFRSYM    DATA     BYTE      PWM0DH
      000000EDH   SFRSYM    DATA     BYTE      PWM1DH
      00000096H   SFRSYM    DATA     BYTE      PINTF0
      000000BDH   SFRSYM    DATA     BYTE      WDTC
      000000F8H   SFRSYM    DATA     BIT       PLVRSTF
      000000F5H   SFRSYM    DATA     BYTE      PWM2DH
      00000098H   SFRSYM    DATA     BYTE      SCON
      00000097H   SFRSYM    DATA     BYTE      PINTF1
      000000A8H.5 SFRSYM    DATA     BIT       EWDT
      000000D1H   SFRSYM    DATA     BYTE      LCDCON
      00000089H   SFRSYM    DATA     BYTE      TMOD
      00000088H   SFRSYM    DATA     BYTE      TCON
      000000E4H   SFRSYM    DATA     BYTE      PWM0DL
      000000ECH   SFRSYM    DATA     BYTE      PWM1DL
      000000A6H   SFRSYM    DATA     BYTE      IICCON
      000000F8H.7 SFRSYM    DATA     BIT       PORF
      000000F4H   SFRSYM    DATA     BYTE      PWM2DL
      000000E1H   SFRSYM    DATA     BYTE      PWM0EN
      000000E9H   SFRSYM    DATA     BYTE      PWM1EN
      000000F1H   SFRSYM    DATA     BYTE      PWM2EN
      00000082H   SFRSYM    DATA     WORD      DPTR
      000000B4H   SFRSYM    DATA     BYTE      ADCC0
      0000008FH   SFRSYM    DATA     BYTE      CLKCON
      000000B5H   SFRSYM    DATA     BYTE      ADCC1
      000000E6H   SFRSYM    DATA     WORD      PWM0DT
      000000E3H   SFRSYM    DATA     BYTE      PWM0PH
      000000EEH   SFRSYM    DATA     WORD      PWM1DT
      000000EBH   SFRSYM    DATA     BYTE      PWM1PH
      000000A7H   SFRSYM    DATA     BYTE      IICSTA
      000000B8H   SFRSYM    DATA     BYTE      IE1
      000000F6H   SFRSYM    DATA     WORD      PWM2DT
      000000F3H   SFRSYM    DATA     BYTE      PWM2PH
      000000F0H   SFRSYM    DATA     BYTE      B
      000000E2H   SFRSYM    DATA     BYTE      PWM0PL
      000000F8H.3 SFRSYM    DATA     BIT       SWRF
      000000EAH   SFRSYM    DATA     BYTE      PWM1PL
      000000F2H   SFRSYM    DATA     BYTE      PWM2PL
      000000E0H   SFRSYM    DATA     BYTE      ACC
      000000BCH   SFRSYM    DATA     BYTE      LVDCMP
      000000A8H.1 SFRSYM    DATA     BIT       ET0
      000000A8H.4 SFRSYM    DATA     BIT       ES1
      000000A9H   SFRSYM    DATA     BYTE      IP0
      00000088H.5 SFRSYM    DATA     BIT       TF0
      000000A8H.3 SFRSYM    DATA     BIT       ET1
      000000A8H.6 SFRSYM    DATA     BIT       ES2
      000000AAH   SFRSYM    DATA     BYTE      IP1
      00000088H.7 SFRSYM    DATA     BIT       TF1
      000000B9H   SFRSYM    DATA     BYTE      IP2
      00000098H.2 SFRSYM    DATA     BIT       RB8
      000000B8H.1 SFRSYM    DATA     BIT       ET3
      0000008CH   SFRSYM    DATA     BYTE      TH0
      000000BAH   SFRSYM    DATA     BYTE      IP3
      000000A2H   SFRSYM    DATA     BYTE      INSCON
      000000B8H.2 SFRSYM    DATA     BIT       ET4
      000000A8H   SFRSYM    DATA     BIT       EX0
      0000008DH   SFRSYM    DATA     BYTE      TH1
LX51 LINKER/LOCATER V4.66.41.0                                                        06/16/2023  10:23:34  PAGE 40


      000000B1H   SFRSYM    DATA     BYTE      IP4
      00000098H.3 SFRSYM    DATA     BIT       TB8
      000000B8H.4 SFRSYM    DATA     BIT       ET5
      000000A8H.2 SFRSYM    DATA     BIT       EX1
      000000D0H   SFRSYM    DATA     BIT       P
      000000CBH   SFRSYM    DATA     BYTE      TH3
      000000CEH   SFRSYM    DATA     BYTE      TH4
      0000008AH   SFRSYM    DATA     BYTE      TL0
      000000C3H   SFRSYM    DATA     BYTE      TH5
      0000008BH   SFRSYM    DATA     BYTE      TL1
      000000CAH   SFRSYM    DATA     BYTE      TL3
      000000CDH   SFRSYM    DATA     BYTE      TL4
      000000D0H.3 SFRSYM    DATA     BIT       RS0
      000000C2H   SFRSYM    DATA     BYTE      TL5
      00000088H.4 SFRSYM    DATA     BIT       TR0
      000000D0H.4 SFRSYM    DATA     BIT       RS1
      000000FBH   SFRSYM    DATA     BYTE      IAP_DATA
      00000088H.6 SFRSYM    DATA     BIT       TR1
      000000F9H   SFRSYM    DATA     WORD      IAP_ADDR
      000000FDH   SFRSYM    DATA     BYTE      IAP_CMDH
      0000008EH   SFRSYM    DATA     BYTE      CLKSWR
      000000C4H   SFRSYM    DATA     WORD      RCAP5
      000000FCH   SFRSYM    DATA     BYTE      IAP_CMDL
      00000083H   SFRSYM    DATA     BYTE      DPH
      000000F8H.6 SFRSYM    DATA     BIT       EXRSTF
      00000082H   SFRSYM    DATA     BYTE      DPL
      000000ADH   SFRSYM    DATA     BYTE      SPSTAT
      000000B7H   SFRSYM    DATA     BYTE      ADCRH
      00000098H.4 SFRSYM    DATA     BIT       REN
      000000B8H.6 SFRSYM    DATA     BIT       EX2_7
      0000009EH   SFRSYM    DATA     BYTE      SCON2
      000000B6H   SFRSYM    DATA     BYTE      ADCRL
      000000DAH   SFRSYM    DATA     BYTE      PWM0C
      000000C9H   SFRSYM    DATA     BYTE      T3CON
      000000E4H   SFRSYM    DATA     WORD      PWM0D
      000000DBH   SFRSYM    DATA     BYTE      PWM1C
      000000CCH   SFRSYM    DATA     BYTE      T4CON
      000000ECH   SFRSYM    DATA     WORD      PWM1D
      000000DCH   SFRSYM    DATA     BYTE      PWM2C
      000000C1H   SFRSYM    DATA     BYTE      T5CON
      000000F4H   SFRSYM    DATA     WORD      PWM2D
      000000DDH   SFRSYM    DATA     BYTE      PWM3C
      000000DFH   SFRSYM    DATA     BYTE      PWM3D
      0000009BH   SFRSYM    DATA     BYTE      SADEN
      0000009AH   SFRSYM    DATA     BYTE      SADDR
      00000093H   SFRSYM    DATA     BYTE      TICKH
      000000D0H.5 SFRSYM    DATA     BIT       F0
      000000E2H   SFRSYM    DATA     WORD      PWM0P
      000000D0H.1 SFRSYM    DATA     BIT       F1
      000000EAH   SFRSYM    DATA     WORD      PWM1P
      000000F2H   SFRSYM    DATA     WORD      PWM2P
      000000DEH   SFRSYM    DATA     BYTE      PWM3P
      00000092H   SFRSYM    DATA     BYTE      TICKL
      000000D0H   SFRSYM    DATA     BYTE      PSW
      000000ABH   SFRSYM    DATA     BYTE      SPDAT
      00000005H   SYMBOL    DATA     BYTE      TxData
      00000007H   SYMBOL    DATA     BYTE      i
      00000006H   SYMBOL    DATA     BYTE      data_output_bit
      00000007H   SYMBOL    DATA     BYTE      bit_ctr
      00000004H   SYMBOL    DATA     BYTE      byte
      00000006H   SYMBOL    DATA     BYTE      temp
      00000007H   SYMBOL    DATA     BYTE      Data
      00000007H   SYMBOL    DATA     BYTE      addr
      00000004H   SYMBOL    DATA     BYTE      D
      00000007H   SYMBOL    DATA     BYTE      addr
LX51 LINKER/LOCATER V4.66.41.0                                                        06/16/2023  10:23:34  PAGE 41


      00000007H   SYMBOL    DATA     BYTE      addr
      00000007H   SYMBOL    DATA     BYTE      rxdata
      00000007H   SYMBOL    DATA     BYTE      addr
      00000007H   SYMBOL    DATA     BYTE      opt
      00000007H   SYMBOL    DATA     BYTE      cmd
      00000004H   SYMBOL    DATA     BYTE      D
      00000003H   SYMBOL    DATA     BYTE      bank
      00000007H   SYMBOL    DATA     BYTE      sta
      00000003H   SYMBOL    DATA     BYTE      rate
      00000007H   SYMBOL    DATA     BYTE      tmp
      00000007H   SYMBOL    DATA     BYTE      chn
      00000003H   SYMBOL    DATA     BYTE      pwr
      00000007H   SYMBOL    DATA     BYTE      tmp
      00000001H   SYMBOL    DATA     ---       buf
      00000005H   SYMBOL    DATA     BYTE      len
      00000001H   SYMBOL    DATA     ---       buf
      00000007H   SYMBOL    DATA     BYTE      sta
      00000007H   SYMBOL    DATA     BYTE      cmd
      00000001H   SYMBOL    DATA     ---       buf
      00000007H   SYMBOL    DATA     BYTE      sta
      00000003H   SYMBOL    DATA     BYTE      cnt
      00000003H   SYMBOL    DATA     BYTE      mod
      00000002H   SYMBOL    DATA     BYTE      tmp

      ---         MODULE    ---      ---       REGISTER
      020000B0H   PUBLIC    XDATA    ---       hs24m_trim
      020000AEH   PUBLIC    XDATA    ---       hs32m_trim
      0100000EH   PUBLIC    CODE     ---       wdt_rpt
      01000FB3H   PUBLIC    CODE     ---       reset_check
      01000006H   PUBLIC    CODE     ---       feed_watchdog
      0100125FH   PUBLIC    CODE     ---       enable_watchdog
      01001269H   PUBLIC    CODE     ---       disable_watchdog
      0100116CH   PUBLIC    CODE     ---       config_sysclk_ihrc_module
      00000080H   SFRSYM    DATA     BYTE      P0
      00000090H   SFRSYM    DATA     BYTE      P1
      000000A0H   SFRSYM    DATA     BYTE      P2
      000000D0H.6 SFRSYM    DATA     BIT       AC
      000000A8H.7 SFRSYM    DATA     BIT       EA
      000000E7H   SFRSYM    DATA     BYTE      PWM0DTH
      000000CAH   SFRSYM    DATA     WORD      T3
      000000EFH   SFRSYM    DATA     BYTE      PWM1DTH
      000000ACH   SFRSYM    DATA     BYTE      SPCTL
      000000CDH   SFRSYM    DATA     WORD      T4
      000000F8H.4 SFRSYM    DATA     BIT       WDTRF
      000000F7H   SFRSYM    DATA     BYTE      PWM2DTH
      000000C2H   SFRSYM    DATA     WORD      T5
      00000098H.7 SFRSYM    DATA     BIT       FE
      000000E6H   SFRSYM    DATA     BYTE      PWM0DTL
      00000098H.5 SFRSYM    DATA     BIT       TXCOL
      000000EEH   SFRSYM    DATA     BYTE      PWM1DTL
      000000F6H   SFRSYM    DATA     BYTE      PWM2DTL
      000000B8H.5 SFRSYM    DATA     BIT       EADC
      00000091H   SFRSYM    DATA     BYTE      TICKCON
      000000A8H   SFRSYM    DATA     BYTE      IE
      00000080H   SFRSYM    DATA     BIT       P0_0
      000000F8H.1 SFRSYM    DATA     BIT       SPOVF
      000000FCH   SFRSYM    DATA     WORD      IAP_CMD
      00000090H   SFRSYM    DATA     BIT       P1_0
      00000080H.1 SFRSYM    DATA     BIT       P0_1
      000000A0H   SFRSYM    DATA     BIT       P2_0
      00000090H.1 SFRSYM    DATA     BIT       P1_1
      00000080H.2 SFRSYM    DATA     BIT       P0_2
      000000A0H.1 SFRSYM    DATA     BIT       P2_1
      00000080H.3 SFRSYM    DATA     BIT       P0_3
      000000F8H   SFRSYM    DATA     BYTE      RSTFR
LX51 LINKER/LOCATER V4.66.41.0                                                        06/16/2023  10:23:34  PAGE 42


      000000A0H.2 SFRSYM    DATA     BIT       P2_2
      00000080H.4 SFRSYM    DATA     BIT       P0_4
      000000A0H.3 SFRSYM    DATA     BIT       P2_3
      00000080H.5 SFRSYM    DATA     BIT       P0_5
      000000A0H.4 SFRSYM    DATA     BIT       P2_4
      00000080H.6 SFRSYM    DATA     BIT       P0_6
      000000A0H.5 SFRSYM    DATA     BIT       P2_5
      00000080H.7 SFRSYM    DATA     BIT       P0_7
      000000A0H.6 SFRSYM    DATA     BIT       P2_6
      000000A0H.7 SFRSYM    DATA     BIT       P2_7
      00000098H   SFRSYM    DATA     BIT       RI
      000000B8H.3 SFRSYM    DATA     BIT       EIIC
      000000B6H   SFRSYM    DATA     WORD      ADCR
      000000B8H.7 SFRSYM    DATA     BIT       EX8_15
      000000D0H.7 SFRSYM    DATA     BIT       CY
      00000098H.1 SFRSYM    DATA     BIT       TI
      000000FAH   SFRSYM    DATA     BYTE      IAP_ADDRH
      000000BFH   SFRSYM    DATA     BYTE      CRCH
      00000098H.6 SFRSYM    DATA     BIT       RXROV
      00000081H   SFRSYM    DATA     BYTE      SP
      000000F9H   SFRSYM    DATA     BYTE      IAP_ADDRL
      000000D0H.2 SFRSYM    DATA     BIT       OV
      000000BEH   SFRSYM    DATA     BYTE      CRCL
      000000C5H   SFRSYM    DATA     BYTE      RCAP5H
      000000C4H   SFRSYM    DATA     BYTE      RCAP5L
      000000F8H.5 SFRSYM    DATA     BIT       BORF
      000000BBH   SFRSYM    DATA     BYTE      LVDC
      000000BEH   SFRSYM    DATA     WORD      CRCR
      000000AFH   SFRSYM    DATA     BYTE      IICADR
      000000AEH   SFRSYM    DATA     BYTE      IICDAT
      00000099H   SFRSYM    DATA     BYTE      SBUF
      00000087H   SFRSYM    DATA     BYTE      PCON
      000000B8H   SFRSYM    DATA     BIT       ESPI
      000000E5H   SFRSYM    DATA     BYTE      PWM0DH
      000000EDH   SFRSYM    DATA     BYTE      PWM1DH
      00000096H   SFRSYM    DATA     BYTE      PINTF0
      000000BDH   SFRSYM    DATA     BYTE      WDTC
      000000F8H   SFRSYM    DATA     BIT       PLVRSTF
      000000F5H   SFRSYM    DATA     BYTE      PWM2DH
      00000098H   SFRSYM    DATA     BYTE      SCON
      00000097H   SFRSYM    DATA     BYTE      PINTF1
      000000A8H.5 SFRSYM    DATA     BIT       EWDT
      000000D1H   SFRSYM    DATA     BYTE      LCDCON
      00000089H   SFRSYM    DATA     BYTE      TMOD
      00000088H   SFRSYM    DATA     BYTE      TCON
      000000E4H   SFRSYM    DATA     BYTE      PWM0DL
      000000ECH   SFRSYM    DATA     BYTE      PWM1DL
      000000A6H   SFRSYM    DATA     BYTE      IICCON
      000000F8H.7 SFRSYM    DATA     BIT       PORF
      000000F4H   SFRSYM    DATA     BYTE      PWM2DL
      000000E1H   SFRSYM    DATA     BYTE      PWM0EN
      000000E9H   SFRSYM    DATA     BYTE      PWM1EN
      000000F1H   SFRSYM    DATA     BYTE      PWM2EN
      00000082H   SFRSYM    DATA     WORD      DPTR
      000000B4H   SFRSYM    DATA     BYTE      ADCC0
      0000008FH   SFRSYM    DATA     BYTE      CLKCON
      000000B5H   SFRSYM    DATA     BYTE      ADCC1
      000000E6H   SFRSYM    DATA     WORD      PWM0DT
      000000E3H   SFRSYM    DATA     BYTE      PWM0PH
      000000EEH   SFRSYM    DATA     WORD      PWM1DT
      000000EBH   SFRSYM    DATA     BYTE      PWM1PH
      000000A7H   SFRSYM    DATA     BYTE      IICSTA
      000000B8H   SFRSYM    DATA     BYTE      IE1
      000000F6H   SFRSYM    DATA     WORD      PWM2DT
      000000F3H   SFRSYM    DATA     BYTE      PWM2PH
LX51 LINKER/LOCATER V4.66.41.0                                                        06/16/2023  10:23:34  PAGE 43


      000000F0H   SFRSYM    DATA     BYTE      B
      000000E2H   SFRSYM    DATA     BYTE      PWM0PL
      000000F8H.3 SFRSYM    DATA     BIT       SWRF
      000000EAH   SFRSYM    DATA     BYTE      PWM1PL
      000000F2H   SFRSYM    DATA     BYTE      PWM2PL
      000000E0H   SFRSYM    DATA     BYTE      ACC
      000000BCH   SFRSYM    DATA     BYTE      LVDCMP
      000000A8H.1 SFRSYM    DATA     BIT       ET0
      000000A8H.4 SFRSYM    DATA     BIT       ES1
      000000A9H   SFRSYM    DATA     BYTE      IP0
      00000088H.5 SFRSYM    DATA     BIT       TF0
      000000A8H.3 SFRSYM    DATA     BIT       ET1
      000000A8H.6 SFRSYM    DATA     BIT       ES2
      000000AAH   SFRSYM    DATA     BYTE      IP1
      00000088H.7 SFRSYM    DATA     BIT       TF1
      000000B9H   SFRSYM    DATA     BYTE      IP2
      00000098H.2 SFRSYM    DATA     BIT       RB8
      000000B8H.1 SFRSYM    DATA     BIT       ET3
      0000008CH   SFRSYM    DATA     BYTE      TH0
      000000BAH   SFRSYM    DATA     BYTE      IP3
      000000A2H   SFRSYM    DATA     BYTE      INSCON
      000000B8H.2 SFRSYM    DATA     BIT       ET4
      000000A8H   SFRSYM    DATA     BIT       EX0
      0000008DH   SFRSYM    DATA     BYTE      TH1
      000000B1H   SFRSYM    DATA     BYTE      IP4
      00000098H.3 SFRSYM    DATA     BIT       TB8
      000000B8H.4 SFRSYM    DATA     BIT       ET5
      000000A8H.2 SFRSYM    DATA     BIT       EX1
      000000D0H   SFRSYM    DATA     BIT       P
      000000CBH   SFRSYM    DATA     BYTE      TH3
      000000CEH   SFRSYM    DATA     BYTE      TH4
      0000008AH   SFRSYM    DATA     BYTE      TL0
      000000C3H   SFRSYM    DATA     BYTE      TH5
      0000008BH   SFRSYM    DATA     BYTE      TL1
      000000CAH   SFRSYM    DATA     BYTE      TL3
      000000CDH   SFRSYM    DATA     BYTE      TL4
      000000D0H.3 SFRSYM    DATA     BIT       RS0
      000000C2H   SFRSYM    DATA     BYTE      TL5
      00000088H.4 SFRSYM    DATA     BIT       TR0
      000000D0H.4 SFRSYM    DATA     BIT       RS1
      000000FBH   SFRSYM    DATA     BYTE      IAP_DATA
      00000088H.6 SFRSYM    DATA     BIT       TR1
      000000F9H   SFRSYM    DATA     WORD      IAP_ADDR
      000000FDH   SFRSYM    DATA     BYTE      IAP_CMDH
      0000008EH   SFRSYM    DATA     BYTE      CLKSWR
      000000C4H   SFRSYM    DATA     WORD      RCAP5
      000000FCH   SFRSYM    DATA     BYTE      IAP_CMDL
      00000083H   SFRSYM    DATA     BYTE      DPH
      000000F8H.6 SFRSYM    DATA     BIT       EXRSTF
      00000082H   SFRSYM    DATA     BYTE      DPL
      000000ADH   SFRSYM    DATA     BYTE      SPSTAT
      000000B7H   SFRSYM    DATA     BYTE      ADCRH
      00000098H.4 SFRSYM    DATA     BIT       REN
      000000B8H.6 SFRSYM    DATA     BIT       EX2_7
      0000009EH   SFRSYM    DATA     BYTE      SCON2
      000000B6H   SFRSYM    DATA     BYTE      ADCRL
      000000DAH   SFRSYM    DATA     BYTE      PWM0C
      000000C9H   SFRSYM    DATA     BYTE      T3CON
      000000E4H   SFRSYM    DATA     WORD      PWM0D
      000000DBH   SFRSYM    DATA     BYTE      PWM1C
      000000CCH   SFRSYM    DATA     BYTE      T4CON
      000000ECH   SFRSYM    DATA     WORD      PWM1D
      000000DCH   SFRSYM    DATA     BYTE      PWM2C
      000000C1H   SFRSYM    DATA     BYTE      T5CON
      000000F4H   SFRSYM    DATA     WORD      PWM2D
LX51 LINKER/LOCATER V4.66.41.0                                                        06/16/2023  10:23:34  PAGE 44


      000000DDH   SFRSYM    DATA     BYTE      PWM3C
      000000DFH   SFRSYM    DATA     BYTE      PWM3D
      0000009BH   SFRSYM    DATA     BYTE      SADEN
      0000009AH   SFRSYM    DATA     BYTE      SADDR
      00000093H   SFRSYM    DATA     BYTE      TICKH
      000000D0H.5 SFRSYM    DATA     BIT       F0
      000000E2H   SFRSYM    DATA     WORD      PWM0P
      000000D0H.1 SFRSYM    DATA     BIT       F1
      000000EAH   SFRSYM    DATA     WORD      PWM1P
      000000F2H   SFRSYM    DATA     WORD      PWM2P
      000000DEH   SFRSYM    DATA     BYTE      PWM3P
      00000092H   SFRSYM    DATA     BYTE      TICKL
      000000D0H   SFRSYM    DATA     BYTE      PSW
      000000ABH   SFRSYM    DATA     BYTE      SPDAT

      0100116CH   BLOCK     CODE     ---       LVL=0
      0100116CH   LINE      CODE     ---       #50
      0100116CH   LINE      CODE     ---       #51
      0100116CH   LINE      CODE     ---       #53
      01001171H   LINE      CODE     ---       #56
      01001173H   LINE      CODE     ---       #57
      01001179H   LINE      CODE     ---       #58
      0100117CH   LINE      CODE     ---       #59
      0100117FH   LINE      CODE     ---       #62
      01001184H   LINE      CODE     ---       #63
      01001187H   LINE      CODE     ---       #64
      0100118FH   LINE      CODE     ---       #65
      01001195H   LINE      CODE     ---       #66
      ---         BLOCKEND  ---      ---       LVL=0

      01001269H   BLOCK     CODE     ---       LVL=0
      01001269H   LINE      CODE     ---       #129
      01001269H   LINE      CODE     ---       #130
      01001269H   LINE      CODE     ---       #131
      0100126CH   LINE      CODE     ---       #132
      01001270H   LINE      CODE     ---       #133
      ---         BLOCKEND  ---      ---       LVL=0

      0100125FH   BLOCK     CODE     ---       LVL=0
      0100125FH   LINE      CODE     ---       #135
      0100125FH   LINE      CODE     ---       #136
      0100125FH   LINE      CODE     ---       #139
      01001262H   LINE      CODE     ---       #141
      01001268H   LINE      CODE     ---       #142
      ---         BLOCKEND  ---      ---       LVL=0

      01000006H   BLOCK     CODE     ---       LVL=0
      01000006H   LINE      CODE     ---       #156
      01000006H   LINE      CODE     ---       #157
      01000006H   LINE      CODE     ---       #159
      01000009H   LINE      CODE     ---       #160
      ---         BLOCKEND  ---      ---       LVL=0

      01000FB3H   BLOCK     CODE     ---       LVL=0
      01000FB3H   LINE      CODE     ---       #173
      01000FB3H   LINE      CODE     ---       #174
      01000FB3H   LINE      CODE     ---       #175
      01000FB8H   LINE      CODE     ---       #176
      01000FB8H   LINE      CODE     ---       #177
      01000FB9H   LINE      CODE     ---       #178
      01000FBCH   LINE      CODE     ---       #179
      01000FBCH   LINE      CODE     ---       #180
      01000FC1H   LINE      CODE     ---       #181
      01000FC1H   LINE      CODE     ---       #182
      01000FC2H   LINE      CODE     ---       #183
LX51 LINKER/LOCATER V4.66.41.0                                                        06/16/2023  10:23:34  PAGE 45


      01000FC5H   LINE      CODE     ---       #184
      01000FC5H   LINE      CODE     ---       #185
      01000FCAH   LINE      CODE     ---       #186
      01000FCAH   LINE      CODE     ---       #187
      01000FCBH   LINE      CODE     ---       #188
      01000FCEH   LINE      CODE     ---       #189
      01000FCEH   LINE      CODE     ---       #190
      01000FD3H   LINE      CODE     ---       #191
      01000FD3H   LINE      CODE     ---       #192
      01000FD4H   LINE      CODE     ---       #193
      01000FD7H   LINE      CODE     ---       #194
      01000FD7H   LINE      CODE     ---       #195
      01000FDCH   LINE      CODE     ---       #196
      01000FDCH   LINE      CODE     ---       #197
      01000FDDH   LINE      CODE     ---       #198
      01000FE0H   LINE      CODE     ---       #199
      01000FE0H   LINE      CODE     ---       #200
      01000FE5H   LINE      CODE     ---       #201
      01000FE5H   LINE      CODE     ---       #202
      01000FE6H   LINE      CODE     ---       #203
      01000FE9H   LINE      CODE     ---       #204
      01000FE9H   LINE      CODE     ---       #205
      01000FEEH   LINE      CODE     ---       #206
      01000FEEH   LINE      CODE     ---       #207
      01000FEFH   LINE      CODE     ---       #208
      01000FF2H   LINE      CODE     ---       #209
      01000FF2H   LINE      CODE     ---       #210
      ---         BLOCKEND  ---      ---       LVL=0
      00000007H   SYMBOL    DATA     BYTE      u8_length
      00000001H   SYMBOL    DATA     ---       u8_data_addr

      0100000EH   BLOCK     CODE     ---       LVL=0
      0100000EH   LINE      CODE     ---       #247
      0100000EH   LINE      CODE     ---       #249
      01000011H   LINE      CODE     ---       #253
      ---         BLOCKEND  ---      ---       LVL=0

      ---         MODULE    ---      ---       GPIO
      0100001EH   PUBLIC    CODE     ---       int8_15_rpt
      01000016H   PUBLIC    CODE     ---       int2_7_rpt
      01000012H   PUBLIC    CODE     ---       int1_rpt
      0100000AH   PUBLIC    CODE     ---       int0_rpt
      00000080H   SFRSYM    DATA     BYTE      P0
      00000090H   SFRSYM    DATA     BYTE      P1
      000000A0H   SFRSYM    DATA     BYTE      P2
      000000D0H.6 SFRSYM    DATA     BIT       AC
      000000A8H.7 SFRSYM    DATA     BIT       EA
      000000E7H   SFRSYM    DATA     BYTE      PWM0DTH
      000000CAH   SFRSYM    DATA     WORD      T3
      000000EFH   SFRSYM    DATA     BYTE      PWM1DTH
      000000ACH   SFRSYM    DATA     BYTE      SPCTL
      000000CDH   SFRSYM    DATA     WORD      T4
      000000F8H.4 SFRSYM    DATA     BIT       WDTRF
      000000F7H   SFRSYM    DATA     BYTE      PWM2DTH
      000000C2H   SFRSYM    DATA     WORD      T5
      00000098H.7 SFRSYM    DATA     BIT       FE
      000000E6H   SFRSYM    DATA     BYTE      PWM0DTL
      00000098H.5 SFRSYM    DATA     BIT       TXCOL
      000000EEH   SFRSYM    DATA     BYTE      PWM1DTL
      000000F6H   SFRSYM    DATA     BYTE      PWM2DTL
      000000B8H.5 SFRSYM    DATA     BIT       EADC
      00000091H   SFRSYM    DATA     BYTE      TICKCON
      000000A8H   SFRSYM    DATA     BYTE      IE
      00000080H   SFRSYM    DATA     BIT       P0_0
      000000F8H.1 SFRSYM    DATA     BIT       SPOVF
LX51 LINKER/LOCATER V4.66.41.0                                                        06/16/2023  10:23:34  PAGE 46


      000000FCH   SFRSYM    DATA     WORD      IAP_CMD
      00000090H   SFRSYM    DATA     BIT       P1_0
      00000080H.1 SFRSYM    DATA     BIT       P0_1
      000000A0H   SFRSYM    DATA     BIT       P2_0
      00000090H.1 SFRSYM    DATA     BIT       P1_1
      00000080H.2 SFRSYM    DATA     BIT       P0_2
      000000A0H.1 SFRSYM    DATA     BIT       P2_1
      00000080H.3 SFRSYM    DATA     BIT       P0_3
      000000F8H   SFRSYM    DATA     BYTE      RSTFR
      000000A0H.2 SFRSYM    DATA     BIT       P2_2
      00000080H.4 SFRSYM    DATA     BIT       P0_4
      000000A0H.3 SFRSYM    DATA     BIT       P2_3
      00000080H.5 SFRSYM    DATA     BIT       P0_5
      000000A0H.4 SFRSYM    DATA     BIT       P2_4
      00000080H.6 SFRSYM    DATA     BIT       P0_6
      000000A0H.5 SFRSYM    DATA     BIT       P2_5
      00000080H.7 SFRSYM    DATA     BIT       P0_7
      000000A0H.6 SFRSYM    DATA     BIT       P2_6
      000000A0H.7 SFRSYM    DATA     BIT       P2_7
      00000098H   SFRSYM    DATA     BIT       RI
      000000B8H.3 SFRSYM    DATA     BIT       EIIC
      000000B6H   SFRSYM    DATA     WORD      ADCR
      000000B8H.7 SFRSYM    DATA     BIT       EX8_15
      000000D0H.7 SFRSYM    DATA     BIT       CY
      00000098H.1 SFRSYM    DATA     BIT       TI
      000000FAH   SFRSYM    DATA     BYTE      IAP_ADDRH
      000000BFH   SFRSYM    DATA     BYTE      CRCH
      00000098H.6 SFRSYM    DATA     BIT       RXROV
      00000081H   SFRSYM    DATA     BYTE      SP
      000000F9H   SFRSYM    DATA     BYTE      IAP_ADDRL
      000000D0H.2 SFRSYM    DATA     BIT       OV
      000000BEH   SFRSYM    DATA     BYTE      CRCL
      000000C5H   SFRSYM    DATA     BYTE      RCAP5H
      000000C4H   SFRSYM    DATA     BYTE      RCAP5L
      000000F8H.5 SFRSYM    DATA     BIT       BORF
      000000BBH   SFRSYM    DATA     BYTE      LVDC
      000000BEH   SFRSYM    DATA     WORD      CRCR
      000000AFH   SFRSYM    DATA     BYTE      IICADR
      000000AEH   SFRSYM    DATA     BYTE      IICDAT
      00000099H   SFRSYM    DATA     BYTE      SBUF
      00000087H   SFRSYM    DATA     BYTE      PCON
      000000B8H   SFRSYM    DATA     BIT       ESPI
      000000E5H   SFRSYM    DATA     BYTE      PWM0DH
      000000EDH   SFRSYM    DATA     BYTE      PWM1DH
      00000096H   SFRSYM    DATA     BYTE      PINTF0
      000000BDH   SFRSYM    DATA     BYTE      WDTC
      000000F8H   SFRSYM    DATA     BIT       PLVRSTF
      000000F5H   SFRSYM    DATA     BYTE      PWM2DH
      00000098H   SFRSYM    DATA     BYTE      SCON
      00000097H   SFRSYM    DATA     BYTE      PINTF1
      000000A8H.5 SFRSYM    DATA     BIT       EWDT
      000000D1H   SFRSYM    DATA     BYTE      LCDCON
      00000089H   SFRSYM    DATA     BYTE      TMOD
      00000088H   SFRSYM    DATA     BYTE      TCON
      000000E4H   SFRSYM    DATA     BYTE      PWM0DL
      000000ECH   SFRSYM    DATA     BYTE      PWM1DL
      000000A6H   SFRSYM    DATA     BYTE      IICCON
      000000F8H.7 SFRSYM    DATA     BIT       PORF
      000000F4H   SFRSYM    DATA     BYTE      PWM2DL
      000000E1H   SFRSYM    DATA     BYTE      PWM0EN
      000000E9H   SFRSYM    DATA     BYTE      PWM1EN
      000000F1H   SFRSYM    DATA     BYTE      PWM2EN
      00000082H   SFRSYM    DATA     WORD      DPTR
      000000B4H   SFRSYM    DATA     BYTE      ADCC0
      0000008FH   SFRSYM    DATA     BYTE      CLKCON
LX51 LINKER/LOCATER V4.66.41.0                                                        06/16/2023  10:23:34  PAGE 47


      000000B5H   SFRSYM    DATA     BYTE      ADCC1
      000000E6H   SFRSYM    DATA     WORD      PWM0DT
      000000E3H   SFRSYM    DATA     BYTE      PWM0PH
      000000EEH   SFRSYM    DATA     WORD      PWM1DT
      000000EBH   SFRSYM    DATA     BYTE      PWM1PH
      000000A7H   SFRSYM    DATA     BYTE      IICSTA
      000000B8H   SFRSYM    DATA     BYTE      IE1
      000000F6H   SFRSYM    DATA     WORD      PWM2DT
      000000F3H   SFRSYM    DATA     BYTE      PWM2PH
      000000F0H   SFRSYM    DATA     BYTE      B
      000000E2H   SFRSYM    DATA     BYTE      PWM0PL
      000000F8H.3 SFRSYM    DATA     BIT       SWRF
      000000EAH   SFRSYM    DATA     BYTE      PWM1PL
      000000F2H   SFRSYM    DATA     BYTE      PWM2PL
      000000E0H   SFRSYM    DATA     BYTE      ACC
      000000BCH   SFRSYM    DATA     BYTE      LVDCMP
      000000A8H.1 SFRSYM    DATA     BIT       ET0
      000000A8H.4 SFRSYM    DATA     BIT       ES1
      000000A9H   SFRSYM    DATA     BYTE      IP0
      00000088H.5 SFRSYM    DATA     BIT       TF0
      000000A8H.3 SFRSYM    DATA     BIT       ET1
      000000A8H.6 SFRSYM    DATA     BIT       ES2
      000000AAH   SFRSYM    DATA     BYTE      IP1
      00000088H.7 SFRSYM    DATA     BIT       TF1
      000000B9H   SFRSYM    DATA     BYTE      IP2
      00000098H.2 SFRSYM    DATA     BIT       RB8
      000000B8H.1 SFRSYM    DATA     BIT       ET3
      0000008CH   SFRSYM    DATA     BYTE      TH0
      000000BAH   SFRSYM    DATA     BYTE      IP3
      000000A2H   SFRSYM    DATA     BYTE      INSCON
      000000B8H.2 SFRSYM    DATA     BIT       ET4
      000000A8H   SFRSYM    DATA     BIT       EX0
      0000008DH   SFRSYM    DATA     BYTE      TH1
      000000B1H   SFRSYM    DATA     BYTE      IP4
      00000098H.3 SFRSYM    DATA     BIT       TB8
      000000B8H.4 SFRSYM    DATA     BIT       ET5
      000000A8H.2 SFRSYM    DATA     BIT       EX1
      000000D0H   SFRSYM    DATA     BIT       P
      000000CBH   SFRSYM    DATA     BYTE      TH3
      000000CEH   SFRSYM    DATA     BYTE      TH4
      0000008AH   SFRSYM    DATA     BYTE      TL0
      000000C3H   SFRSYM    DATA     BYTE      TH5
      0000008BH   SFRSYM    DATA     BYTE      TL1
      000000CAH   SFRSYM    DATA     BYTE      TL3
      000000CDH   SFRSYM    DATA     BYTE      TL4
      000000D0H.3 SFRSYM    DATA     BIT       RS0
      000000C2H   SFRSYM    DATA     BYTE      TL5
      00000088H.4 SFRSYM    DATA     BIT       TR0
      000000D0H.4 SFRSYM    DATA     BIT       RS1
      000000FBH   SFRSYM    DATA     BYTE      IAP_DATA
      00000088H.6 SFRSYM    DATA     BIT       TR1
      000000F9H   SFRSYM    DATA     WORD      IAP_ADDR
      000000FDH   SFRSYM    DATA     BYTE      IAP_CMDH
      0000008EH   SFRSYM    DATA     BYTE      CLKSWR
      000000C4H   SFRSYM    DATA     WORD      RCAP5
      000000FCH   SFRSYM    DATA     BYTE      IAP_CMDL
      00000083H   SFRSYM    DATA     BYTE      DPH
      000000F8H.6 SFRSYM    DATA     BIT       EXRSTF
      00000082H   SFRSYM    DATA     BYTE      DPL
      000000ADH   SFRSYM    DATA     BYTE      SPSTAT
      000000B7H   SFRSYM    DATA     BYTE      ADCRH
      00000098H.4 SFRSYM    DATA     BIT       REN
      000000B8H.6 SFRSYM    DATA     BIT       EX2_7
      0000009EH   SFRSYM    DATA     BYTE      SCON2
      000000B6H   SFRSYM    DATA     BYTE      ADCRL
LX51 LINKER/LOCATER V4.66.41.0                                                        06/16/2023  10:23:34  PAGE 48


      000000DAH   SFRSYM    DATA     BYTE      PWM0C
      000000C9H   SFRSYM    DATA     BYTE      T3CON
      000000E4H   SFRSYM    DATA     WORD      PWM0D
      000000DBH   SFRSYM    DATA     BYTE      PWM1C
      000000CCH   SFRSYM    DATA     BYTE      T4CON
      000000ECH   SFRSYM    DATA     WORD      PWM1D
      000000DCH   SFRSYM    DATA     BYTE      PWM2C
      000000C1H   SFRSYM    DATA     BYTE      T5CON
      000000F4H   SFRSYM    DATA     WORD      PWM2D
      000000DDH   SFRSYM    DATA     BYTE      PWM3C
      000000DFH   SFRSYM    DATA     BYTE      PWM3D
      0000009BH   SFRSYM    DATA     BYTE      SADEN
      0000009AH   SFRSYM    DATA     BYTE      SADDR
      00000093H   SFRSYM    DATA     BYTE      TICKH
      000000D0H.5 SFRSYM    DATA     BIT       F0
      000000E2H   SFRSYM    DATA     WORD      PWM0P
      000000D0H.1 SFRSYM    DATA     BIT       F1
      000000EAH   SFRSYM    DATA     WORD      PWM1P
      000000F2H   SFRSYM    DATA     WORD      PWM2P
      000000DEH   SFRSYM    DATA     BYTE      PWM3P
      00000092H   SFRSYM    DATA     BYTE      TICKL
      000000D0H   SFRSYM    DATA     BYTE      PSW
      000000ABH   SFRSYM    DATA     BYTE      SPDAT

      0100000AH   BLOCK     CODE     ---       LVL=0
      0100000AH   LINE      CODE     ---       #97
      0100000AH   LINE      CODE     ---       #101
      0100000AH   LINE      CODE     ---       #102
      0100000AH   LINE      CODE     ---       #104
      0100000AH   LINE      CODE     ---       #106
      0100000AH   LINE      CODE     ---       #108
      0100000AH   LINE      CODE     ---       #109
      ---         BLOCKEND  ---      ---       LVL=0

      01000012H   BLOCK     CODE     ---       LVL=0
      01000012H   LINE      CODE     ---       #120
      01000012H   LINE      CODE     ---       #128
      ---         BLOCKEND  ---      ---       LVL=0

      01000016H   BLOCK     CODE     ---       LVL=0
      01000016H   LINE      CODE     ---       #139
      01000016H   LINE      CODE     ---       #141
      01000019H   LINE      CODE     ---       #147
      ---         BLOCKEND  ---      ---       LVL=0

      0100001EH   BLOCK     CODE     ---       LVL=0
      0100001EH   LINE      CODE     ---       #158
      0100001EH   LINE      CODE     ---       #160
      01000021H   LINE      CODE     ---       #166
      ---         BLOCKEND  ---      ---       LVL=0

      ---         MODULE    ---      ---       TIMER
      020000BAH   PUBLIC    XDATA    BYTE      b_t5_input_level
      020000B8H   PUBLIC    XDATA    WORD      u16_t5_catch_val
      01000D82H   PUBLIC    CODE     ---       timer5_service
      01000022H   PUBLIC    CODE     ---       timer4_service
      01001031H   PUBLIC    CODE     ---       timer3_service
      0100001AH   PUBLIC    CODE     ---       timer1_service
      0100113DH   PUBLIC    CODE     ---       timer0_service
      0100121AH   PUBLIC    CODE     ---       config_timer0_module
      00000080H   SFRSYM    DATA     BYTE      P0
      00000090H   SFRSYM    DATA     BYTE      P1
      000000A0H   SFRSYM    DATA     BYTE      P2
      000000D0H.6 SFRSYM    DATA     BIT       AC
      000000A8H.7 SFRSYM    DATA     BIT       EA
LX51 LINKER/LOCATER V4.66.41.0                                                        06/16/2023  10:23:34  PAGE 49


      000000E7H   SFRSYM    DATA     BYTE      PWM0DTH
      000000CAH   SFRSYM    DATA     WORD      T3
      000000EFH   SFRSYM    DATA     BYTE      PWM1DTH
      000000ACH   SFRSYM    DATA     BYTE      SPCTL
      000000CDH   SFRSYM    DATA     WORD      T4
      000000F8H.4 SFRSYM    DATA     BIT       WDTRF
      000000F7H   SFRSYM    DATA     BYTE      PWM2DTH
      000000C2H   SFRSYM    DATA     WORD      T5
      00000098H.7 SFRSYM    DATA     BIT       FE
      000000E6H   SFRSYM    DATA     BYTE      PWM0DTL
      00000098H.5 SFRSYM    DATA     BIT       TXCOL
      000000EEH   SFRSYM    DATA     BYTE      PWM1DTL
      000000F6H   SFRSYM    DATA     BYTE      PWM2DTL
      000000B8H.5 SFRSYM    DATA     BIT       EADC
      00000091H   SFRSYM    DATA     BYTE      TICKCON
      000000A8H   SFRSYM    DATA     BYTE      IE
      00000080H   SFRSYM    DATA     BIT       P0_0
      000000F8H.1 SFRSYM    DATA     BIT       SPOVF
      000000FCH   SFRSYM    DATA     WORD      IAP_CMD
      00000090H   SFRSYM    DATA     BIT       P1_0
      00000080H.1 SFRSYM    DATA     BIT       P0_1
      000000A0H   SFRSYM    DATA     BIT       P2_0
      00000090H.1 SFRSYM    DATA     BIT       P1_1
      00000080H.2 SFRSYM    DATA     BIT       P0_2
      000000A0H.1 SFRSYM    DATA     BIT       P2_1
      00000080H.3 SFRSYM    DATA     BIT       P0_3
      000000F8H   SFRSYM    DATA     BYTE      RSTFR
      000000A0H.2 SFRSYM    DATA     BIT       P2_2
      00000080H.4 SFRSYM    DATA     BIT       P0_4
      000000A0H.3 SFRSYM    DATA     BIT       P2_3
      00000080H.5 SFRSYM    DATA     BIT       P0_5
      000000A0H.4 SFRSYM    DATA     BIT       P2_4
      00000080H.6 SFRSYM    DATA     BIT       P0_6
      000000A0H.5 SFRSYM    DATA     BIT       P2_5
      00000080H.7 SFRSYM    DATA     BIT       P0_7
      000000A0H.6 SFRSYM    DATA     BIT       P2_6
      000000A0H.7 SFRSYM    DATA     BIT       P2_7
      00000098H   SFRSYM    DATA     BIT       RI
      000000B8H.3 SFRSYM    DATA     BIT       EIIC
      000000B6H   SFRSYM    DATA     WORD      ADCR
      000000B8H.7 SFRSYM    DATA     BIT       EX8_15
      000000D0H.7 SFRSYM    DATA     BIT       CY
      00000098H.1 SFRSYM    DATA     BIT       TI
      000000FAH   SFRSYM    DATA     BYTE      IAP_ADDRH
      000000BFH   SFRSYM    DATA     BYTE      CRCH
      00000098H.6 SFRSYM    DATA     BIT       RXROV
      00000081H   SFRSYM    DATA     BYTE      SP
      000000F9H   SFRSYM    DATA     BYTE      IAP_ADDRL
      000000D0H.2 SFRSYM    DATA     BIT       OV
      000000BEH   SFRSYM    DATA     BYTE      CRCL
      000000C5H   SFRSYM    DATA     BYTE      RCAP5H
      000000C4H   SFRSYM    DATA     BYTE      RCAP5L
      000000F8H.5 SFRSYM    DATA     BIT       BORF
      000000BBH   SFRSYM    DATA     BYTE      LVDC
      000000BEH   SFRSYM    DATA     WORD      CRCR
      000000AFH   SFRSYM    DATA     BYTE      IICADR
      000000AEH   SFRSYM    DATA     BYTE      IICDAT
      00000099H   SFRSYM    DATA     BYTE      SBUF
      00000087H   SFRSYM    DATA     BYTE      PCON
      000000B8H   SFRSYM    DATA     BIT       ESPI
      000000E5H   SFRSYM    DATA     BYTE      PWM0DH
      000000EDH   SFRSYM    DATA     BYTE      PWM1DH
      00000096H   SFRSYM    DATA     BYTE      PINTF0
      000000BDH   SFRSYM    DATA     BYTE      WDTC
      000000F8H   SFRSYM    DATA     BIT       PLVRSTF
LX51 LINKER/LOCATER V4.66.41.0                                                        06/16/2023  10:23:34  PAGE 50


      000000F5H   SFRSYM    DATA     BYTE      PWM2DH
      00000098H   SFRSYM    DATA     BYTE      SCON
      00000097H   SFRSYM    DATA     BYTE      PINTF1
      000000A8H.5 SFRSYM    DATA     BIT       EWDT
      000000D1H   SFRSYM    DATA     BYTE      LCDCON
      00000089H   SFRSYM    DATA     BYTE      TMOD
      00000088H   SFRSYM    DATA     BYTE      TCON
      000000E4H   SFRSYM    DATA     BYTE      PWM0DL
      000000ECH   SFRSYM    DATA     BYTE      PWM1DL
      000000A6H   SFRSYM    DATA     BYTE      IICCON
      000000F8H.7 SFRSYM    DATA     BIT       PORF
      000000F4H   SFRSYM    DATA     BYTE      PWM2DL
      000000E1H   SFRSYM    DATA     BYTE      PWM0EN
      000000E9H   SFRSYM    DATA     BYTE      PWM1EN
      000000F1H   SFRSYM    DATA     BYTE      PWM2EN
      00000082H   SFRSYM    DATA     WORD      DPTR
      000000B4H   SFRSYM    DATA     BYTE      ADCC0
      0000008FH   SFRSYM    DATA     BYTE      CLKCON
      000000B5H   SFRSYM    DATA     BYTE      ADCC1
      000000E6H   SFRSYM    DATA     WORD      PWM0DT
      000000E3H   SFRSYM    DATA     BYTE      PWM0PH
      000000EEH   SFRSYM    DATA     WORD      PWM1DT
      000000EBH   SFRSYM    DATA     BYTE      PWM1PH
      000000A7H   SFRSYM    DATA     BYTE      IICSTA
      000000B8H   SFRSYM    DATA     BYTE      IE1
      000000F6H   SFRSYM    DATA     WORD      PWM2DT
      000000F3H   SFRSYM    DATA     BYTE      PWM2PH
      000000F0H   SFRSYM    DATA     BYTE      B
      000000E2H   SFRSYM    DATA     BYTE      PWM0PL
      000000F8H.3 SFRSYM    DATA     BIT       SWRF
      000000EAH   SFRSYM    DATA     BYTE      PWM1PL
      000000F2H   SFRSYM    DATA     BYTE      PWM2PL
      000000E0H   SFRSYM    DATA     BYTE      ACC
      000000BCH   SFRSYM    DATA     BYTE      LVDCMP
      000000A8H.1 SFRSYM    DATA     BIT       ET0
      000000A8H.4 SFRSYM    DATA     BIT       ES1
      000000A9H   SFRSYM    DATA     BYTE      IP0
      00000088H.5 SFRSYM    DATA     BIT       TF0
      000000A8H.3 SFRSYM    DATA     BIT       ET1
      000000A8H.6 SFRSYM    DATA     BIT       ES2
      000000AAH   SFRSYM    DATA     BYTE      IP1
      00000088H.7 SFRSYM    DATA     BIT       TF1
      000000B9H   SFRSYM    DATA     BYTE      IP2
      00000098H.2 SFRSYM    DATA     BIT       RB8
      000000B8H.1 SFRSYM    DATA     BIT       ET3
      0000008CH   SFRSYM    DATA     BYTE      TH0
      000000BAH   SFRSYM    DATA     BYTE      IP3
      000000A2H   SFRSYM    DATA     BYTE      INSCON
      000000B8H.2 SFRSYM    DATA     BIT       ET4
      000000A8H   SFRSYM    DATA     BIT       EX0
      0000008DH   SFRSYM    DATA     BYTE      TH1
      000000B1H   SFRSYM    DATA     BYTE      IP4
      00000098H.3 SFRSYM    DATA     BIT       TB8
      000000B8H.4 SFRSYM    DATA     BIT       ET5
      000000A8H.2 SFRSYM    DATA     BIT       EX1
      000000D0H   SFRSYM    DATA     BIT       P
      000000CBH   SFRSYM    DATA     BYTE      TH3
      000000CEH   SFRSYM    DATA     BYTE      TH4
      0000008AH   SFRSYM    DATA     BYTE      TL0
      000000C3H   SFRSYM    DATA     BYTE      TH5
      0000008BH   SFRSYM    DATA     BYTE      TL1
      000000CAH   SFRSYM    DATA     BYTE      TL3
      000000CDH   SFRSYM    DATA     BYTE      TL4
      000000D0H.3 SFRSYM    DATA     BIT       RS0
      000000C2H   SFRSYM    DATA     BYTE      TL5
LX51 LINKER/LOCATER V4.66.41.0                                                        06/16/2023  10:23:34  PAGE 51


      00000088H.4 SFRSYM    DATA     BIT       TR0
      000000D0H.4 SFRSYM    DATA     BIT       RS1
      000000FBH   SFRSYM    DATA     BYTE      IAP_DATA
      00000088H.6 SFRSYM    DATA     BIT       TR1
      000000F9H   SFRSYM    DATA     WORD      IAP_ADDR
      000000FDH   SFRSYM    DATA     BYTE      IAP_CMDH
      0000008EH   SFRSYM    DATA     BYTE      CLKSWR
      000000C4H   SFRSYM    DATA     WORD      RCAP5
      000000FCH   SFRSYM    DATA     BYTE      IAP_CMDL
      00000083H   SFRSYM    DATA     BYTE      DPH
      000000F8H.6 SFRSYM    DATA     BIT       EXRSTF
      00000082H   SFRSYM    DATA     BYTE      DPL
      000000ADH   SFRSYM    DATA     BYTE      SPSTAT
      000000B7H   SFRSYM    DATA     BYTE      ADCRH
      00000098H.4 SFRSYM    DATA     BIT       REN
      000000B8H.6 SFRSYM    DATA     BIT       EX2_7
      0000009EH   SFRSYM    DATA     BYTE      SCON2
      000000B6H   SFRSYM    DATA     BYTE      ADCRL
      000000DAH   SFRSYM    DATA     BYTE      PWM0C
      000000C9H   SFRSYM    DATA     BYTE      T3CON
      000000E4H   SFRSYM    DATA     WORD      PWM0D
      000000DBH   SFRSYM    DATA     BYTE      PWM1C
      000000CCH   SFRSYM    DATA     BYTE      T4CON
      000000ECH   SFRSYM    DATA     WORD      PWM1D
      000000DCH   SFRSYM    DATA     BYTE      PWM2C
      000000C1H   SFRSYM    DATA     BYTE      T5CON
      000000F4H   SFRSYM    DATA     WORD      PWM2D
      000000DDH   SFRSYM    DATA     BYTE      PWM3C
      000000DFH   SFRSYM    DATA     BYTE      PWM3D
      0000009BH   SFRSYM    DATA     BYTE      SADEN
      0000009AH   SFRSYM    DATA     BYTE      SADDR
      00000093H   SFRSYM    DATA     BYTE      TICKH
      000000D0H.5 SFRSYM    DATA     BIT       F0
      000000E2H   SFRSYM    DATA     WORD      PWM0P
      000000D0H.1 SFRSYM    DATA     BIT       F1
      000000EAH   SFRSYM    DATA     WORD      PWM1P
      000000F2H   SFRSYM    DATA     WORD      PWM2P
      000000DEH   SFRSYM    DATA     BYTE      PWM3P
      00000092H   SFRSYM    DATA     BYTE      TICKL
      000000D0H   SFRSYM    DATA     BYTE      PSW
      000000ABH   SFRSYM    DATA     BYTE      SPDAT

      0100121AH   BLOCK     CODE     ---       LVL=0
      0100121AH   LINE      CODE     ---       #100
      0100121AH   LINE      CODE     ---       #101
      0100121AH   LINE      CODE     ---       #105
      01001221H   LINE      CODE     ---       #106
      01001221H   LINE      CODE     ---       #107
      01001224H   LINE      CODE     ---       #108
      01001227H   LINE      CODE     ---       #110
      0100122AH   LINE      CODE     ---       #112
      0100122DH   LINE      CODE     ---       #113
      ---         BLOCKEND  ---      ---       LVL=0

      0100113DH   BLOCK     CODE     ---       LVL=0
      0100113DH   LINE      CODE     ---       #219
      01001143H   LINE      CODE     ---       #225
      01001145H   LINE      CODE     ---       #226
      0100114BH   LINE      CODE     ---       #227
      01001151H   LINE      CODE     ---       #228
      0100115FH   LINE      CODE     ---       #229
      01001165H   LINE      CODE     ---       #241
      ---         BLOCKEND  ---      ---       LVL=0

      0100001AH   BLOCK     CODE     ---       LVL=0
LX51 LINKER/LOCATER V4.66.41.0                                                        06/16/2023  10:23:34  PAGE 52


      0100001AH   LINE      CODE     ---       #252
      0100001AH   LINE      CODE     ---       #260
      ---         BLOCKEND  ---      ---       LVL=0

      01001031H   BLOCK     CODE     ---       LVL=0
      01001031H   LINE      CODE     ---       #271
      01001039H   LINE      CODE     ---       #278
      0100103FH   LINE      CODE     ---       #279
      01001045H   LINE      CODE     ---       #280
      01001045H   LINE      CODE     ---       #281
      01001047H   LINE      CODE     ---       #282
      0100104DH   LINE      CODE     ---       #283
      01001052H   LINE      CODE     ---       #284
      01001052H   LINE      CODE     ---       #285
      01001054H   LINE      CODE     ---       #286
      0100105AH   LINE      CODE     ---       #287
      0100105FH   LINE      CODE     ---       #288
      0100105FH   LINE      CODE     ---       #289
      01001061H   LINE      CODE     ---       #290
      01001061H   LINE      CODE     ---       #291
      01001061H   LINE      CODE     ---       #292
      01001061H   LINE      CODE     ---       #293
      ---         BLOCKEND  ---      ---       LVL=0

      01000022H   BLOCK     CODE     ---       LVL=0
      01000022H   LINE      CODE     ---       #304
      01000022H   LINE      CODE     ---       #312
      ---         BLOCKEND  ---      ---       LVL=0

      01000D82H   BLOCK     CODE     ---       LVL=0
      01000D82H   LINE      CODE     ---       #324
      01000D8AH   LINE      CODE     ---       #326
      01000D8FH   LINE      CODE     ---       #327
      01000D8FH   LINE      CODE     ---       #328
      01000D92H   LINE      CODE     ---       #329
      01000D92H   LINE      CODE     ---       #334
      01000D97H   LINE      CODE     ---       #335
      01000D97H   LINE      CODE     ---       #336
      01000DA4H   LINE      CODE     ---       #337
      01000DA7H   LINE      CODE     ---       #339
      01000DABH   LINE      CODE     ---       #340
      01000DABH   LINE      CODE     ---       #341
      01000DAEH   LINE      CODE     ---       #342
      01000DB1H   LINE      CODE     ---       #343
      01000DB4H   LINE      CODE     ---       #344
      01000DB9H   LINE      CODE     ---       #345
      01000DBDH   LINE      CODE     ---       #346
      01000DBFH   LINE      CODE     ---       #348
      01000DBFH   LINE      CODE     ---       #349
      01000DC2H   LINE      CODE     ---       #350
      01000DC5H   LINE      CODE     ---       #351
      01000DC8H   LINE      CODE     ---       #352
      01000DCDH   LINE      CODE     ---       #353
      01000DD2H   LINE      CODE     ---       #354
      01000DD2H   LINE      CODE     ---       #355
      01000DD2H   LINE      CODE     ---       #356
      ---         BLOCKEND  ---      ---       LVL=0

      ---         MODULE    ---      ---       UART
      020000A9H   PUBLIC    XDATA    ---       u8_uart1_rx_data
      020000A8H   PUBLIC    XDATA    BYTE      u8_uart1_rx_data_index
      020000A7H   PUBLIC    XDATA    BYTE      u8_uart1_rx_ok
      01000ED1H   PUBLIC    CODE     ---       uart1_rpt
      00000080H   SFRSYM    DATA     BYTE      P0
      00000090H   SFRSYM    DATA     BYTE      P1
LX51 LINKER/LOCATER V4.66.41.0                                                        06/16/2023  10:23:34  PAGE 53


      000000A0H   SFRSYM    DATA     BYTE      P2
      000000D0H.6 SFRSYM    DATA     BIT       AC
      000000A8H.7 SFRSYM    DATA     BIT       EA
      000000E7H   SFRSYM    DATA     BYTE      PWM0DTH
      000000CAH   SFRSYM    DATA     WORD      T3
      000000EFH   SFRSYM    DATA     BYTE      PWM1DTH
      000000ACH   SFRSYM    DATA     BYTE      SPCTL
      000000CDH   SFRSYM    DATA     WORD      T4
      000000F8H.4 SFRSYM    DATA     BIT       WDTRF
      000000F7H   SFRSYM    DATA     BYTE      PWM2DTH
      000000C2H   SFRSYM    DATA     WORD      T5
      00000098H.7 SFRSYM    DATA     BIT       FE
      000000E6H   SFRSYM    DATA     BYTE      PWM0DTL
      00000098H.5 SFRSYM    DATA     BIT       TXCOL
      000000EEH   SFRSYM    DATA     BYTE      PWM1DTL
      000000F6H   SFRSYM    DATA     BYTE      PWM2DTL
      000000B8H.5 SFRSYM    DATA     BIT       EADC
      00000091H   SFRSYM    DATA     BYTE      TICKCON
      000000A8H   SFRSYM    DATA     BYTE      IE
      00000080H   SFRSYM    DATA     BIT       P0_0
      000000F8H.1 SFRSYM    DATA     BIT       SPOVF
      000000FCH   SFRSYM    DATA     WORD      IAP_CMD
      00000090H   SFRSYM    DATA     BIT       P1_0
      00000080H.1 SFRSYM    DATA     BIT       P0_1
      000000A0H   SFRSYM    DATA     BIT       P2_0
      00000090H.1 SFRSYM    DATA     BIT       P1_1
      00000080H.2 SFRSYM    DATA     BIT       P0_2
      000000A0H.1 SFRSYM    DATA     BIT       P2_1
      00000080H.3 SFRSYM    DATA     BIT       P0_3
      000000F8H   SFRSYM    DATA     BYTE      RSTFR
      000000A0H.2 SFRSYM    DATA     BIT       P2_2
      00000080H.4 SFRSYM    DATA     BIT       P0_4
      000000A0H.3 SFRSYM    DATA     BIT       P2_3
      00000080H.5 SFRSYM    DATA     BIT       P0_5
      000000A0H.4 SFRSYM    DATA     BIT       P2_4
      00000080H.6 SFRSYM    DATA     BIT       P0_6
      000000A0H.5 SFRSYM    DATA     BIT       P2_5
      00000080H.7 SFRSYM    DATA     BIT       P0_7
      000000A0H.6 SFRSYM    DATA     BIT       P2_6
      000000A0H.7 SFRSYM    DATA     BIT       P2_7
      00000098H   SFRSYM    DATA     BIT       RI
      000000B8H.3 SFRSYM    DATA     BIT       EIIC
      000000B6H   SFRSYM    DATA     WORD      ADCR
      000000B8H.7 SFRSYM    DATA     BIT       EX8_15
      000000D0H.7 SFRSYM    DATA     BIT       CY
      00000098H.1 SFRSYM    DATA     BIT       TI
      000000FAH   SFRSYM    DATA     BYTE      IAP_ADDRH
      000000BFH   SFRSYM    DATA     BYTE      CRCH
      00000098H.6 SFRSYM    DATA     BIT       RXROV
      00000081H   SFRSYM    DATA     BYTE      SP
      000000F9H   SFRSYM    DATA     BYTE      IAP_ADDRL
      000000D0H.2 SFRSYM    DATA     BIT       OV
      000000BEH   SFRSYM    DATA     BYTE      CRCL
      000000C5H   SFRSYM    DATA     BYTE      RCAP5H
      000000C4H   SFRSYM    DATA     BYTE      RCAP5L
      000000F8H.5 SFRSYM    DATA     BIT       BORF
      000000BBH   SFRSYM    DATA     BYTE      LVDC
      000000BEH   SFRSYM    DATA     WORD      CRCR
      000000AFH   SFRSYM    DATA     BYTE      IICADR
      000000AEH   SFRSYM    DATA     BYTE      IICDAT
      00000099H   SFRSYM    DATA     BYTE      SBUF
      00000087H   SFRSYM    DATA     BYTE      PCON
      000000B8H   SFRSYM    DATA     BIT       ESPI
      000000E5H   SFRSYM    DATA     BYTE      PWM0DH
      000000EDH   SFRSYM    DATA     BYTE      PWM1DH
LX51 LINKER/LOCATER V4.66.41.0                                                        06/16/2023  10:23:34  PAGE 54


      00000096H   SFRSYM    DATA     BYTE      PINTF0
      000000BDH   SFRSYM    DATA     BYTE      WDTC
      000000F8H   SFRSYM    DATA     BIT       PLVRSTF
      000000F5H   SFRSYM    DATA     BYTE      PWM2DH
      00000098H   SFRSYM    DATA     BYTE      SCON
      00000097H   SFRSYM    DATA     BYTE      PINTF1
      000000A8H.5 SFRSYM    DATA     BIT       EWDT
      000000D1H   SFRSYM    DATA     BYTE      LCDCON
      00000089H   SFRSYM    DATA     BYTE      TMOD
      00000088H   SFRSYM    DATA     BYTE      TCON
      000000E4H   SFRSYM    DATA     BYTE      PWM0DL
      000000ECH   SFRSYM    DATA     BYTE      PWM1DL
      000000A6H   SFRSYM    DATA     BYTE      IICCON
      000000F8H.7 SFRSYM    DATA     BIT       PORF
      000000F4H   SFRSYM    DATA     BYTE      PWM2DL
      000000E1H   SFRSYM    DATA     BYTE      PWM0EN
      000000E9H   SFRSYM    DATA     BYTE      PWM1EN
      000000F1H   SFRSYM    DATA     BYTE      PWM2EN
      00000082H   SFRSYM    DATA     WORD      DPTR
      000000B4H   SFRSYM    DATA     BYTE      ADCC0
      0000008FH   SFRSYM    DATA     BYTE      CLKCON
      000000B5H   SFRSYM    DATA     BYTE      ADCC1
      000000E6H   SFRSYM    DATA     WORD      PWM0DT
      000000E3H   SFRSYM    DATA     BYTE      PWM0PH
      000000EEH   SFRSYM    DATA     WORD      PWM1DT
      000000EBH   SFRSYM    DATA     BYTE      PWM1PH
      000000A7H   SFRSYM    DATA     BYTE      IICSTA
      000000B8H   SFRSYM    DATA     BYTE      IE1
      000000F6H   SFRSYM    DATA     WORD      PWM2DT
      000000F3H   SFRSYM    DATA     BYTE      PWM2PH
      000000F0H   SFRSYM    DATA     BYTE      B
      000000E2H   SFRSYM    DATA     BYTE      PWM0PL
      000000F8H.3 SFRSYM    DATA     BIT       SWRF
      000000EAH   SFRSYM    DATA     BYTE      PWM1PL
      000000F2H   SFRSYM    DATA     BYTE      PWM2PL
      000000E0H   SFRSYM    DATA     BYTE      ACC
      000000BCH   SFRSYM    DATA     BYTE      LVDCMP
      000000A8H.1 SFRSYM    DATA     BIT       ET0
      000000A8H.4 SFRSYM    DATA     BIT       ES1
      000000A9H   SFRSYM    DATA     BYTE      IP0
      00000088H.5 SFRSYM    DATA     BIT       TF0
      000000A8H.3 SFRSYM    DATA     BIT       ET1
      000000A8H.6 SFRSYM    DATA     BIT       ES2
      000000AAH   SFRSYM    DATA     BYTE      IP1
      00000088H.7 SFRSYM    DATA     BIT       TF1
      000000B9H   SFRSYM    DATA     BYTE      IP2
      00000098H.2 SFRSYM    DATA     BIT       RB8
      000000B8H.1 SFRSYM    DATA     BIT       ET3
      0000008CH   SFRSYM    DATA     BYTE      TH0
      000000BAH   SFRSYM    DATA     BYTE      IP3
      000000A2H   SFRSYM    DATA     BYTE      INSCON
      000000B8H.2 SFRSYM    DATA     BIT       ET4
      000000A8H   SFRSYM    DATA     BIT       EX0
      0000008DH   SFRSYM    DATA     BYTE      TH1
      000000B1H   SFRSYM    DATA     BYTE      IP4
      00000098H.3 SFRSYM    DATA     BIT       TB8
      000000B8H.4 SFRSYM    DATA     BIT       ET5
      000000A8H.2 SFRSYM    DATA     BIT       EX1
      000000D0H   SFRSYM    DATA     BIT       P
      000000CBH   SFRSYM    DATA     BYTE      TH3
      000000CEH   SFRSYM    DATA     BYTE      TH4
      0000008AH   SFRSYM    DATA     BYTE      TL0
      000000C3H   SFRSYM    DATA     BYTE      TH5
      0000008BH   SFRSYM    DATA     BYTE      TL1
      000000CAH   SFRSYM    DATA     BYTE      TL3
LX51 LINKER/LOCATER V4.66.41.0                                                        06/16/2023  10:23:34  PAGE 55


      000000CDH   SFRSYM    DATA     BYTE      TL4
      000000D0H.3 SFRSYM    DATA     BIT       RS0
      000000C2H   SFRSYM    DATA     BYTE      TL5
      00000088H.4 SFRSYM    DATA     BIT       TR0
      000000D0H.4 SFRSYM    DATA     BIT       RS1
      000000FBH   SFRSYM    DATA     BYTE      IAP_DATA
      00000088H.6 SFRSYM    DATA     BIT       TR1
      000000F9H   SFRSYM    DATA     WORD      IAP_ADDR
      000000FDH   SFRSYM    DATA     BYTE      IAP_CMDH
      0000008EH   SFRSYM    DATA     BYTE      CLKSWR
      000000C4H   SFRSYM    DATA     WORD      RCAP5
      000000FCH   SFRSYM    DATA     BYTE      IAP_CMDL
      00000083H   SFRSYM    DATA     BYTE      DPH
      000000F8H.6 SFRSYM    DATA     BIT       EXRSTF
      00000082H   SFRSYM    DATA     BYTE      DPL
      000000ADH   SFRSYM    DATA     BYTE      SPSTAT
      000000B7H   SFRSYM    DATA     BYTE      ADCRH
      00000098H.4 SFRSYM    DATA     BIT       REN
      000000B8H.6 SFRSYM    DATA     BIT       EX2_7
      0000009EH   SFRSYM    DATA     BYTE      SCON2
      000000B6H   SFRSYM    DATA     BYTE      ADCRL
      000000DAH   SFRSYM    DATA     BYTE      PWM0C
      000000C9H   SFRSYM    DATA     BYTE      T3CON
      000000E4H   SFRSYM    DATA     WORD      PWM0D
      000000DBH   SFRSYM    DATA     BYTE      PWM1C
      000000CCH   SFRSYM    DATA     BYTE      T4CON
      000000ECH   SFRSYM    DATA     WORD      PWM1D
      000000DCH   SFRSYM    DATA     BYTE      PWM2C
      000000C1H   SFRSYM    DATA     BYTE      T5CON
      000000F4H   SFRSYM    DATA     WORD      PWM2D
      000000DDH   SFRSYM    DATA     BYTE      PWM3C
      000000DFH   SFRSYM    DATA     BYTE      PWM3D
      0000009BH   SFRSYM    DATA     BYTE      SADEN
      0000009AH   SFRSYM    DATA     BYTE      SADDR
      00000093H   SFRSYM    DATA     BYTE      TICKH
      000000D0H.5 SFRSYM    DATA     BIT       F0
      000000E2H   SFRSYM    DATA     WORD      PWM0P
      000000D0H.1 SFRSYM    DATA     BIT       F1
      000000EAH   SFRSYM    DATA     WORD      PWM1P
      000000F2H   SFRSYM    DATA     WORD      PWM2P
      000000DEH   SFRSYM    DATA     BYTE      PWM3P
      00000092H   SFRSYM    DATA     BYTE      TICKL
      000000D0H   SFRSYM    DATA     BYTE      PSW
      000000ABH   SFRSYM    DATA     BYTE      SPDAT
      01000925H   SYMBOL    CODE     ---       _uart1_rx_data_int
      00000007H   SYMBOL    DATA     BYTE      u8_type
      00000007H   SYMBOL    DATA     BYTE      u8_data
      00000007H   SYMBOL    DATA     BYTE      u8_length
      00000006H   SYMBOL    DATA     BYTE      i
      00000001H   SYMBOL    DATA     ---       u8_index
      00000001H   SYMBOL    DATA     ---       u8_index

      01000925H   BLOCK     CODE     ---       LVL=0
      02000028H   SYMBOL    XDATA    ---       u8_index
      0200002BH   SYMBOL    XDATA    ---       u8_buf
      0200002EH   SYMBOL    XDATA    ---       u8_flag
      01000930H   BLOCK     CODE     NEAR LAB  LVL=1
      00000007H   SYMBOL    DATA     BYTE      buf
      ---         BLOCKEND  ---      ---       LVL=1
      01000925H   LINE      CODE     ---       #165
      01000930H   LINE      CODE     ---       #166
      01000930H   LINE      CODE     ---       #169
      01000938H   LINE      CODE     ---       #170
      01000938H   LINE      CODE     ---       #171
      0100093BH   LINE      CODE     ---       #172
LX51 LINKER/LOCATER V4.66.41.0                                                        06/16/2023  10:23:34  PAGE 56


      0100093DH   LINE      CODE     ---       #174
      01000950H   LINE      CODE     ---       #175
      01000950H   LINE      CODE     ---       #176
      01000954H   LINE      CODE     ---       #177
      01000954H   LINE      CODE     ---       #178
      01000966H   LINE      CODE     ---       #179
      01000966H   LINE      CODE     ---       #180
      0100097AH   LINE      CODE     ---       #181
      0100097AH   LINE      CODE     ---       #182
      01000987H   LINE      CODE     ---       #183
      01000989H   LINE      CODE     ---       #185
      01000989H   LINE      CODE     ---       #186
      01000999H   LINE      CODE     ---       #187
      010009B1H   LINE      CODE     ---       #188
      010009B7H   LINE      CODE     ---       #189
      010009B7H   LINE      CODE     ---       #190
      010009C7H   LINE      CODE     ---       #191
      010009D6H   LINE      CODE     ---       #192
      010009D6H   LINE      CODE     ---       #193
      010009D6H   LINE      CODE     ---       #194
      010009D6H   LINE      CODE     ---       #195
      010009D6H   LINE      CODE     ---       #196
      ---         BLOCKEND  ---      ---       LVL=0

      01000ED1H   BLOCK     CODE     ---       LVL=0
      01000ED1H   LINE      CODE     ---       #209
      01000EE8H   LINE      CODE     ---       #211
      01000F0BH   LINE      CODE     ---       #246
      ---         BLOCKEND  ---      ---       LVL=0
      00000004H   SYMBOL    DATA     DWORD     u32_num

      ---         MODULE    ---      ---       PWM
      0200008CH   PUBLIC    XDATA    WORD      u16_pwm2_ch1_duty
      0200008AH   PUBLIC    XDATA    WORD      u16_pwm1_ch1_duty
      02000088H   PUBLIC    XDATA    WORD      u16_pwm2_ch0_duty
      02000086H   PUBLIC    XDATA    WORD      u16_pwm0_ch1_duty
      02000084H   PUBLIC    XDATA    WORD      u16_pwm1_ch0_duty
      02000082H   PUBLIC    XDATA    WORD      u16_pwm0_ch0_duty
      02000081H   PUBLIC    XDATA    BYTE      u8_pwm3_duty
      01001196H   PUBLIC    CODE     ---       pwm_rpt
      010010D6H   PUBLIC    CODE     ---       _turn_off_pwm0
      01000CBFH   PUBLIC    CODE     ---       _turn_on_pwm0_idp
      01000F6AH   PUBLIC    CODE     ---       _config_pwm0_module
      00000080H   SFRSYM    DATA     BYTE      P0
      00000090H   SFRSYM    DATA     BYTE      P1
      000000A0H   SFRSYM    DATA     BYTE      P2
      000000D0H.6 SFRSYM    DATA     BIT       AC
      000000A8H.7 SFRSYM    DATA     BIT       EA
      000000E7H   SFRSYM    DATA     BYTE      PWM0DTH
      000000CAH   SFRSYM    DATA     WORD      T3
      000000EFH   SFRSYM    DATA     BYTE      PWM1DTH
      000000ACH   SFRSYM    DATA     BYTE      SPCTL
      000000CDH   SFRSYM    DATA     WORD      T4
      000000F8H.4 SFRSYM    DATA     BIT       WDTRF
      000000F7H   SFRSYM    DATA     BYTE      PWM2DTH
      000000C2H   SFRSYM    DATA     WORD      T5
      00000098H.7 SFRSYM    DATA     BIT       FE
      000000E6H   SFRSYM    DATA     BYTE      PWM0DTL
      00000098H.5 SFRSYM    DATA     BIT       TXCOL
      000000EEH   SFRSYM    DATA     BYTE      PWM1DTL
      000000F6H   SFRSYM    DATA     BYTE      PWM2DTL
      000000B8H.5 SFRSYM    DATA     BIT       EADC
      00000091H   SFRSYM    DATA     BYTE      TICKCON
      000000A8H   SFRSYM    DATA     BYTE      IE
      00000080H   SFRSYM    DATA     BIT       P0_0
LX51 LINKER/LOCATER V4.66.41.0                                                        06/16/2023  10:23:34  PAGE 57


      000000F8H.1 SFRSYM    DATA     BIT       SPOVF
      000000FCH   SFRSYM    DATA     WORD      IAP_CMD
      00000090H   SFRSYM    DATA     BIT       P1_0
      00000080H.1 SFRSYM    DATA     BIT       P0_1
      000000A0H   SFRSYM    DATA     BIT       P2_0
      00000090H.1 SFRSYM    DATA     BIT       P1_1
      00000080H.2 SFRSYM    DATA     BIT       P0_2
      000000A0H.1 SFRSYM    DATA     BIT       P2_1
      00000080H.3 SFRSYM    DATA     BIT       P0_3
      000000F8H   SFRSYM    DATA     BYTE      RSTFR
      000000A0H.2 SFRSYM    DATA     BIT       P2_2
      00000080H.4 SFRSYM    DATA     BIT       P0_4
      000000A0H.3 SFRSYM    DATA     BIT       P2_3
      00000080H.5 SFRSYM    DATA     BIT       P0_5
      000000A0H.4 SFRSYM    DATA     BIT       P2_4
      00000080H.6 SFRSYM    DATA     BIT       P0_6
      000000A0H.5 SFRSYM    DATA     BIT       P2_5
      00000080H.7 SFRSYM    DATA     BIT       P0_7
      000000A0H.6 SFRSYM    DATA     BIT       P2_6
      000000A0H.7 SFRSYM    DATA     BIT       P2_7
      00000098H   SFRSYM    DATA     BIT       RI
      000000B8H.3 SFRSYM    DATA     BIT       EIIC
      000000B6H   SFRSYM    DATA     WORD      ADCR
      000000B8H.7 SFRSYM    DATA     BIT       EX8_15
      000000D0H.7 SFRSYM    DATA     BIT       CY
      00000098H.1 SFRSYM    DATA     BIT       TI
      000000FAH   SFRSYM    DATA     BYTE      IAP_ADDRH
      000000BFH   SFRSYM    DATA     BYTE      CRCH
      00000098H.6 SFRSYM    DATA     BIT       RXROV
      00000081H   SFRSYM    DATA     BYTE      SP
      000000F9H   SFRSYM    DATA     BYTE      IAP_ADDRL
      000000D0H.2 SFRSYM    DATA     BIT       OV
      000000BEH   SFRSYM    DATA     BYTE      CRCL
      000000C5H   SFRSYM    DATA     BYTE      RCAP5H
      000000C4H   SFRSYM    DATA     BYTE      RCAP5L
      000000F8H.5 SFRSYM    DATA     BIT       BORF
      000000BBH   SFRSYM    DATA     BYTE      LVDC
      000000BEH   SFRSYM    DATA     WORD      CRCR
      000000AFH   SFRSYM    DATA     BYTE      IICADR
      000000AEH   SFRSYM    DATA     BYTE      IICDAT
      00000099H   SFRSYM    DATA     BYTE      SBUF
      00000087H   SFRSYM    DATA     BYTE      PCON
      000000B8H   SFRSYM    DATA     BIT       ESPI
      000000E5H   SFRSYM    DATA     BYTE      PWM0DH
      000000EDH   SFRSYM    DATA     BYTE      PWM1DH
      00000096H   SFRSYM    DATA     BYTE      PINTF0
      000000BDH   SFRSYM    DATA     BYTE      WDTC
      000000F8H   SFRSYM    DATA     BIT       PLVRSTF
      000000F5H   SFRSYM    DATA     BYTE      PWM2DH
      00000098H   SFRSYM    DATA     BYTE      SCON
      00000097H   SFRSYM    DATA     BYTE      PINTF1
      000000A8H.5 SFRSYM    DATA     BIT       EWDT
      000000D1H   SFRSYM    DATA     BYTE      LCDCON
      00000089H   SFRSYM    DATA     BYTE      TMOD
      00000088H   SFRSYM    DATA     BYTE      TCON
      000000E4H   SFRSYM    DATA     BYTE      PWM0DL
      000000ECH   SFRSYM    DATA     BYTE      PWM1DL
      000000A6H   SFRSYM    DATA     BYTE      IICCON
      000000F8H.7 SFRSYM    DATA     BIT       PORF
      000000F4H   SFRSYM    DATA     BYTE      PWM2DL
      000000E1H   SFRSYM    DATA     BYTE      PWM0EN
      000000E9H   SFRSYM    DATA     BYTE      PWM1EN
      000000F1H   SFRSYM    DATA     BYTE      PWM2EN
      00000082H   SFRSYM    DATA     WORD      DPTR
      000000B4H   SFRSYM    DATA     BYTE      ADCC0
LX51 LINKER/LOCATER V4.66.41.0                                                        06/16/2023  10:23:34  PAGE 58


      0000008FH   SFRSYM    DATA     BYTE      CLKCON
      000000B5H   SFRSYM    DATA     BYTE      ADCC1
      000000E6H   SFRSYM    DATA     WORD      PWM0DT
      000000E3H   SFRSYM    DATA     BYTE      PWM0PH
      000000EEH   SFRSYM    DATA     WORD      PWM1DT
      000000EBH   SFRSYM    DATA     BYTE      PWM1PH
      000000A7H   SFRSYM    DATA     BYTE      IICSTA
      000000B8H   SFRSYM    DATA     BYTE      IE1
      000000F6H   SFRSYM    DATA     WORD      PWM2DT
      000000F3H   SFRSYM    DATA     BYTE      PWM2PH
      000000F0H   SFRSYM    DATA     BYTE      B
      000000E2H   SFRSYM    DATA     BYTE      PWM0PL
      000000F8H.3 SFRSYM    DATA     BIT       SWRF
      000000EAH   SFRSYM    DATA     BYTE      PWM1PL
      000000F2H   SFRSYM    DATA     BYTE      PWM2PL
      000000E0H   SFRSYM    DATA     BYTE      ACC
      000000BCH   SFRSYM    DATA     BYTE      LVDCMP
      000000A8H.1 SFRSYM    DATA     BIT       ET0
      000000A8H.4 SFRSYM    DATA     BIT       ES1
      000000A9H   SFRSYM    DATA     BYTE      IP0
      00000088H.5 SFRSYM    DATA     BIT       TF0
      000000A8H.3 SFRSYM    DATA     BIT       ET1
      000000A8H.6 SFRSYM    DATA     BIT       ES2
      000000AAH   SFRSYM    DATA     BYTE      IP1
      00000088H.7 SFRSYM    DATA     BIT       TF1
      000000B9H   SFRSYM    DATA     BYTE      IP2
      00000098H.2 SFRSYM    DATA     BIT       RB8
      000000B8H.1 SFRSYM    DATA     BIT       ET3
      0000008CH   SFRSYM    DATA     BYTE      TH0
      000000BAH   SFRSYM    DATA     BYTE      IP3
      000000A2H   SFRSYM    DATA     BYTE      INSCON
      000000B8H.2 SFRSYM    DATA     BIT       ET4
      000000A8H   SFRSYM    DATA     BIT       EX0
      0000008DH   SFRSYM    DATA     BYTE      TH1
      000000B1H   SFRSYM    DATA     BYTE      IP4
      00000098H.3 SFRSYM    DATA     BIT       TB8
      000000B8H.4 SFRSYM    DATA     BIT       ET5
      000000A8H.2 SFRSYM    DATA     BIT       EX1
      000000D0H   SFRSYM    DATA     BIT       P
      000000CBH   SFRSYM    DATA     BYTE      TH3
      000000CEH   SFRSYM    DATA     BYTE      TH4
      0000008AH   SFRSYM    DATA     BYTE      TL0
      000000C3H   SFRSYM    DATA     BYTE      TH5
      0000008BH   SFRSYM    DATA     BYTE      TL1
      000000CAH   SFRSYM    DATA     BYTE      TL3
      000000CDH   SFRSYM    DATA     BYTE      TL4
      000000D0H.3 SFRSYM    DATA     BIT       RS0
      000000C2H   SFRSYM    DATA     BYTE      TL5
      00000088H.4 SFRSYM    DATA     BIT       TR0
      000000D0H.4 SFRSYM    DATA     BIT       RS1
      000000FBH   SFRSYM    DATA     BYTE      IAP_DATA
      00000088H.6 SFRSYM    DATA     BIT       TR1
      000000F9H   SFRSYM    DATA     WORD      IAP_ADDR
      000000FDH   SFRSYM    DATA     BYTE      IAP_CMDH
      0000008EH   SFRSYM    DATA     BYTE      CLKSWR
      000000C4H   SFRSYM    DATA     WORD      RCAP5
      000000FCH   SFRSYM    DATA     BYTE      IAP_CMDL
      00000083H   SFRSYM    DATA     BYTE      DPH
      000000F8H.6 SFRSYM    DATA     BIT       EXRSTF
      00000082H   SFRSYM    DATA     BYTE      DPL
      000000ADH   SFRSYM    DATA     BYTE      SPSTAT
      000000B7H   SFRSYM    DATA     BYTE      ADCRH
      00000098H.4 SFRSYM    DATA     BIT       REN
      000000B8H.6 SFRSYM    DATA     BIT       EX2_7
      0000009EH   SFRSYM    DATA     BYTE      SCON2
LX51 LINKER/LOCATER V4.66.41.0                                                        06/16/2023  10:23:34  PAGE 59


      000000B6H   SFRSYM    DATA     BYTE      ADCRL
      000000DAH   SFRSYM    DATA     BYTE      PWM0C
      000000C9H   SFRSYM    DATA     BYTE      T3CON
      000000E4H   SFRSYM    DATA     WORD      PWM0D
      000000DBH   SFRSYM    DATA     BYTE      PWM1C
      000000CCH   SFRSYM    DATA     BYTE      T4CON
      000000ECH   SFRSYM    DATA     WORD      PWM1D
      000000DCH   SFRSYM    DATA     BYTE      PWM2C
      000000C1H   SFRSYM    DATA     BYTE      T5CON
      000000F4H   SFRSYM    DATA     WORD      PWM2D
      000000DDH   SFRSYM    DATA     BYTE      PWM3C
      000000DFH   SFRSYM    DATA     BYTE      PWM3D
      0000009BH   SFRSYM    DATA     BYTE      SADEN
      0000009AH   SFRSYM    DATA     BYTE      SADDR
      00000093H   SFRSYM    DATA     BYTE      TICKH
      000000D0H.5 SFRSYM    DATA     BIT       F0
      000000E2H   SFRSYM    DATA     WORD      PWM0P
      000000D0H.1 SFRSYM    DATA     BIT       F1
      000000EAH   SFRSYM    DATA     WORD      PWM1P
      000000F2H   SFRSYM    DATA     WORD      PWM2P
      000000DEH   SFRSYM    DATA     BYTE      PWM3P
      00000092H   SFRSYM    DATA     BYTE      TICKL
      000000D0H   SFRSYM    DATA     BYTE      PSW
      000000ABH   SFRSYM    DATA     BYTE      SPDAT

      01000F6AH   BLOCK     CODE     ---       LVL=0
      00000007H   SYMBOL    DATA     BYTE      u8_ch
      01000F6AH   LINE      CODE     ---       #33
      01000F6AH   LINE      CODE     ---       #34
      01000F6AH   LINE      CODE     ---       #35
      01000F76H   LINE      CODE     ---       #36
      01000F76H   LINE      CODE     ---       #37
      01000F76H   LINE      CODE     ---       #38
      01000F7FH   LINE      CODE     ---       #39
      01000F81H   LINE      CODE     ---       #40
      01000F83H   LINE      CODE     ---       #41
      01000F83H   LINE      CODE     ---       #42
      01000F86H   LINE      CODE     ---       #43
      01000F86H   LINE      CODE     ---       #44
      01000F88H   LINE      CODE     ---       #45
      01000F88H   LINE      CODE     ---       #46
      01000F91H   LINE      CODE     ---       #47
      01000F93H   LINE      CODE     ---       #48
      01000F99H   LINE      CODE     ---       #49
      01000F9BH   LINE      CODE     ---       #50
      01000F9BH   LINE      CODE     ---       #51
      01000F9BH   LINE      CODE     ---       #54
      01000FA2H   LINE      CODE     ---       #55
      01000FA6H   LINE      CODE     ---       #58
      01000FA9H   LINE      CODE     ---       #59
      01000FACH   LINE      CODE     ---       #62
      01000FAFH   LINE      CODE     ---       #64
      01000FB2H   LINE      CODE     ---       #76
      ---         BLOCKEND  ---      ---       LVL=0
      00000002H   SYMBOL    DATA     WORD      u16_duty
      00000002H   SYMBOL    DATA     WORD      u16_duty

      01000CBFH   BLOCK     CODE     ---       LVL=0
      00000007H   SYMBOL    DATA     BYTE      u8_ch
      00000004H   SYMBOL    DATA     WORD      u16_duty0
      00000002H   SYMBOL    DATA     WORD      u16_duty1
      01000CBFH   LINE      CODE     ---       #116
      01000CBFH   LINE      CODE     ---       #117
      01000CBFH   LINE      CODE     ---       #118
      01000CC2H   LINE      CODE     ---       #119
LX51 LINKER/LOCATER V4.66.41.0                                                        06/16/2023  10:23:34  PAGE 60


      01000CCEH   LINE      CODE     ---       #120
      01000CCEH   LINE      CODE     ---       #121
      01000CCEH   LINE      CODE     ---       #122
      01000CD6H   LINE      CODE     ---       #123
      01000CD9H   LINE      CODE     ---       #124
      01000CDBH   LINE      CODE     ---       #126
      01000CE1H   LINE      CODE     ---       #127
      01000CE4H   LINE      CODE     ---       #128
      01000CE5H   LINE      CODE     ---       #129
      01000CE5H   LINE      CODE     ---       #130
      01000CEDH   LINE      CODE     ---       #131
      01000CF0H   LINE      CODE     ---       #132
      01000CF2H   LINE      CODE     ---       #134
      01000CF8H   LINE      CODE     ---       #135
      01000CFBH   LINE      CODE     ---       #136
      01000CFCH   LINE      CODE     ---       #137
      01000CFCH   LINE      CODE     ---       #138
      01000D04H   LINE      CODE     ---       #139
      01000D07H   LINE      CODE     ---       #140
      01000D0BH   LINE      CODE     ---       #141
      01000D13H   LINE      CODE     ---       #142
      01000D16H   LINE      CODE     ---       #143
      01000D1AH   LINE      CODE     ---       #145
      01000D20H   LINE      CODE     ---       #146
      01000D25H   LINE      CODE     ---       #147
      01000D28H   LINE      CODE     ---       #148
      01000D28H   LINE      CODE     ---       #149
      01000D28H   LINE      CODE     ---       #150
      ---         BLOCKEND  ---      ---       LVL=0
      00000006H   SYMBOL    DATA     INT       u8_ch
      00000004H   SYMBOL    DATA     WORD      u16_duty0
      00000002H   SYMBOL    DATA     WORD      u16_duty1

      010010D6H   BLOCK     CODE     ---       LVL=0
      00000007H   SYMBOL    DATA     BYTE      u8_ch
      010010D6H   LINE      CODE     ---       #183
      010010D6H   LINE      CODE     ---       #184
      010010D6H   LINE      CODE     ---       #185
      010010E2H   LINE      CODE     ---       #186
      010010E2H   LINE      CODE     ---       #187
      010010E2H   LINE      CODE     ---       #188
      010010E5H   LINE      CODE     ---       #189
      010010EBH   LINE      CODE     ---       #190
      010010EDH   LINE      CODE     ---       #191
      010010EEH   LINE      CODE     ---       #192
      010010EEH   LINE      CODE     ---       #193
      010010F1H   LINE      CODE     ---       #194
      010010F6H   LINE      CODE     ---       #195
      010010F6H   LINE      CODE     ---       #196
      010010F8H   LINE      CODE     ---       #197
      010010F8H   LINE      CODE     ---       #198
      010010FBH   LINE      CODE     ---       #199
      01001101H   LINE      CODE     ---       #200
      01001103H   LINE      CODE     ---       #201
      01001107H   LINE      CODE     ---       #202
      01001109H   LINE      CODE     ---       #203
      01001109H   LINE      CODE     ---       #204
      01001109H   LINE      CODE     ---       #205
      ---         BLOCKEND  ---      ---       LVL=0
      00000007H   SYMBOL    DATA     BYTE      u8_ch
      00000002H   SYMBOL    DATA     WORD      u16_duty
      00000002H   SYMBOL    DATA     WORD      u16_duty
      00000007H   SYMBOL    DATA     BYTE      u8_ch
      00000004H   SYMBOL    DATA     WORD      u16_duty0
      00000002H   SYMBOL    DATA     WORD      u16_duty1
LX51 LINKER/LOCATER V4.66.41.0                                                        06/16/2023  10:23:34  PAGE 61


      00000006H   SYMBOL    DATA     INT       u8_ch
      00000004H   SYMBOL    DATA     WORD      u16_duty0
      00000002H   SYMBOL    DATA     WORD      u16_duty1
      00000007H   SYMBOL    DATA     BYTE      u8_ch
      00000007H   SYMBOL    DATA     BYTE      u8_ch
      00000002H   SYMBOL    DATA     WORD      u16_duty
      00000002H   SYMBOL    DATA     WORD      u16_duty
      00000007H   SYMBOL    DATA     BYTE      u8_ch
      00000004H   SYMBOL    DATA     WORD      u16_duty0
      00000002H   SYMBOL    DATA     WORD      u16_duty1
      00000006H   SYMBOL    DATA     INT       u8_ch
      00000004H   SYMBOL    DATA     WORD      u16_duty0
      00000002H   SYMBOL    DATA     WORD      u16_duty1
      00000007H   SYMBOL    DATA     BYTE      u8_ch
      00000007H   SYMBOL    DATA     BYTE      u8_duty

      01001196H   BLOCK     CODE     ---       LVL=0
      01001196H   LINE      CODE     ---       #614
      01001198H   LINE      CODE     ---       #616
      0100119DH   LINE      CODE     ---       #617
      0100119DH   LINE      CODE     ---       #619
      010011A0H   LINE      CODE     ---       #621
      010011A0H   LINE      CODE     ---       #623
      010011A5H   LINE      CODE     ---       #624
      010011A5H   LINE      CODE     ---       #626
      010011A8H   LINE      CODE     ---       #628
      010011A8H   LINE      CODE     ---       #630
      010011ADH   LINE      CODE     ---       #631
      010011ADH   LINE      CODE     ---       #633
      010011B0H   LINE      CODE     ---       #635
      010011B0H   LINE      CODE     ---       #637
      010011B5H   LINE      CODE     ---       #638
      010011B5H   LINE      CODE     ---       #640
      010011B8H   LINE      CODE     ---       #642
      010011B8H   LINE      CODE     ---       #643
      ---         BLOCKEND  ---      ---       LVL=0

      ---         MODULE    ---      ---       ADC
      01000026H   PUBLIC    CODE     ---       adc_rpt
      010009D7H   PUBLIC    CODE     ---       _adc_sampling_continuous
      01001240H   PUBLIC    CODE     ---       adc_sampling_single
      010011BBH   PUBLIC    CODE     ---       config_adc_module
      00000080H   SFRSYM    DATA     BYTE      P0
      00000090H   SFRSYM    DATA     BYTE      P1
      000000A0H   SFRSYM    DATA     BYTE      P2
      000000D0H.6 SFRSYM    DATA     BIT       AC
      000000A8H.7 SFRSYM    DATA     BIT       EA
      000000E7H   SFRSYM    DATA     BYTE      PWM0DTH
      000000CAH   SFRSYM    DATA     WORD      T3
      000000EFH   SFRSYM    DATA     BYTE      PWM1DTH
      000000ACH   SFRSYM    DATA     BYTE      SPCTL
      000000CDH   SFRSYM    DATA     WORD      T4
      000000F8H.4 SFRSYM    DATA     BIT       WDTRF
      000000F7H   SFRSYM    DATA     BYTE      PWM2DTH
      000000C2H   SFRSYM    DATA     WORD      T5
      00000098H.7 SFRSYM    DATA     BIT       FE
      000000E6H   SFRSYM    DATA     BYTE      PWM0DTL
      00000098H.5 SFRSYM    DATA     BIT       TXCOL
      000000EEH   SFRSYM    DATA     BYTE      PWM1DTL
      000000F6H   SFRSYM    DATA     BYTE      PWM2DTL
      000000B8H.5 SFRSYM    DATA     BIT       EADC
      00000091H   SFRSYM    DATA     BYTE      TICKCON
      000000A8H   SFRSYM    DATA     BYTE      IE
      00000080H   SFRSYM    DATA     BIT       P0_0
      000000F8H.1 SFRSYM    DATA     BIT       SPOVF
LX51 LINKER/LOCATER V4.66.41.0                                                        06/16/2023  10:23:34  PAGE 62


      000000FCH   SFRSYM    DATA     WORD      IAP_CMD
      00000090H   SFRSYM    DATA     BIT       P1_0
      00000080H.1 SFRSYM    DATA     BIT       P0_1
      000000A0H   SFRSYM    DATA     BIT       P2_0
      00000090H.1 SFRSYM    DATA     BIT       P1_1
      00000080H.2 SFRSYM    DATA     BIT       P0_2
      000000A0H.1 SFRSYM    DATA     BIT       P2_1
      00000080H.3 SFRSYM    DATA     BIT       P0_3
      000000F8H   SFRSYM    DATA     BYTE      RSTFR
      000000A0H.2 SFRSYM    DATA     BIT       P2_2
      00000080H.4 SFRSYM    DATA     BIT       P0_4
      000000A0H.3 SFRSYM    DATA     BIT       P2_3
      00000080H.5 SFRSYM    DATA     BIT       P0_5
      000000A0H.4 SFRSYM    DATA     BIT       P2_4
      00000080H.6 SFRSYM    DATA     BIT       P0_6
      000000A0H.5 SFRSYM    DATA     BIT       P2_5
      00000080H.7 SFRSYM    DATA     BIT       P0_7
      000000A0H.6 SFRSYM    DATA     BIT       P2_6
      000000A0H.7 SFRSYM    DATA     BIT       P2_7
      00000098H   SFRSYM    DATA     BIT       RI
      000000B8H.3 SFRSYM    DATA     BIT       EIIC
      000000B6H   SFRSYM    DATA     WORD      ADCR
      000000B8H.7 SFRSYM    DATA     BIT       EX8_15
      000000D0H.7 SFRSYM    DATA     BIT       CY
      00000098H.1 SFRSYM    DATA     BIT       TI
      000000FAH   SFRSYM    DATA     BYTE      IAP_ADDRH
      000000BFH   SFRSYM    DATA     BYTE      CRCH
      00000098H.6 SFRSYM    DATA     BIT       RXROV
      00000081H   SFRSYM    DATA     BYTE      SP
      000000F9H   SFRSYM    DATA     BYTE      IAP_ADDRL
      000000D0H.2 SFRSYM    DATA     BIT       OV
      000000BEH   SFRSYM    DATA     BYTE      CRCL
      000000C5H   SFRSYM    DATA     BYTE      RCAP5H
      000000C4H   SFRSYM    DATA     BYTE      RCAP5L
      000000F8H.5 SFRSYM    DATA     BIT       BORF
      000000BBH   SFRSYM    DATA     BYTE      LVDC
      000000BEH   SFRSYM    DATA     WORD      CRCR
      000000AFH   SFRSYM    DATA     BYTE      IICADR
      000000AEH   SFRSYM    DATA     BYTE      IICDAT
      00000099H   SFRSYM    DATA     BYTE      SBUF
      00000087H   SFRSYM    DATA     BYTE      PCON
      000000B8H   SFRSYM    DATA     BIT       ESPI
      000000E5H   SFRSYM    DATA     BYTE      PWM0DH
      000000EDH   SFRSYM    DATA     BYTE      PWM1DH
      00000096H   SFRSYM    DATA     BYTE      PINTF0
      000000BDH   SFRSYM    DATA     BYTE      WDTC
      000000F8H   SFRSYM    DATA     BIT       PLVRSTF
      000000F5H   SFRSYM    DATA     BYTE      PWM2DH
      00000098H   SFRSYM    DATA     BYTE      SCON
      00000097H   SFRSYM    DATA     BYTE      PINTF1
      000000A8H.5 SFRSYM    DATA     BIT       EWDT
      000000D1H   SFRSYM    DATA     BYTE      LCDCON
      00000089H   SFRSYM    DATA     BYTE      TMOD
      00000088H   SFRSYM    DATA     BYTE      TCON
      000000E4H   SFRSYM    DATA     BYTE      PWM0DL
      000000ECH   SFRSYM    DATA     BYTE      PWM1DL
      000000A6H   SFRSYM    DATA     BYTE      IICCON
      000000F8H.7 SFRSYM    DATA     BIT       PORF
      000000F4H   SFRSYM    DATA     BYTE      PWM2DL
      000000E1H   SFRSYM    DATA     BYTE      PWM0EN
      000000E9H   SFRSYM    DATA     BYTE      PWM1EN
      000000F1H   SFRSYM    DATA     BYTE      PWM2EN
      00000082H   SFRSYM    DATA     WORD      DPTR
      000000B4H   SFRSYM    DATA     BYTE      ADCC0
      0000008FH   SFRSYM    DATA     BYTE      CLKCON
LX51 LINKER/LOCATER V4.66.41.0                                                        06/16/2023  10:23:34  PAGE 63


      000000B5H   SFRSYM    DATA     BYTE      ADCC1
      000000E6H   SFRSYM    DATA     WORD      PWM0DT
      000000E3H   SFRSYM    DATA     BYTE      PWM0PH
      000000EEH   SFRSYM    DATA     WORD      PWM1DT
      000000EBH   SFRSYM    DATA     BYTE      PWM1PH
      000000A7H   SFRSYM    DATA     BYTE      IICSTA
      000000B8H   SFRSYM    DATA     BYTE      IE1
      000000F6H   SFRSYM    DATA     WORD      PWM2DT
      000000F3H   SFRSYM    DATA     BYTE      PWM2PH
      000000F0H   SFRSYM    DATA     BYTE      B
      000000E2H   SFRSYM    DATA     BYTE      PWM0PL
      000000F8H.3 SFRSYM    DATA     BIT       SWRF
      000000EAH   SFRSYM    DATA     BYTE      PWM1PL
      000000F2H   SFRSYM    DATA     BYTE      PWM2PL
      000000E0H   SFRSYM    DATA     BYTE      ACC
      000000BCH   SFRSYM    DATA     BYTE      LVDCMP
      000000A8H.1 SFRSYM    DATA     BIT       ET0
      000000A8H.4 SFRSYM    DATA     BIT       ES1
      000000A9H   SFRSYM    DATA     BYTE      IP0
      00000088H.5 SFRSYM    DATA     BIT       TF0
      000000A8H.3 SFRSYM    DATA     BIT       ET1
      000000A8H.6 SFRSYM    DATA     BIT       ES2
      000000AAH   SFRSYM    DATA     BYTE      IP1
      00000088H.7 SFRSYM    DATA     BIT       TF1
      000000B9H   SFRSYM    DATA     BYTE      IP2
      00000098H.2 SFRSYM    DATA     BIT       RB8
      000000B8H.1 SFRSYM    DATA     BIT       ET3
      0000008CH   SFRSYM    DATA     BYTE      TH0
      000000BAH   SFRSYM    DATA     BYTE      IP3
      000000A2H   SFRSYM    DATA     BYTE      INSCON
      000000B8H.2 SFRSYM    DATA     BIT       ET4
      000000A8H   SFRSYM    DATA     BIT       EX0
      0000008DH   SFRSYM    DATA     BYTE      TH1
      000000B1H   SFRSYM    DATA     BYTE      IP4
      00000098H.3 SFRSYM    DATA     BIT       TB8
      000000B8H.4 SFRSYM    DATA     BIT       ET5
      000000A8H.2 SFRSYM    DATA     BIT       EX1
      000000D0H   SFRSYM    DATA     BIT       P
      000000CBH   SFRSYM    DATA     BYTE      TH3
      000000CEH   SFRSYM    DATA     BYTE      TH4
      0000008AH   SFRSYM    DATA     BYTE      TL0
      000000C3H   SFRSYM    DATA     BYTE      TH5
      0000008BH   SFRSYM    DATA     BYTE      TL1
      000000CAH   SFRSYM    DATA     BYTE      TL3
      000000CDH   SFRSYM    DATA     BYTE      TL4
      000000D0H.3 SFRSYM    DATA     BIT       RS0
      000000C2H   SFRSYM    DATA     BYTE      TL5
      00000088H.4 SFRSYM    DATA     BIT       TR0
      000000D0H.4 SFRSYM    DATA     BIT       RS1
      000000FBH   SFRSYM    DATA     BYTE      IAP_DATA
      00000088H.6 SFRSYM    DATA     BIT       TR1
      000000F9H   SFRSYM    DATA     WORD      IAP_ADDR
      000000FDH   SFRSYM    DATA     BYTE      IAP_CMDH
      0000008EH   SFRSYM    DATA     BYTE      CLKSWR
      000000C4H   SFRSYM    DATA     WORD      RCAP5
      000000FCH   SFRSYM    DATA     BYTE      IAP_CMDL
      00000083H   SFRSYM    DATA     BYTE      DPH
      000000F8H.6 SFRSYM    DATA     BIT       EXRSTF
      00000082H   SFRSYM    DATA     BYTE      DPL
      000000ADH   SFRSYM    DATA     BYTE      SPSTAT
      000000B7H   SFRSYM    DATA     BYTE      ADCRH
      00000098H.4 SFRSYM    DATA     BIT       REN
      000000B8H.6 SFRSYM    DATA     BIT       EX2_7
      0000009EH   SFRSYM    DATA     BYTE      SCON2
      000000B6H   SFRSYM    DATA     BYTE      ADCRL
LX51 LINKER/LOCATER V4.66.41.0                                                        06/16/2023  10:23:34  PAGE 64


      000000DAH   SFRSYM    DATA     BYTE      PWM0C
      000000C9H   SFRSYM    DATA     BYTE      T3CON
      000000E4H   SFRSYM    DATA     WORD      PWM0D
      000000DBH   SFRSYM    DATA     BYTE      PWM1C
      000000CCH   SFRSYM    DATA     BYTE      T4CON
      000000ECH   SFRSYM    DATA     WORD      PWM1D
      000000DCH   SFRSYM    DATA     BYTE      PWM2C
      000000C1H   SFRSYM    DATA     BYTE      T5CON
      000000F4H   SFRSYM    DATA     WORD      PWM2D
      000000DDH   SFRSYM    DATA     BYTE      PWM3C
      000000DFH   SFRSYM    DATA     BYTE      PWM3D
      0000009BH   SFRSYM    DATA     BYTE      SADEN
      0000009AH   SFRSYM    DATA     BYTE      SADDR
      00000093H   SFRSYM    DATA     BYTE      TICKH
      000000D0H.5 SFRSYM    DATA     BIT       F0
      000000E2H   SFRSYM    DATA     WORD      PWM0P
      000000D0H.1 SFRSYM    DATA     BIT       F1
      000000EAH   SFRSYM    DATA     WORD      PWM1P
      000000F2H   SFRSYM    DATA     WORD      PWM2P
      000000DEH   SFRSYM    DATA     BYTE      PWM3P
      00000092H   SFRSYM    DATA     BYTE      TICKL
      000000D0H   SFRSYM    DATA     BYTE      PSW
      000000ABH   SFRSYM    DATA     BYTE      SPDAT

      010011BBH   BLOCK     CODE     ---       LVL=0
      010011BBH   LINE      CODE     ---       #45
      010011BBH   LINE      CODE     ---       #46
      010011BBH   LINE      CODE     ---       #50
      010011BEH   LINE      CODE     ---       #52
      010011C1H   LINE      CODE     ---       #54
      010011C7H   LINE      CODE     ---       #56
      010011CCH   LINE      CODE     ---       #59
      010011D6H   LINE      CODE     ---       #60
      010011D9H   LINE      CODE     ---       #66
      ---         BLOCKEND  ---      ---       LVL=0

      01001240H   BLOCK     CODE     ---       LVL=0
      01001240H   LINE      CODE     ---       #78
      01001240H   LINE      CODE     ---       #79
      01001240H   LINE      CODE     ---       #81
      01001243H   LINE      CODE     ---       #83
      01001248H   LINE      CODE     ---       #85
      0100124BH   LINE      CODE     ---       #87
      0100124FH   LINE      CODE     ---       #88
      ---         BLOCKEND  ---      ---       LVL=0

      010009D7H   BLOCK     CODE     ---       LVL=0
      00000005H   SYMBOL    DATA     BYTE      u8_times
      010009D9H   BLOCK     CODE     NEAR LAB  LVL=1
      00000004H   SYMBOL    DATA     BYTE      i
      02000000H   SYMBOL    XDATA    WORD      tmp
      02000002H   SYMBOL    XDATA    WORD      min
      02000004H   SYMBOL    XDATA    WORD      max
      02000006H   SYMBOL    XDATA    WORD      sum
      ---         BLOCKEND  ---      ---       LVL=1
      010009D7H   LINE      CODE     ---       #100
      010009D9H   LINE      CODE     ---       #101
      010009D9H   LINE      CODE     ---       #106
      010009DCH   LINE      CODE     ---       #107
      010009E7H   LINE      CODE     ---       #108
      010009EDH   LINE      CODE     ---       #109
      010009F8H   LINE      CODE     ---       #110
      010009F8H   LINE      CODE     ---       #111
      010009FDH   LINE      CODE     ---       #112
      01000A08H   LINE      CODE     ---       #113
LX51 LINKER/LOCATER V4.66.41.0                                                        06/16/2023  10:23:34  PAGE 65


      01000A15H   LINE      CODE     ---       #114
      01000A15H   LINE      CODE     ---       #115
      01000A24H   LINE      CODE     ---       #116
      01000A24H   LINE      CODE     ---       #117
      01000A3AH   LINE      CODE     ---       #118
      01000A3AH   LINE      CODE     ---       #119
      01000A40H   LINE      CODE     ---       #120
      01000A40H   LINE      CODE     ---       #121
      01000A4CH   LINE      CODE     ---       #122
      01000A4FH   LINE      CODE     ---       #123
      01000A77H   LINE      CODE     ---       #124
      01000A7AH   LINE      CODE     ---       #126
      01000A88H   LINE      CODE     ---       #127
      ---         BLOCKEND  ---      ---       LVL=0
      02000070H   SYMBOL    XDATA    BYTE      u8_times
      02000071H   SYMBOL    XDATA    ---       u16_buf

      01000026H   BLOCK     CODE     ---       LVL=0
      01000026H   LINE      CODE     ---       #214
      01000026H   LINE      CODE     ---       #216
      01000029H   LINE      CODE     ---       #221
      ---         BLOCKEND  ---      ---       LVL=0

      ---         MODULE    ---      ---       FLASH
      00000080H   SFRSYM    DATA     BYTE      P0
      00000090H   SFRSYM    DATA     BYTE      P1
      000000A0H   SFRSYM    DATA     BYTE      P2
      000000D0H.6 SFRSYM    DATA     BIT       AC
      000000A8H.7 SFRSYM    DATA     BIT       EA
      000000E7H   SFRSYM    DATA     BYTE      PWM0DTH
      000000CAH   SFRSYM    DATA     WORD      T3
      000000EFH   SFRSYM    DATA     BYTE      PWM1DTH
      000000ACH   SFRSYM    DATA     BYTE      SPCTL
      000000CDH   SFRSYM    DATA     WORD      T4
      000000F8H.4 SFRSYM    DATA     BIT       WDTRF
      000000F7H   SFRSYM    DATA     BYTE      PWM2DTH
      000000C2H   SFRSYM    DATA     WORD      T5
      00000098H.7 SFRSYM    DATA     BIT       FE
      000000E6H   SFRSYM    DATA     BYTE      PWM0DTL
      00000098H.5 SFRSYM    DATA     BIT       TXCOL
      000000EEH   SFRSYM    DATA     BYTE      PWM1DTL
      000000F6H   SFRSYM    DATA     BYTE      PWM2DTL
      000000B8H.5 SFRSYM    DATA     BIT       EADC
      00000091H   SFRSYM    DATA     BYTE      TICKCON
      000000A8H   SFRSYM    DATA     BYTE      IE
      00000080H   SFRSYM    DATA     BIT       P0_0
      000000F8H.1 SFRSYM    DATA     BIT       SPOVF
      000000FCH   SFRSYM    DATA     WORD      IAP_CMD
      00000090H   SFRSYM    DATA     BIT       P1_0
      00000080H.1 SFRSYM    DATA     BIT       P0_1
      000000A0H   SFRSYM    DATA     BIT       P2_0
      00000090H.1 SFRSYM    DATA     BIT       P1_1
      00000080H.2 SFRSYM    DATA     BIT       P0_2
      000000A0H.1 SFRSYM    DATA     BIT       P2_1
      00000080H.3 SFRSYM    DATA     BIT       P0_3
      000000F8H   SFRSYM    DATA     BYTE      RSTFR
      000000A0H.2 SFRSYM    DATA     BIT       P2_2
      00000080H.4 SFRSYM    DATA     BIT       P0_4
      000000A0H.3 SFRSYM    DATA     BIT       P2_3
      00000080H.5 SFRSYM    DATA     BIT       P0_5
      000000A0H.4 SFRSYM    DATA     BIT       P2_4
      00000080H.6 SFRSYM    DATA     BIT       P0_6
      000000A0H.5 SFRSYM    DATA     BIT       P2_5
      00000080H.7 SFRSYM    DATA     BIT       P0_7
      000000A0H.6 SFRSYM    DATA     BIT       P2_6
LX51 LINKER/LOCATER V4.66.41.0                                                        06/16/2023  10:23:34  PAGE 66


      000000A0H.7 SFRSYM    DATA     BIT       P2_7
      00000098H   SFRSYM    DATA     BIT       RI
      000000B8H.3 SFRSYM    DATA     BIT       EIIC
      000000B6H   SFRSYM    DATA     WORD      ADCR
      000000B8H.7 SFRSYM    DATA     BIT       EX8_15
      000000D0H.7 SFRSYM    DATA     BIT       CY
      00000098H.1 SFRSYM    DATA     BIT       TI
      000000FAH   SFRSYM    DATA     BYTE      IAP_ADDRH
      000000BFH   SFRSYM    DATA     BYTE      CRCH
      00000098H.6 SFRSYM    DATA     BIT       RXROV
      00000081H   SFRSYM    DATA     BYTE      SP
      000000F9H   SFRSYM    DATA     BYTE      IAP_ADDRL
      000000D0H.2 SFRSYM    DATA     BIT       OV
      000000BEH   SFRSYM    DATA     BYTE      CRCL
      000000C5H   SFRSYM    DATA     BYTE      RCAP5H
      000000C4H   SFRSYM    DATA     BYTE      RCAP5L
      000000F8H.5 SFRSYM    DATA     BIT       BORF
      000000BBH   SFRSYM    DATA     BYTE      LVDC
      000000BEH   SFRSYM    DATA     WORD      CRCR
      000000AFH   SFRSYM    DATA     BYTE      IICADR
      000000AEH   SFRSYM    DATA     BYTE      IICDAT
      00000099H   SFRSYM    DATA     BYTE      SBUF
      00000087H   SFRSYM    DATA     BYTE      PCON
      000000B8H   SFRSYM    DATA     BIT       ESPI
      000000E5H   SFRSYM    DATA     BYTE      PWM0DH
      000000EDH   SFRSYM    DATA     BYTE      PWM1DH
      00000096H   SFRSYM    DATA     BYTE      PINTF0
      000000BDH   SFRSYM    DATA     BYTE      WDTC
      000000F8H   SFRSYM    DATA     BIT       PLVRSTF
      000000F5H   SFRSYM    DATA     BYTE      PWM2DH
      00000098H   SFRSYM    DATA     BYTE      SCON
      00000097H   SFRSYM    DATA     BYTE      PINTF1
      000000A8H.5 SFRSYM    DATA     BIT       EWDT
      000000D1H   SFRSYM    DATA     BYTE      LCDCON
      00000089H   SFRSYM    DATA     BYTE      TMOD
      00000088H   SFRSYM    DATA     BYTE      TCON
      000000E4H   SFRSYM    DATA     BYTE      PWM0DL
      000000ECH   SFRSYM    DATA     BYTE      PWM1DL
      000000A6H   SFRSYM    DATA     BYTE      IICCON
      000000F8H.7 SFRSYM    DATA     BIT       PORF
      000000F4H   SFRSYM    DATA     BYTE      PWM2DL
      000000E1H   SFRSYM    DATA     BYTE      PWM0EN
      000000E9H   SFRSYM    DATA     BYTE      PWM1EN
      000000F1H   SFRSYM    DATA     BYTE      PWM2EN
      00000082H   SFRSYM    DATA     WORD      DPTR
      000000B4H   SFRSYM    DATA     BYTE      ADCC0
      0000008FH   SFRSYM    DATA     BYTE      CLKCON
      000000B5H   SFRSYM    DATA     BYTE      ADCC1
      000000E6H   SFRSYM    DATA     WORD      PWM0DT
      000000E3H   SFRSYM    DATA     BYTE      PWM0PH
      000000EEH   SFRSYM    DATA     WORD      PWM1DT
      000000EBH   SFRSYM    DATA     BYTE      PWM1PH
      000000A7H   SFRSYM    DATA     BYTE      IICSTA
      000000B8H   SFRSYM    DATA     BYTE      IE1
      000000F6H   SFRSYM    DATA     WORD      PWM2DT
      000000F3H   SFRSYM    DATA     BYTE      PWM2PH
      000000F0H   SFRSYM    DATA     BYTE      B
      000000E2H   SFRSYM    DATA     BYTE      PWM0PL
      000000F8H.3 SFRSYM    DATA     BIT       SWRF
      000000EAH   SFRSYM    DATA     BYTE      PWM1PL
      000000F2H   SFRSYM    DATA     BYTE      PWM2PL
      000000E0H   SFRSYM    DATA     BYTE      ACC
      000000BCH   SFRSYM    DATA     BYTE      LVDCMP
      000000A8H.1 SFRSYM    DATA     BIT       ET0
      000000A8H.4 SFRSYM    DATA     BIT       ES1
LX51 LINKER/LOCATER V4.66.41.0                                                        06/16/2023  10:23:34  PAGE 67


      000000A9H   SFRSYM    DATA     BYTE      IP0
      00000088H.5 SFRSYM    DATA     BIT       TF0
      000000A8H.3 SFRSYM    DATA     BIT       ET1
      000000A8H.6 SFRSYM    DATA     BIT       ES2
      000000AAH   SFRSYM    DATA     BYTE      IP1
      00000088H.7 SFRSYM    DATA     BIT       TF1
      000000B9H   SFRSYM    DATA     BYTE      IP2
      00000098H.2 SFRSYM    DATA     BIT       RB8
      000000B8H.1 SFRSYM    DATA     BIT       ET3
      0000008CH   SFRSYM    DATA     BYTE      TH0
      000000BAH   SFRSYM    DATA     BYTE      IP3
      000000A2H   SFRSYM    DATA     BYTE      INSCON
      000000B8H.2 SFRSYM    DATA     BIT       ET4
      000000A8H   SFRSYM    DATA     BIT       EX0
      0000008DH   SFRSYM    DATA     BYTE      TH1
      000000B1H   SFRSYM    DATA     BYTE      IP4
      00000098H.3 SFRSYM    DATA     BIT       TB8
      000000B8H.4 SFRSYM    DATA     BIT       ET5
      000000A8H.2 SFRSYM    DATA     BIT       EX1
      000000D0H   SFRSYM    DATA     BIT       P
      000000CBH   SFRSYM    DATA     BYTE      TH3
      000000CEH   SFRSYM    DATA     BYTE      TH4
      0000008AH   SFRSYM    DATA     BYTE      TL0
      000000C3H   SFRSYM    DATA     BYTE      TH5
      0000008BH   SFRSYM    DATA     BYTE      TL1
      000000CAH   SFRSYM    DATA     BYTE      TL3
      000000CDH   SFRSYM    DATA     BYTE      TL4
      000000D0H.3 SFRSYM    DATA     BIT       RS0
      000000C2H   SFRSYM    DATA     BYTE      TL5
      00000088H.4 SFRSYM    DATA     BIT       TR0
      000000D0H.4 SFRSYM    DATA     BIT       RS1
      000000FBH   SFRSYM    DATA     BYTE      IAP_DATA
      00000088H.6 SFRSYM    DATA     BIT       TR1
      000000F9H   SFRSYM    DATA     WORD      IAP_ADDR
      000000FDH   SFRSYM    DATA     BYTE      IAP_CMDH
      0000008EH   SFRSYM    DATA     BYTE      CLKSWR
      000000C4H   SFRSYM    DATA     WORD      RCAP5
      000000FCH   SFRSYM    DATA     BYTE      IAP_CMDL
      00000083H   SFRSYM    DATA     BYTE      DPH
      000000F8H.6 SFRSYM    DATA     BIT       EXRSTF
      00000082H   SFRSYM    DATA     BYTE      DPL
      000000ADH   SFRSYM    DATA     BYTE      SPSTAT
      000000B7H   SFRSYM    DATA     BYTE      ADCRH
      00000098H.4 SFRSYM    DATA     BIT       REN
      000000B8H.6 SFRSYM    DATA     BIT       EX2_7
      0000009EH   SFRSYM    DATA     BYTE      SCON2
      000000B6H   SFRSYM    DATA     BYTE      ADCRL
      000000DAH   SFRSYM    DATA     BYTE      PWM0C
      000000C9H   SFRSYM    DATA     BYTE      T3CON
      000000E4H   SFRSYM    DATA     WORD      PWM0D
      000000DBH   SFRSYM    DATA     BYTE      PWM1C
      000000CCH   SFRSYM    DATA     BYTE      T4CON
      000000ECH   SFRSYM    DATA     WORD      PWM1D
      000000DCH   SFRSYM    DATA     BYTE      PWM2C
      000000C1H   SFRSYM    DATA     BYTE      T5CON
      000000F4H   SFRSYM    DATA     WORD      PWM2D
      000000DDH   SFRSYM    DATA     BYTE      PWM3C
      000000DFH   SFRSYM    DATA     BYTE      PWM3D
      0000009BH   SFRSYM    DATA     BYTE      SADEN
      0000009AH   SFRSYM    DATA     BYTE      SADDR
      00000093H   SFRSYM    DATA     BYTE      TICKH
      000000D0H.5 SFRSYM    DATA     BIT       F0
      000000E2H   SFRSYM    DATA     WORD      PWM0P
      000000D0H.1 SFRSYM    DATA     BIT       F1
      000000EAH   SFRSYM    DATA     WORD      PWM1P
LX51 LINKER/LOCATER V4.66.41.0                                                        06/16/2023  10:23:34  PAGE 68


      000000F2H   SFRSYM    DATA     WORD      PWM2P
      000000DEH   SFRSYM    DATA     BYTE      PWM3P
      00000092H   SFRSYM    DATA     BYTE      TICKL
      000000D0H   SFRSYM    DATA     BYTE      PSW
      000000ABH   SFRSYM    DATA     BYTE      SPDAT
      00000006H   SYMBOL    DATA     WORD      u16_addr
      00000006H   SYMBOL    DATA     WORD      u16_addr
      00000005H   SYMBOL    DATA     BYTE      u8_data
      00000001H   SYMBOL    DATA     ---       u8_save_arr
      00000004H   SYMBOL    DATA     BYTE      i
      00000005H   SYMBOL    DATA     BYTE      u8_length
      00000001H   SYMBOL    DATA     ---       u8_save_arr

      ---         MODULE    ---      ---       SPI
      0200009FH   PUBLIC    XDATA    BYTE      u8_spi_rx_cnt
      02000099H   PUBLIC    XDATA    ---       u8_spi_receive_buf
      02000098H   PUBLIC    XDATA    BYTE      u8_spi_rx_flag
      01000E30H   PUBLIC    CODE     ---       SPI_Rpt
      00000080H   SFRSYM    DATA     BYTE      P0
      00000090H   SFRSYM    DATA     BYTE      P1
      000000A0H   SFRSYM    DATA     BYTE      P2
      000000D0H.6 SFRSYM    DATA     BIT       AC
      000000A8H.7 SFRSYM    DATA     BIT       EA
      000000E7H   SFRSYM    DATA     BYTE      PWM0DTH
      000000CAH   SFRSYM    DATA     WORD      T3
      000000EFH   SFRSYM    DATA     BYTE      PWM1DTH
      000000ACH   SFRSYM    DATA     BYTE      SPCTL
      000000CDH   SFRSYM    DATA     WORD      T4
      000000F8H.4 SFRSYM    DATA     BIT       WDTRF
      000000F7H   SFRSYM    DATA     BYTE      PWM2DTH
      000000C2H   SFRSYM    DATA     WORD      T5
      00000098H.7 SFRSYM    DATA     BIT       FE
      000000E6H   SFRSYM    DATA     BYTE      PWM0DTL
      00000098H.5 SFRSYM    DATA     BIT       TXCOL
      000000EEH   SFRSYM    DATA     BYTE      PWM1DTL
      000000F6H   SFRSYM    DATA     BYTE      PWM2DTL
      000000B8H.5 SFRSYM    DATA     BIT       EADC
      00000091H   SFRSYM    DATA     BYTE      TICKCON
      000000A8H   SFRSYM    DATA     BYTE      IE
      00000080H   SFRSYM    DATA     BIT       P0_0
      000000F8H.1 SFRSYM    DATA     BIT       SPOVF
      000000FCH   SFRSYM    DATA     WORD      IAP_CMD
      00000090H   SFRSYM    DATA     BIT       P1_0
      00000080H.1 SFRSYM    DATA     BIT       P0_1
      000000A0H   SFRSYM    DATA     BIT       P2_0
      00000090H.1 SFRSYM    DATA     BIT       P1_1
      00000080H.2 SFRSYM    DATA     BIT       P0_2
      000000A0H.1 SFRSYM    DATA     BIT       P2_1
      00000080H.3 SFRSYM    DATA     BIT       P0_3
      000000F8H   SFRSYM    DATA     BYTE      RSTFR
      000000A0H.2 SFRSYM    DATA     BIT       P2_2
      00000080H.4 SFRSYM    DATA     BIT       P0_4
      000000A0H.3 SFRSYM    DATA     BIT       P2_3
      00000080H.5 SFRSYM    DATA     BIT       P0_5
      000000A0H.4 SFRSYM    DATA     BIT       P2_4
      00000080H.6 SFRSYM    DATA     BIT       P0_6
      000000A0H.5 SFRSYM    DATA     BIT       P2_5
      00000080H.7 SFRSYM    DATA     BIT       P0_7
      000000A0H.6 SFRSYM    DATA     BIT       P2_6
      000000A0H.7 SFRSYM    DATA     BIT       P2_7
      00000098H   SFRSYM    DATA     BIT       RI
      000000B8H.3 SFRSYM    DATA     BIT       EIIC
      000000B6H   SFRSYM    DATA     WORD      ADCR
      000000B8H.7 SFRSYM    DATA     BIT       EX8_15
      000000D0H.7 SFRSYM    DATA     BIT       CY
LX51 LINKER/LOCATER V4.66.41.0                                                        06/16/2023  10:23:34  PAGE 69


      00000098H.1 SFRSYM    DATA     BIT       TI
      000000FAH   SFRSYM    DATA     BYTE      IAP_ADDRH
      000000BFH   SFRSYM    DATA     BYTE      CRCH
      00000098H.6 SFRSYM    DATA     BIT       RXROV
      00000081H   SFRSYM    DATA     BYTE      SP
      000000F9H   SFRSYM    DATA     BYTE      IAP_ADDRL
      000000D0H.2 SFRSYM    DATA     BIT       OV
      000000BEH   SFRSYM    DATA     BYTE      CRCL
      000000C5H   SFRSYM    DATA     BYTE      RCAP5H
      000000C4H   SFRSYM    DATA     BYTE      RCAP5L
      000000F8H.5 SFRSYM    DATA     BIT       BORF
      000000BBH   SFRSYM    DATA     BYTE      LVDC
      000000BEH   SFRSYM    DATA     WORD      CRCR
      000000AFH   SFRSYM    DATA     BYTE      IICADR
      000000AEH   SFRSYM    DATA     BYTE      IICDAT
      00000099H   SFRSYM    DATA     BYTE      SBUF
      00000087H   SFRSYM    DATA     BYTE      PCON
      000000B8H   SFRSYM    DATA     BIT       ESPI
      000000E5H   SFRSYM    DATA     BYTE      PWM0DH
      000000EDH   SFRSYM    DATA     BYTE      PWM1DH
      00000096H   SFRSYM    DATA     BYTE      PINTF0
      000000BDH   SFRSYM    DATA     BYTE      WDTC
      000000F8H   SFRSYM    DATA     BIT       PLVRSTF
      000000F5H   SFRSYM    DATA     BYTE      PWM2DH
      00000098H   SFRSYM    DATA     BYTE      SCON
      00000097H   SFRSYM    DATA     BYTE      PINTF1
      000000A8H.5 SFRSYM    DATA     BIT       EWDT
      000000D1H   SFRSYM    DATA     BYTE      LCDCON
      00000089H   SFRSYM    DATA     BYTE      TMOD
      00000088H   SFRSYM    DATA     BYTE      TCON
      000000E4H   SFRSYM    DATA     BYTE      PWM0DL
      000000ECH   SFRSYM    DATA     BYTE      PWM1DL
      000000A6H   SFRSYM    DATA     BYTE      IICCON
      000000F8H.7 SFRSYM    DATA     BIT       PORF
      000000F4H   SFRSYM    DATA     BYTE      PWM2DL
      000000E1H   SFRSYM    DATA     BYTE      PWM0EN
      000000E9H   SFRSYM    DATA     BYTE      PWM1EN
      000000F1H   SFRSYM    DATA     BYTE      PWM2EN
      00000082H   SFRSYM    DATA     WORD      DPTR
      000000B4H   SFRSYM    DATA     BYTE      ADCC0
      0000008FH   SFRSYM    DATA     BYTE      CLKCON
      000000B5H   SFRSYM    DATA     BYTE      ADCC1
      000000E6H   SFRSYM    DATA     WORD      PWM0DT
      000000E3H   SFRSYM    DATA     BYTE      PWM0PH
      000000EEH   SFRSYM    DATA     WORD      PWM1DT
      000000EBH   SFRSYM    DATA     BYTE      PWM1PH
      000000A7H   SFRSYM    DATA     BYTE      IICSTA
      000000B8H   SFRSYM    DATA     BYTE      IE1
      000000F6H   SFRSYM    DATA     WORD      PWM2DT
      000000F3H   SFRSYM    DATA     BYTE      PWM2PH
      000000F0H   SFRSYM    DATA     BYTE      B
      000000E2H   SFRSYM    DATA     BYTE      PWM0PL
      000000F8H.3 SFRSYM    DATA     BIT       SWRF
      000000EAH   SFRSYM    DATA     BYTE      PWM1PL
      000000F2H   SFRSYM    DATA     BYTE      PWM2PL
      000000E0H   SFRSYM    DATA     BYTE      ACC
      000000BCH   SFRSYM    DATA     BYTE      LVDCMP
      000000A8H.1 SFRSYM    DATA     BIT       ET0
      000000A8H.4 SFRSYM    DATA     BIT       ES1
      000000A9H   SFRSYM    DATA     BYTE      IP0
      00000088H.5 SFRSYM    DATA     BIT       TF0
      000000A8H.3 SFRSYM    DATA     BIT       ET1
      000000A8H.6 SFRSYM    DATA     BIT       ES2
      000000AAH   SFRSYM    DATA     BYTE      IP1
      00000088H.7 SFRSYM    DATA     BIT       TF1
LX51 LINKER/LOCATER V4.66.41.0                                                        06/16/2023  10:23:34  PAGE 70


      000000B9H   SFRSYM    DATA     BYTE      IP2
      00000098H.2 SFRSYM    DATA     BIT       RB8
      000000B8H.1 SFRSYM    DATA     BIT       ET3
      0000008CH   SFRSYM    DATA     BYTE      TH0
      000000BAH   SFRSYM    DATA     BYTE      IP3
      000000A2H   SFRSYM    DATA     BYTE      INSCON
      000000B8H.2 SFRSYM    DATA     BIT       ET4
      000000A8H   SFRSYM    DATA     BIT       EX0
      0000008DH   SFRSYM    DATA     BYTE      TH1
      000000B1H   SFRSYM    DATA     BYTE      IP4
      00000098H.3 SFRSYM    DATA     BIT       TB8
      000000B8H.4 SFRSYM    DATA     BIT       ET5
      000000A8H.2 SFRSYM    DATA     BIT       EX1
      000000D0H   SFRSYM    DATA     BIT       P
      000000CBH   SFRSYM    DATA     BYTE      TH3
      000000CEH   SFRSYM    DATA     BYTE      TH4
      0000008AH   SFRSYM    DATA     BYTE      TL0
      000000C3H   SFRSYM    DATA     BYTE      TH5
      0000008BH   SFRSYM    DATA     BYTE      TL1
      000000CAH   SFRSYM    DATA     BYTE      TL3
      000000CDH   SFRSYM    DATA     BYTE      TL4
      000000D0H.3 SFRSYM    DATA     BIT       RS0
      000000C2H   SFRSYM    DATA     BYTE      TL5
      00000088H.4 SFRSYM    DATA     BIT       TR0
      000000D0H.4 SFRSYM    DATA     BIT       RS1
      000000FBH   SFRSYM    DATA     BYTE      IAP_DATA
      00000088H.6 SFRSYM    DATA     BIT       TR1
      000000F9H   SFRSYM    DATA     WORD      IAP_ADDR
      000000FDH   SFRSYM    DATA     BYTE      IAP_CMDH
      0000008EH   SFRSYM    DATA     BYTE      CLKSWR
      000000C4H   SFRSYM    DATA     WORD      RCAP5
      000000FCH   SFRSYM    DATA     BYTE      IAP_CMDL
      00000083H   SFRSYM    DATA     BYTE      DPH
      000000F8H.6 SFRSYM    DATA     BIT       EXRSTF
      00000082H   SFRSYM    DATA     BYTE      DPL
      000000ADH   SFRSYM    DATA     BYTE      SPSTAT
      000000B7H   SFRSYM    DATA     BYTE      ADCRH
      00000098H.4 SFRSYM    DATA     BIT       REN
      000000B8H.6 SFRSYM    DATA     BIT       EX2_7
      0000009EH   SFRSYM    DATA     BYTE      SCON2
      000000B6H   SFRSYM    DATA     BYTE      ADCRL
      000000DAH   SFRSYM    DATA     BYTE      PWM0C
      000000C9H   SFRSYM    DATA     BYTE      T3CON
      000000E4H   SFRSYM    DATA     WORD      PWM0D
      000000DBH   SFRSYM    DATA     BYTE      PWM1C
      000000CCH   SFRSYM    DATA     BYTE      T4CON
      000000ECH   SFRSYM    DATA     WORD      PWM1D
      000000DCH   SFRSYM    DATA     BYTE      PWM2C
      000000C1H   SFRSYM    DATA     BYTE      T5CON
      000000F4H   SFRSYM    DATA     WORD      PWM2D
      000000DDH   SFRSYM    DATA     BYTE      PWM3C
      000000DFH   SFRSYM    DATA     BYTE      PWM3D
      0000009BH   SFRSYM    DATA     BYTE      SADEN
      0000009AH   SFRSYM    DATA     BYTE      SADDR
      00000093H   SFRSYM    DATA     BYTE      TICKH
      000000D0H.5 SFRSYM    DATA     BIT       F0
      000000E2H   SFRSYM    DATA     WORD      PWM0P
      000000D0H.1 SFRSYM    DATA     BIT       F1
      000000EAH   SFRSYM    DATA     WORD      PWM1P
      000000F2H   SFRSYM    DATA     WORD      PWM2P
      000000DEH   SFRSYM    DATA     BYTE      PWM3P
      00000092H   SFRSYM    DATA     BYTE      TICKL
      000000D0H   SFRSYM    DATA     BYTE      PSW
      000000ABH   SFRSYM    DATA     BYTE      SPDAT
      01000A89H   SYMBOL    CODE     ---       _spi_slave_read_int
LX51 LINKER/LOCATER V4.66.41.0                                                        06/16/2023  10:23:34  PAGE 71


      00000007H   SYMBOL    DATA     BYTE      u8_length
      00000006H   SYMBOL    DATA     BYTE      i
      00000007H   SYMBOL    DATA     BYTE      u8_length
      00000006H   SYMBOL    DATA     BYTE      i

      01000A89H   BLOCK     CODE     ---       LVL=0
      02000031H   SYMBOL    XDATA    ---       u8_index
      02000034H   SYMBOL    XDATA    ---       u8_buf
      02000037H   SYMBOL    XDATA    ---       u8_flag
      01000A94H   BLOCK     CODE     NEAR LAB  LVL=1
      00000007H   SYMBOL    DATA     BYTE      buf
      ---         BLOCKEND  ---      ---       LVL=1
      01000A89H   LINE      CODE     ---       #153
      01000A94H   LINE      CODE     ---       #154
      01000A94H   LINE      CODE     ---       #157
      01000A96H   LINE      CODE     ---       #159
      01000A9EH   LINE      CODE     ---       #160
      01000A9EH   LINE      CODE     ---       #161
      01000AADH   LINE      CODE     ---       #162
      01000AADH   LINE      CODE     ---       #163
      01000ABFH   LINE      CODE     ---       #164
      01000ABFH   LINE      CODE     ---       #165
      01000AD3H   LINE      CODE     ---       #166
      01000AD3H   LINE      CODE     ---       #167
      01000AE0H   LINE      CODE     ---       #168
      01000AE2H   LINE      CODE     ---       #170
      01000AE2H   LINE      CODE     ---       #171
      01000AF2H   LINE      CODE     ---       #172
      01000B0AH   LINE      CODE     ---       #173
      01000B10H   LINE      CODE     ---       #174
      01000B10H   LINE      CODE     ---       #175
      01000B20H   LINE      CODE     ---       #176
      01000B2FH   LINE      CODE     ---       #177
      01000B2FH   LINE      CODE     ---       #178
      01000B2FH   LINE      CODE     ---       #179
      01000B2FH   LINE      CODE     ---       #180
      ---         BLOCKEND  ---      ---       LVL=0

      01000E30H   BLOCK     CODE     ---       LVL=0
      01000E30H   LINE      CODE     ---       #191
      01000E47H   LINE      CODE     ---       #194
      01000E4AH   LINE      CODE     ---       #196
      01000E6DH   LINE      CODE     ---       #197
      ---         BLOCKEND  ---      ---       LVL=0

      ---         MODULE    ---      ---       IIC
      02000097H   PUBLIC    XDATA    BYTE      u8_iic_send_cnt
      02000093H   PUBLIC    XDATA    ---       u8_iic_send_buf
      02000092H   PUBLIC    XDATA    BYTE      u8_iic_rece_cnt
      0200008EH   PUBLIC    XDATA    ---       u8_iic_rece_buf
      01000857H   PUBLIC    CODE     ---       IIC_Rpt
      00000080H   SFRSYM    DATA     BYTE      P0
      00000090H   SFRSYM    DATA     BYTE      P1
      000000A0H   SFRSYM    DATA     BYTE      P2
      000000D0H.6 SFRSYM    DATA     BIT       AC
      000000A8H.7 SFRSYM    DATA     BIT       EA
      000000E7H   SFRSYM    DATA     BYTE      PWM0DTH
      000000CAH   SFRSYM    DATA     WORD      T3
      000000EFH   SFRSYM    DATA     BYTE      PWM1DTH
      000000ACH   SFRSYM    DATA     BYTE      SPCTL
      000000CDH   SFRSYM    DATA     WORD      T4
      000000F8H.4 SFRSYM    DATA     BIT       WDTRF
      000000F7H   SFRSYM    DATA     BYTE      PWM2DTH
      000000C2H   SFRSYM    DATA     WORD      T5
      00000098H.7 SFRSYM    DATA     BIT       FE
LX51 LINKER/LOCATER V4.66.41.0                                                        06/16/2023  10:23:34  PAGE 72


      000000E6H   SFRSYM    DATA     BYTE      PWM0DTL
      00000098H.5 SFRSYM    DATA     BIT       TXCOL
      000000EEH   SFRSYM    DATA     BYTE      PWM1DTL
      000000F6H   SFRSYM    DATA     BYTE      PWM2DTL
      000000B8H.5 SFRSYM    DATA     BIT       EADC
      00000091H   SFRSYM    DATA     BYTE      TICKCON
      000000A8H   SFRSYM    DATA     BYTE      IE
      00000080H   SFRSYM    DATA     BIT       P0_0
      000000F8H.1 SFRSYM    DATA     BIT       SPOVF
      000000FCH   SFRSYM    DATA     WORD      IAP_CMD
      00000090H   SFRSYM    DATA     BIT       P1_0
      00000080H.1 SFRSYM    DATA     BIT       P0_1
      000000A0H   SFRSYM    DATA     BIT       P2_0
      00000090H.1 SFRSYM    DATA     BIT       P1_1
      00000080H.2 SFRSYM    DATA     BIT       P0_2
      000000A0H.1 SFRSYM    DATA     BIT       P2_1
      00000080H.3 SFRSYM    DATA     BIT       P0_3
      000000F8H   SFRSYM    DATA     BYTE      RSTFR
      000000A0H.2 SFRSYM    DATA     BIT       P2_2
      00000080H.4 SFRSYM    DATA     BIT       P0_4
      000000A0H.3 SFRSYM    DATA     BIT       P2_3
      00000080H.5 SFRSYM    DATA     BIT       P0_5
      000000A0H.4 SFRSYM    DATA     BIT       P2_4
      00000080H.6 SFRSYM    DATA     BIT       P0_6
      000000A0H.5 SFRSYM    DATA     BIT       P2_5
      00000080H.7 SFRSYM    DATA     BIT       P0_7
      000000A0H.6 SFRSYM    DATA     BIT       P2_6
      000000A0H.7 SFRSYM    DATA     BIT       P2_7
      00000098H   SFRSYM    DATA     BIT       RI
      000000B8H.3 SFRSYM    DATA     BIT       EIIC
      000000B6H   SFRSYM    DATA     WORD      ADCR
      000000B8H.7 SFRSYM    DATA     BIT       EX8_15
      000000D0H.7 SFRSYM    DATA     BIT       CY
      00000098H.1 SFRSYM    DATA     BIT       TI
      000000FAH   SFRSYM    DATA     BYTE      IAP_ADDRH
      000000BFH   SFRSYM    DATA     BYTE      CRCH
      00000098H.6 SFRSYM    DATA     BIT       RXROV
      00000081H   SFRSYM    DATA     BYTE      SP
      000000F9H   SFRSYM    DATA     BYTE      IAP_ADDRL
      000000D0H.2 SFRSYM    DATA     BIT       OV
      000000BEH   SFRSYM    DATA     BYTE      CRCL
      000000C5H   SFRSYM    DATA     BYTE      RCAP5H
      000000C4H   SFRSYM    DATA     BYTE      RCAP5L
      000000F8H.5 SFRSYM    DATA     BIT       BORF
      000000BBH   SFRSYM    DATA     BYTE      LVDC
      000000BEH   SFRSYM    DATA     WORD      CRCR
      000000AFH   SFRSYM    DATA     BYTE      IICADR
      000000AEH   SFRSYM    DATA     BYTE      IICDAT
      00000099H   SFRSYM    DATA     BYTE      SBUF
      00000087H   SFRSYM    DATA     BYTE      PCON
      000000B8H   SFRSYM    DATA     BIT       ESPI
      000000E5H   SFRSYM    DATA     BYTE      PWM0DH
      000000EDH   SFRSYM    DATA     BYTE      PWM1DH
      00000096H   SFRSYM    DATA     BYTE      PINTF0
      000000BDH   SFRSYM    DATA     BYTE      WDTC
      000000F8H   SFRSYM    DATA     BIT       PLVRSTF
      000000F5H   SFRSYM    DATA     BYTE      PWM2DH
      00000098H   SFRSYM    DATA     BYTE      SCON
      00000097H   SFRSYM    DATA     BYTE      PINTF1
      000000A8H.5 SFRSYM    DATA     BIT       EWDT
      000000D1H   SFRSYM    DATA     BYTE      LCDCON
      00000089H   SFRSYM    DATA     BYTE      TMOD
      00000088H   SFRSYM    DATA     BYTE      TCON
      000000E4H   SFRSYM    DATA     BYTE      PWM0DL
      000000ECH   SFRSYM    DATA     BYTE      PWM1DL
LX51 LINKER/LOCATER V4.66.41.0                                                        06/16/2023  10:23:34  PAGE 73


      000000A6H   SFRSYM    DATA     BYTE      IICCON
      000000F8H.7 SFRSYM    DATA     BIT       PORF
      000000F4H   SFRSYM    DATA     BYTE      PWM2DL
      000000E1H   SFRSYM    DATA     BYTE      PWM0EN
      000000E9H   SFRSYM    DATA     BYTE      PWM1EN
      000000F1H   SFRSYM    DATA     BYTE      PWM2EN
      00000082H   SFRSYM    DATA     WORD      DPTR
      000000B4H   SFRSYM    DATA     BYTE      ADCC0
      0000008FH   SFRSYM    DATA     BYTE      CLKCON
      000000B5H   SFRSYM    DATA     BYTE      ADCC1
      000000E6H   SFRSYM    DATA     WORD      PWM0DT
      000000E3H   SFRSYM    DATA     BYTE      PWM0PH
      000000EEH   SFRSYM    DATA     WORD      PWM1DT
      000000EBH   SFRSYM    DATA     BYTE      PWM1PH
      000000A7H   SFRSYM    DATA     BYTE      IICSTA
      000000B8H   SFRSYM    DATA     BYTE      IE1
      000000F6H   SFRSYM    DATA     WORD      PWM2DT
      000000F3H   SFRSYM    DATA     BYTE      PWM2PH
      000000F0H   SFRSYM    DATA     BYTE      B
      000000E2H   SFRSYM    DATA     BYTE      PWM0PL
      000000F8H.3 SFRSYM    DATA     BIT       SWRF
      000000EAH   SFRSYM    DATA     BYTE      PWM1PL
      000000F2H   SFRSYM    DATA     BYTE      PWM2PL
      000000E0H   SFRSYM    DATA     BYTE      ACC
      000000BCH   SFRSYM    DATA     BYTE      LVDCMP
      000000A8H.1 SFRSYM    DATA     BIT       ET0
      000000A8H.4 SFRSYM    DATA     BIT       ES1
      000000A9H   SFRSYM    DATA     BYTE      IP0
      00000088H.5 SFRSYM    DATA     BIT       TF0
      000000A8H.3 SFRSYM    DATA     BIT       ET1
      000000A8H.6 SFRSYM    DATA     BIT       ES2
      000000AAH   SFRSYM    DATA     BYTE      IP1
      00000088H.7 SFRSYM    DATA     BIT       TF1
      000000B9H   SFRSYM    DATA     BYTE      IP2
      00000098H.2 SFRSYM    DATA     BIT       RB8
      000000B8H.1 SFRSYM    DATA     BIT       ET3
      0000008CH   SFRSYM    DATA     BYTE      TH0
      000000BAH   SFRSYM    DATA     BYTE      IP3
      000000A2H   SFRSYM    DATA     BYTE      INSCON
      000000B8H.2 SFRSYM    DATA     BIT       ET4
      000000A8H   SFRSYM    DATA     BIT       EX0
      0000008DH   SFRSYM    DATA     BYTE      TH1
      000000B1H   SFRSYM    DATA     BYTE      IP4
      00000098H.3 SFRSYM    DATA     BIT       TB8
      000000B8H.4 SFRSYM    DATA     BIT       ET5
      000000A8H.2 SFRSYM    DATA     BIT       EX1
      000000D0H   SFRSYM    DATA     BIT       P
      000000CBH   SFRSYM    DATA     BYTE      TH3
      000000CEH   SFRSYM    DATA     BYTE      TH4
      0000008AH   SFRSYM    DATA     BYTE      TL0
      000000C3H   SFRSYM    DATA     BYTE      TH5
      0000008BH   SFRSYM    DATA     BYTE      TL1
      000000CAH   SFRSYM    DATA     BYTE      TL3
      000000CDH   SFRSYM    DATA     BYTE      TL4
      000000D0H.3 SFRSYM    DATA     BIT       RS0
      000000C2H   SFRSYM    DATA     BYTE      TL5
      00000088H.4 SFRSYM    DATA     BIT       TR0
      000000D0H.4 SFRSYM    DATA     BIT       RS1
      000000FBH   SFRSYM    DATA     BYTE      IAP_DATA
      00000088H.6 SFRSYM    DATA     BIT       TR1
      000000F9H   SFRSYM    DATA     WORD      IAP_ADDR
      000000FDH   SFRSYM    DATA     BYTE      IAP_CMDH
      0000008EH   SFRSYM    DATA     BYTE      CLKSWR
      000000C4H   SFRSYM    DATA     WORD      RCAP5
      000000FCH   SFRSYM    DATA     BYTE      IAP_CMDL
LX51 LINKER/LOCATER V4.66.41.0                                                        06/16/2023  10:23:34  PAGE 74


      00000083H   SFRSYM    DATA     BYTE      DPH
      000000F8H.6 SFRSYM    DATA     BIT       EXRSTF
      00000082H   SFRSYM    DATA     BYTE      DPL
      000000ADH   SFRSYM    DATA     BYTE      SPSTAT
      000000B7H   SFRSYM    DATA     BYTE      ADCRH
      00000098H.4 SFRSYM    DATA     BIT       REN
      000000B8H.6 SFRSYM    DATA     BIT       EX2_7
      0000009EH   SFRSYM    DATA     BYTE      SCON2
      000000B6H   SFRSYM    DATA     BYTE      ADCRL
      000000DAH   SFRSYM    DATA     BYTE      PWM0C
      000000C9H   SFRSYM    DATA     BYTE      T3CON
      000000E4H   SFRSYM    DATA     WORD      PWM0D
      000000DBH   SFRSYM    DATA     BYTE      PWM1C
      000000CCH   SFRSYM    DATA     BYTE      T4CON
      000000ECH   SFRSYM    DATA     WORD      PWM1D
      000000DCH   SFRSYM    DATA     BYTE      PWM2C
      000000C1H   SFRSYM    DATA     BYTE      T5CON
      000000F4H   SFRSYM    DATA     WORD      PWM2D
      000000DDH   SFRSYM    DATA     BYTE      PWM3C
      000000DFH   SFRSYM    DATA     BYTE      PWM3D
      0000009BH   SFRSYM    DATA     BYTE      SADEN
      0000009AH   SFRSYM    DATA     BYTE      SADDR
      00000093H   SFRSYM    DATA     BYTE      TICKH
      000000D0H.5 SFRSYM    DATA     BIT       F0
      000000E2H   SFRSYM    DATA     WORD      PWM0P
      000000D0H.1 SFRSYM    DATA     BIT       F1
      000000EAH   SFRSYM    DATA     WORD      PWM1P
      000000F2H   SFRSYM    DATA     WORD      PWM2P
      000000DEH   SFRSYM    DATA     BYTE      PWM3P
      00000092H   SFRSYM    DATA     BYTE      TICKL
      000000D0H   SFRSYM    DATA     BYTE      PSW
      000000ABH   SFRSYM    DATA     BYTE      SPDAT
      00000007H   SYMBOL    DATA     BYTE      u8_length
      00000006H   SYMBOL    DATA     BYTE      i
      00000007H   SYMBOL    DATA     BYTE      u8_length
      00000006H   SYMBOL    DATA     BYTE      i

      01000857H   BLOCK     CODE     ---       LVL=0
      01000857H   LINE      CODE     ---       #201
      01000864H   LINE      CODE     ---       #203
      0100087EH   LINE      CODE     ---       #204
      0100087EH   LINE      CODE     ---       #205
      0100087EH   LINE      CODE     ---       #207
      01000881H   LINE      CODE     ---       #208
      01000884H   LINE      CODE     ---       #209
      01000884H   LINE      CODE     ---       #211
      01000887H   LINE      CODE     ---       #212
      0100088AH   LINE      CODE     ---       #213
      0100088AH   LINE      CODE     ---       #215
      0100089EH   LINE      CODE     ---       #216
      010008A1H   LINE      CODE     ---       #217
      010008AAH   LINE      CODE     ---       #218
      010008AAH   LINE      CODE     ---       #219
      010008ACH   LINE      CODE     ---       #221
      010008B4H   LINE      CODE     ---       #222
      010008BCH   LINE      CODE     ---       #223
      010008C4H   LINE      CODE     ---       #224
      010008CCH   LINE      CODE     ---       #225
      010008CFH   LINE      CODE     ---       #226
      010008CFH   LINE      CODE     ---       #227
      010008D1H   LINE      CODE     ---       #228
      010008D1H   LINE      CODE     ---       #230
      010008E5H   LINE      CODE     ---       #231
      010008E8H   LINE      CODE     ---       #233
      010008F1H   LINE      CODE     ---       #234
LX51 LINKER/LOCATER V4.66.41.0                                                        06/16/2023  10:23:34  PAGE 75


      010008F1H   LINE      CODE     ---       #235
      010008F3H   LINE      CODE     ---       #236
      010008F3H   LINE      CODE     ---       #237
      010008F5H   LINE      CODE     ---       #238
      010008F5H   LINE      CODE     ---       #240
      01000909H   LINE      CODE     ---       #241
      0100090CH   LINE      CODE     ---       #243
      01000915H   LINE      CODE     ---       #244
      01000915H   LINE      CODE     ---       #245
      01000917H   LINE      CODE     ---       #246
      01000917H   LINE      CODE     ---       #247
      01000917H   LINE      CODE     ---       #248
      01000917H   LINE      CODE     ---       #250
      0100091AH   LINE      CODE     ---       #251
      ---         BLOCKEND  ---      ---       LVL=0

      ---         MODULE    ---      ---       ?C_INIT
      01000C0EH   PUBLIC    CODE     ---       ?C_START

      ---         MODULE    ---      ---       ?C?COPY
      01000156H   PUBLIC    CODE     ---       ?C?COPY

      ---         MODULE    ---      ---       ?C?CLDPTR
      0100017CH   PUBLIC    CODE     ---       ?C?CLDPTR

      ---         MODULE    ---      ---       ?C?CLDOPTR
      01000195H   PUBLIC    CODE     ---       ?C?CLDOPTR

      ---         MODULE    ---      ---       ?C?CILDPTR
      010001C2H   PUBLIC    CODE     ---       ?C?CILDPTR

      ---         MODULE    ---      ---       ?C?CSTPTR
      010001E4H   PUBLIC    CODE     ---       ?C?CSTPTR

      ---         MODULE    ---      ---       ?C?CSTOPTR
      010001F6H   PUBLIC    CODE     ---       ?C?CSTOPTR

      ---         MODULE    ---      ---       ?C?IMUL
      01000218H   PUBLIC    CODE     ---       ?C?IMUL

      ---         MODULE    ---      ---       ?C?UIDIV
      0100022AH   PUBLIC    CODE     ---       ?C?UIDIV

      ---         MODULE    ---      ---       ?C?ILDIX
      0100027FH   PUBLIC    CODE     ---       ?C?ILDIX

      ---         MODULE    ---      ---       ?C?ULDIV
      010002D1H   PUBLIC    CODE     ---       ?C?ULDIV

      ---         MODULE    ---      ---       ?C?ULCMP
      01000363H   PUBLIC    CODE     ---       ?C?ULCMP

      ---         MODULE    ---      ---       ?C?LSTXDATA
      01000374H   PUBLIC    CODE     ---       ?C?LSTXDATA

      ---         MODULE    ---      ---       ?C?LSTKXDATA
      01000380H   PUBLIC    CODE     ---       ?C?LSTKXDATA

      ---         MODULE    ---      ---       ?C?LIMUL
      010003B1H   PUBLIC    CODE     ---       ?C?LIMUL

      ---         MODULE    ---      ---       PRINTF
      02000000H   PUBLIC    XDATA    ---       ?_PRINTF517?BYTE
      02000000H   PUBLIC    XDATA    ---       ?_PRINTF?BYTE
      02000000H   PUBLIC    XDATA    ---       ?_SPRINTF517?BYTE
LX51 LINKER/LOCATER V4.66.41.0                                                        06/16/2023  10:23:34  PAGE 76


      02000000H   PUBLIC    XDATA    ---       ?_SPRINTF?BYTE
      0100048FH   PUBLIC    CODE     ---       _PRINTF
      0100048FH   PUBLIC    CODE     ---       _PRINTF517
      01000489H   PUBLIC    CODE     ---       _SPRINTF
      01000489H   PUBLIC    CODE     ---       _SPRINTF517

      ---         MODULE    ---      ---       ?C?PLDIXDATA
      010003DEH   PUBLIC    CODE     ---       ?C?PLDIXDATA

      ---         MODULE    ---      ---       ?C?PSTXDATA
      010003F5H   PUBLIC    CODE     ---       ?C?PSTXDATA

      ---         MODULE    ---      ---       ?C?CCASE
      010003FEH   PUBLIC    CODE     ---       ?C?CCASE



FUNCTION REGISTER MASKS


FUNCTION . . . . . . . . . . . . REG MASK
==========================================

_adc_sampling_continuous . . . . @0x1e000cfd
_change_duty_pwm0_cpm. . . . . . @0x18000cfd
_change_duty_pwm0_idp. . . . . . @0x1e000880
_change_duty_pwm1_cpm. . . . . . @0x18000cfd
_change_duty_pwm1_idp. . . . . . @0x1e000880
_change_duty_pwm2_cpm. . . . . . @0x18000cfd
_change_duty_pwm2_idp. . . . . . @0x1e000880
_config_pwm0_module. . . . . . . @0x1e000800
_config_pwm1_module. . . . . . . @0x1e000800
_config_pwm2_module. . . . . . . @0x1e000800
_config_uart1_module . . . . . . @0x1e000800
_debug_putchar . . . . . . . . . @0x0e000800
_delay_ms. . . . . . . . . . . . @0x180008f0
_delay_ms_int. . . . . . . . . . @0x1e000800
_delay_us. . . . . . . . . . . . @0x18000880
_flash_erase_sector. . . . . . . @0x08000800
_flash_read_multi_byte . . . . . @0x1e000866
_flash_write_multi_byte. . . . . @0x1e0008f6
_flash_write_one_byte. . . . . . @0x08000800
_hd_crc_calculate. . . . . . . . @0x1e0008c6
_HS6220_Bank_Switch. . . . . . . @0x1e0008f8
_HS6220_Change_Addr. . . . . . . @0x1e000cef
_HS6220_Change_CH. . . . . . . . @0x1e0008f0
_HS6220_Change_Pwr . . . . . . . @0x1e0008f8
_HS6220_Change_Rate. . . . . . . @0x1e0008f8
_HS6220_ModeSwitch . . . . . . . @0x1e0008fc
_HS6220_Operation. . . . . . . . @0x1e0008e0
_HS6220_read_buffer. . . . . . . @0x1e000cff
_HS6220_read_byte. . . . . . . . @0x1e0008f0
_HS6220_wr_buffer. . . . . . . . @0x1e000cef
_HS6220_wr_cmd . . . . . . . . . @0x1e0008f0
_HS6220_write_byte . . . . . . . @0x1e0008f0
_Iic_Master_ReadData . . . . . . @0x1e00084f
_Iic_Master_SendData . . . . . . @0x1e00084f
_putchar . . . . . . . . . . . . @0x0e0008a0
_SPI_3wire_sendByte. . . . . . . @0x1e0008e0
_spi_master_read . . . . . . . . @0x1e00084f
_spi_master_write. . . . . . . . @0x1e00084f
_SPI_SendByte. . . . . . . . . . @0x1e0008e0
_turn_off_pwm0 . . . . . . . . . @0x1e000800
_turn_off_pwm1 . . . . . . . . . @0x1e000800
_turn_off_pwm2 . . . . . . . . . @0x1e000800
LX51 LINKER/LOCATER V4.66.41.0                                                        06/16/2023  10:23:34  PAGE 77


_turn_on_pwm0_cpm. . . . . . . . @0x1e000cfd
_turn_on_pwm0_idp. . . . . . . . @0x1e000880
_turn_on_pwm1_cpm. . . . . . . . @0x1e000cfd
_turn_on_pwm1_idp. . . . . . . . @0x1e000880
_turn_on_pwm2_cpm. . . . . . . . @0x1e000cfd
_turn_on_pwm2_idp. . . . . . . . @0x1e000880
_turn_on_pwm3. . . . . . . . . . @0x0e000800
_uart1_tx_byte . . . . . . . . . @0x08000800
_uart1_tx_data . . . . . . . . . @0x1e00084f
_uart1_tx_data_start . . . . . . @0x1e00080e
_user_printf . . . . . . . . . . @0x1e000c8f
adc_rpt. . . . . . . . . . . . . @0x80000000
adc_sampling_single. . . . . . . @0x080008c0
config_adc_module. . . . . . . . @0x0e000800
config_gpio_ext_int. . . . . . . @0x0e000800
config_gpio_power_on . . . . . . @0x0e000800
config_iic_master_module . . . . @0x0e000800
config_iic_slave_module. . . . . @0x0e000800
config_pwm3_module . . . . . . . @0x0e000800
config_spi_master_module . . . . @0x0e000800
config_spi_slave_module. . . . . @0x0e000800
config_sysclk_crystal_module . . @0x1e000880
config_sysclk_ihrc_module. . . . @0x1e000880
config_sysclk_output . . . . . . @0x0e000800
config_timer0_module . . . . . . @0x0e000800
config_timer1_module . . . . . . @0x0e000800
config_timer3_module . . . . . . @0x0e000800
config_timer4_module . . . . . . @0x0e000800
config_timer5_module . . . . . . @0x0e000800
debug_init . . . . . . . . . . . @0x0e000800
debug_rpt. . . . . . . . . . . . @0x1e0008c0
disable_watchdog . . . . . . . . @0x0e000800
enable_watchdog. . . . . . . . . @0x0e000800
enable_watchdog_for_stop . . . . @0x0e000800
feed_watchdog. . . . . . . . . . @0x80000000
hardware_init. . . . . . . . . . @0x1e000880
HS6220_CE_High . . . . . . . . . @0x1e0008e0
HS6220_CE_Low. . . . . . . . . . @0x1e0008e0
HS6220_Clear_All_Irq . . . . . . @0x1e0008f0
HS6220_Flush_Rx. . . . . . . . . @0x1e0008e0
HS6220_Flush_Tx. . . . . . . . . @0x1e0008e0
HS6220_read_payload_length . . . @0x1e0008f0
HS6220_SPI_Init. . . . . . . . . @0x0e000800
IIC_Rpt. . . . . . . . . . . . . @0x1e000880
int0_rpt . . . . . . . . . . . . @0x80000000
int1_rpt . . . . . . . . . . . . @0x80000000
int2_7_rpt . . . . . . . . . . . @0x80000000
int8_15_rpt. . . . . . . . . . . @0x80000000
pwm_rpt. . . . . . . . . . . . . @0x08000800
reset_check. . . . . . . . . . . @0x08000800
SPI_3wire_readByte . . . . . . . @0x1e0008d0
SPI_ReadByte . . . . . . . . . . @0x1e0008d0
SPI_Rpt. . . . . . . . . . . . . @0x1e0008cf
system_flow_control. . . . . . . @0x1e0008bc
system_power_down. . . . . . . . @0x1e000880
task_key_scan. . . . . . . . . . @0x1e0008c0
timer0_service . . . . . . . . . @0x0e000800
timer1_service . . . . . . . . . @0x80000000
timer3_service . . . . . . . . . @0x1e000800
timer4_service . . . . . . . . . @0x80000000
timer5_service . . . . . . . . . @0x1e000800
turn_off_pwm3. . . . . . . . . . @0x0e000800
uart1_rpt. . . . . . . . . . . . @0x1e0008cf
user_gpio_initial. . . . . . . . @0x0e000800
user_key_pro . . . . . . . . . . @0x1e0008bc
LX51 LINKER/LOCATER V4.66.41.0                                                        06/16/2023  10:23:34  PAGE 78


user_register_initial. . . . . . @0x0e000800
wdt_rpt. . . . . . . . . . . . . @0x80000000

Program Size: data=16.1 xdata=312 const=0 code=4678
LX51 RUN COMPLETE.  0 WARNING(S),  0 ERROR(S)
